:100000000C94320B0C94630B0C94630B0C94630BE9
:100010000C94630B0C94630B0C94630B0C94630BA8
:100020000C94630B0C94630B0C94630B0C94630B98
:100030000C94630B0C94B4120C94630B0C94630B30
:100040000C94630B0C94630B0C94630B0C94630B78
:100050000C94630B0C94630B0C94630B0C942FA9FE
:100060000C94630B0C94BF9B0C94959B0C94630BAA
:100070000C94630B0C94630B0C94630B0C94630B48
:100080000C94630B0C94630B0C94630B0C94630B38
:100090000C946B9B0C94419B0C94630B0C943F143D
:1000A0000C94630B0C94630B0C94630B0C94630B18
:1000B0000C94630B0C94630B0C94630B0C94630B08
:1000C0000C94630B0C94630B0C94630B0C94179BB4
:1000D0000C94ED9A0C94630B0C94C39A0C94999A1B
:1000E0000C94630B084AD73B3BCE016E84BCBFFD2A
:1000F000C12F3D6C74319ABD56833DDA3D00C77FF8
:1001000011BED9E4BB4C3E916BAAAABE0000008090
:100110003F07634236B79BD8A71A39685618AEBA5C
:10012000AB558C1D3CB7CC5763BD6DEDFD753EF6F0
:10013000177231BF000000803F08000000BE92240B
:1001400049123EABAAAA2ABECDCCCC4C3E00000040
:1001500080BEABAAAAAA3E00000000BF000000803B
:100160003F0000000000084178D3BB4387D1133D16
:10017000190E3CC3BD4282AD2B3E68EC8276BED9DF
:100180008FE1A93E4C80EFFFBE01C4FF7F3F00001E
:10019000000000000C94AD0B0C94CD7E0C94638990
:1001A0000C942C730C94C0720C943A890C944F8963
:1001B0000C94CD880C94878A0C94FD0B0C94678961
:1001C0000C94DC830C9431860C94EB730C94628752
:1001D0000C94650B0C946B890C94040D0C94718930
:1001E0000C946D790C9447730C94717E0C949977F0
:1001F0000C9452820C947C860C94CA7E0C94867E5D
:100200000C94B2870C94C9720C944B890C94088896
:100210000C94A8840C941C880C94897E0C9470898E
:100220000C94E2730C941B730C9479800C943089B9
:100230000C94010D0C94B3870C945D890C94AB0B5A
:100240000C943E890C9436890C9475890C947286B2
:100250000C94BD0B0C94F9870C9459890C948475FB
:100260000C94E3720C9445890C949D120C940A76BC
:100270000C9492860C9480880C94C7860C941F7DF5
:100280000C9471AA0C94AE0B0C94BF860C9436821D
:100290000C9455890C94D00B0C9470830C94D272EE
:1002A0000C94B7720C941C7E0C94108A0C942A85C2
:1002B0000C946C0B0C942F0C0C9479890C94357362
:1002C0000C94080D0C94AC0B0C9492770C942A8827
:1002D0000C94207A0C940B720C9432850C94428905
:1002E0000C9419750C94487B0C9477860C942C0C08
:1002F0000C943E730C94A2720C94F4730C94BEA9EB
:100300000C94EC724E414E494E495459494E46CDDB
:10031000CCCC3D0AD7233C17B7D13877CC2B3295BC
:1003200095E6241FB14F0A000020410000C842009A
:10033000401C4620BCBE4CCA1B0E5AAEC59D740064
:10034000407A10F35A00A0724E18090010A5D4E8A4
:100350000000E87648170000E40B54020000CA9A37
:100360003B000000E1F50500008096980000004089
:10037000420F000000A086010000001027000000CE
:1003800000E803000000006400000000000A000014
:100390000000000100000000002C76D888DC674FC8
:1003A0000823DFC1DFAE59E1B1B796E5E3E453C6F8
:1003B0003AE651997696E8E6C28426EB898C9B62F0
:1003C000ED407C6FFCEFBC9C9F40F2BAA56FA5F49A
:1003D00090055A2AF75C936B6CF9676DC11BFCE0C2
:1003E000E40D47FEF520E6B500D0ED902E03009415
:1003F0003577050080841E080000204E0A000000AA
:10040000C80C333333330F986E12831141EF8D21B3
:1004100014893BE65516CFFEE6DB18D1844B381B1A
:10042000F77C1D901DA4BBE424203284725E2281DF
:1004300000C9F124ECA1E53D274E6F2073656E7372
:100440006F72210049522054656D70657261747538
:100450007265004D6561737572696E672E2E004E70
:100460006F2073656E736F723F0049522054656D43
:100470007065726174757265004D6561737572693E
:100480006E672E2E004E6F2053656E736F722100C3
:100490004E6F20445320546865726D6F6D657465AE
:1004A000722100445320546865726D2E004D6F74A4
:1004B000696F6E0046696E64696E672057694669A8
:1004C000204950007365703D006976616C3D006E97
:1004D000697465723D00230043616C2E204661699A
:1004E0006C65640043616C2E20446F6E65004E6F36
:1004F000206E6565642100496E76616C69642050E8
:1005000028506129005365614C6576656C20502840
:100510005061293A0043616C6962726174652050D0
:10052000004169722054656D70286F43293A004379
:10053000616C2E204D6F74696F6E004453542054CB
:10054000656D702073656E736F72004375727265AE
:100550006E742073656E736F72004F322073656E18
:10056000736F720055562073656E736F720043612E
:100570006C696272617465004661696C65640054FF
:10058000422063616C2E20646F6E6500557070654B
:1005900072204C696D69743A3E004C6F7765722029
:1005A0004C696D69743A3E0054757262696469748D
:1005B00079004661696C65640070482063616C2E47
:1005C00020646F6E6500704831302050726573731F
:1005D00020420070483420507265737320410043FC
:1005E000616C696272617465004E45543D426C7580
:1005F00065746F6F7468204C45004E45543D426CE5
:100600007565746F6F7468004E45543D576946694F
:100610000053657474696E67204661696C65640097
:1006200053657474696E6720446F6E65004368613A
:100630006E6765204E6574776F726B3E00547970FB
:10064000653A0042542F57694669204E6574776FAA
:10065000726B004368616E67652053656E736F72DD
:100660003E0043757272656E742053656E736F72CF
:10067000004F7468657200496E642E20342D32304C
:100680006D4100414353373132203C33304100410A
:100690004353373132203C323041004143533731EC
:1006A00032203C3541003E4D617820566F6C743AE3
:1006B0003E004368616E676520766F6C74616765A4
:1006C0003E00547970652000566F6C746167652038
:1006D00053656E736F72004368616E67652074794D
:1006E000706520746F0053656E736F723D4448549B
:1006F0000054656D702048756D69646974790020D7
:1007000028303D6175746F3B313D616363656C3BBF
:10071000323D696E636C20616E676C652900234110
:100720003D00556E6B6E6F776E00496E6475737425
:100730007269616C20342D32306D41004143533772
:100740003132204D61783D35410023437572726529
:100750006E742073656E736F723A00696E70757493
:100760002044535463616C6962726174653A00207D
:10077000766F6C746167653D0023547572626964BD
:10078000697479205570706572204C696D69743A8E
:10079000200020766F6C746167653D00235475728C
:1007A000626964697479204C6F776572204C696D59
:1007B00069743A20002354757262696469747920FF
:1007C0004C6F776572204C696D69742056696E664E
:1007D0003A20004D61782072616E67653D002356B6
:1007E0006F6C746167652073656E736F723A003465
:1007F0002D32306D4100414353373132204D617805
:100800003D00414353373132204D61783D35410041
:100810002343757272656E742073656E736F723ADE
:100820000023445320546865726D6F6D6574657262
:100830002063616C6962726174656420666F722006
:10084000230044535400234E6F206E65656420746A
:100850006F2063616C696272617465206375727286
:10086000656E742073656E736F722100234143536C
:100870003731322063757272656E742073656E73E2
:100880006F72206F666673657420563D002355565F
:10089000207A65726F20766F6C74616765203D0009
:1008A00055565A00234F3220766F6C253D00234F5A
:1008B000322063616C6962726174696F6E3A200004
:1008C00023566F6C746167652870483D3130293A52
:1008D0000023566F6C746167652870483D34293A6F
:1008E00000504834005554454D503D004448543D57
:1008F00000413D002354696D65206475726174691F
:100900006F6E3D002354696D6520696E7465727663
:10091000616C3D00576946692049503A00234D53A8
:1009200020456E61626C656400234D5320446973F9
:1009300061626C656400235265737420706172613A
:100940006D657465727320746F2064656661756C83
:10095000742076616C756573004C6F6767657220F3
:100960004E616D653A2000697465726174696F6EDD
:100970003D0073656E736F72233D0043757272653F
:100980006E74207374617475733A206379636C6557
:100990003D006E6379636C653D006E73656E736FC9
:1009A00072733D006D61786E73656E736F72733D27
:1009B00000656E61626C65643D00234D756C746901
:1009C00073656E736F7273206D6561737572656D9B
:1009D000656E742073657474696E67733A0023538F
:1009E000657474696E6773206F6620616C6C207328
:1009F000656E736F72733A002353697A65206F6670
:100A000020686561646572202B20616C6C207365C1
:100A10006E736F72733A20002353697A65206F6694
:100A2000206865616465723A20004F6666206169DE
:100A3000722D636F6E6421004974277320746F6F89
:100A400020636F6F6C210054656D702069732066A0
:100A5000696E6521004973206169722D636F6E6450
:100A6000206F6E3F0049742773207175697465208B
:100A7000686F742100497427732076657279206845
:100A80006F742120004F6666206169722D636F6E5E
:100A90006421004974277320746F6F20636F6F6C3B
:100AA000210054656D702069732066696E652100B0
:100AB0004973206169722D636F6E64206F6E3F0011
:100AC0004974277320717569746520686F742100FB
:100AD00049742773207665727920686F74210054F9
:100AE000656D702048756D696469747900232061B3
:100AF0006E6420726561647920746F20757365215E
:100B000000206D6F62696C65206C6F67676572208D
:100B100073746172746564200043616C6962726110
:100B200074696F6E2050726573737572653D005302
:100B30006561206C6576656C20502863616C632963
:100B40003D00234572726F723A70726573737572ED
:100B50006520424D503038352C20636865636B202A
:100B6000776972696E67210049522054656D702063
:100B700073656E736F7220666F756E6400206D6FA3
:100B800062696C65206C6F6767657220737461724F
:100B9000746564202E2E2E20005769466920495026
:100BA0003A002357694669204950206164647265A0
:100BB00073733A2000456455484B205345534C6F9E
:100BC000676765720053656E736F7220736C6F7424
:100BD00020616E6420747970653A0057656C636FAC
:100BE0006D6520746F20456455484B00005EBCE283
:100BF000613FDD83C29C7E20A3FD1F41009D23BE7B
:100C000046DB65F88C11AF32CA57E974232D2D2DC0
:100C10002D2D2D2D2D2D2D2D2D2D2D2D2D2D2D2D04
:100C20002D2D2D2D2D2D2D2D2D2D2D2D2D2D2D2DF4
:100C30002D00235265736F6C7574696F6E3A2020B6
:100C40002000234D696E2056616C75653A20202086
:100C50002000234D61782056616C75653A20202074
:100C6000200023556E697175652049443A20202083
:100C7000200023447269766572205665723A2020FE
:100C800020002353656E736F723A202020202020AD
:100C90002000232D2D2D2D204D61676E6574696315
:100CA0002053656E736F72202D2D2D2D2D2D2D2D22
:100CB0002D2D2D2D2D2D2D2D2D2D2D2D00482D663D
:100CC00069656C643A202800202020202020202004
:100CD0002020202020202020002020202020202034
:100CE0002020202020202020200020202020202024
:100CF0002020202020202020202000202020202014
:100D00002020202020202020202020002020202003
:100D100020202020202020202020200020202020F3
:100D2000202020202020202020202000233A53684B
:100D30006F772F48696465204C4344002A3A546811
:100D400069732048656C700044233A43616C6962A2
:100D5000726174696F6E00442A3A53657474696EE7
:100D600067730044423A5265736574204C6F67673D
:100D700065720044433A436C656172204C43440001
:100D800044443A4D756C746953656E736F727300A9
:100D900044393A43757272656E7400566F6C7461B3
:100DA00067652B43757272656E740044383A456C02
:100DB0006563747269630044373A4D6F74696F6E8E
:100DC0000044363A44532054656D700044353A551A
:100DD0005620496E74656E736974790044343A4FD5
:100DE0003220636F6E632E0044333A434F322063E8
:100DF0006F6E632E0044323A504D28313A322E3510
:100E00003A3130290044323A504D28313A322E35A9
:100E10003A3130292A0044313A5475726269646962
:100E200074790044303A566F6C7461676500393AE2
:100E30006F7220334420616363656C2E00393A4938
:100E40006E636C2E20616E672E00383A70482076F3
:100E5000616C756500373A49522054656D700037F2
:100E60003A49522054656D702A00363A4D61676EDA
:100E700065746963206669656C6400353A4761731F
:100E8000204C6576656C00343A495220466C616DA1
:100E90006500333A4C6967687420496E742E0032DD
:100EA0003A616E642048656967687400323A546537
:100EB0006D7020507265737375726500313A5465B8
:100EC0006D702048756D696469747900303A536FAC
:100ED000756E64204C6576656C00303A536F756EA4
:100EE00064204C6576656C2A0054696D65206C61E0
:100EF0007073653A00576946692049503A004D6F52
:100F000074696F6E00555620496E742E0055562038
:100F1000496E74656E73697479004F3220436F6E49
:100F20006300434F3220436F6E630053656E736FEF
:100F300072206572726F722100234E6F2073656E8E
:100F4000736F722100434F3220436F6E63004D6513
:100F500061737572696E6700234E6F2073656E73DF
:100F60006F7220666F7220504D21004E6F207365A6
:100F70006E736F722100206E672F4C00504D313A16
:100F8000322E353A3130004D6561737572696E6786
:100F90002E2E00234E6F2054422073656E736F72A5
:100FA0003F00234E6F2073656E736F722100536F85
:100FB000756E64204C6576656C004D656173757265
:100FC000696E672E2E00234E6F2073656E736F72ED
:100FD0002100536F756E64204C6576656C00234E5E
:100FE0006F2073656E736F7220666F722074656D0B
:100FF0007020262068756D696469747921004E6FD0
:101000002053656E736F72210020666F72207465C5
:101010006D7020262068756D6964697479210023DC
:1010200053656E736F72204572726F722000536544
:101030006E736F72204572726F7221002357726F48
:101040006E672073656E736F7220666F72207465B1
:101050006D7020262068756D696469747921005768
:10106000726F6E672053656E736F72210054656DE9
:10107000702048756D6964697479004C696768749B
:1010800020496E74656E7369747900466C616D6594
:1010900020495200482D6669656C64005365617291
:1010A000636820446972656374696F6E00234E6FD4
:1010B0002070482073656E736F722100704820762F
:1010C000616C75650023496E76616C6964206B659F
:1010D000792100204D756C746973656E736F72733E
:1010E000004D756C746973656E736F72730044693B
:1010F0007361626C6500456E61626C650052656289
:101100006F6F74696E672E2E2E002344413A2D3284
:101110003300237265706C6965733D0067657453B5
:10112000656C665465737442697428293A200069B5
:1011300073496E74657272757074456E61626C6528
:10114000642831293A2000676574496E74657272AB
:101150007570744D617070696E672831293A20008E
:10116000676574496E74657272757074536F7572C9
:1011700063652831293A2000676574496E74657289
:1011800072757074536F7572636528293A20006711
:1011900065745261746528293A20332E3134313513
:1011A000393F00616363656C2E69734C6F77506FD4
:1011B00077657228293A2000616363656C2E697334
:1011C00041736C65657028293A2000616363656C22
:1011D0002E6973546170536F757263654F6E5A2830
:1011E000293A2000616363656C2E69735461705302
:1011F0006F757263654F6E5928293A2000616363E9
:10120000656C2E6973546170536F757263654F6EB0
:101210005828293A2000616363656C2E6973416325
:10122000746976697479536F757263654F6E5A2865
:10123000293A2000616363656C2E697341637469A8
:1012400076697479536F757263654F6E5928293AC0
:10125000200069734163746976697479536F75729C
:1012600063654F6E5828293A2000697354617044B1
:101270006574656374696F6E4F6E5A28293B2066EA
:10128000616C73653F2000697354617044657465D7
:101290006374696F6E4F6E5A28293B2074727565AE
:1012A0003F20006973546170446574656374696FAD
:1012B0006E4F6E5928293B2066616C73653F200094
:1012C0006973546170446574656374696F6E4F6EC1
:1012D0005928293B20747275653F20006973546159
:1012E00070446574656374696F6E4F6E5828293B4E
:1012F0002066616C73653F200069735461704465BA
:1013000074656374696F6E4F6E5828293B20747240
:1013100075653F20006765745375707072657373EF
:1013200042697428293B2066616C73653F20006721
:101330006574537570707265737342697428293BC4
:1013400020747275653F2000697341637469766922
:101350007479416328293A20006973496E61637486
:1013600069766974795A456E61626C656428293AB8
:1013700020006973496E61637469766974795945AF
:101380006E61626C656428293A20006973496E6158
:101390006374697669747958456E61626C65642816
:1013A000293A2000697341637469766974795A45F2
:1013B0006E61626C656428293A2000697341637428
:1013C000697669747959456E61626C656428293A59
:1013D00020006973416374697669747958456E6158
:1013E000626C656428293A200067657446726565F9
:1013F00046616C6C4475726174696F6E28293A207D
:10140000006765744672656546616C6C5468726508
:1014100073686F6C6428293A200067657454696D9D
:1014200065496E616374697669747928293A200088
:10143000676574496E61637469766974795468721A
:101440006573686F6C642829200067657441637454
:1014500069766974795468726573686F6C64282959
:101460002000676574446F75626C655461705769DC
:101470006E646F7728292000676574446F75626C0D
:10148000655461704C6174656E637928293A200057
:101490006765745461704475726174696F6E282950
:1014A0003A2000676574417869734F6666736574A6
:1014B0002826782C2026792C20267A293A200067A5
:1014C00065745461705468726573686F6C64282920
:1014D0003A200058595A2047733A200058595A2048
:1014E000434F554E54533A20007365742067616929
:1014F0006E735B5D3A006761696E735F6F726967F7
:101500005B5D3A00416E676C65732F00496E636CDA
:101510002E20616E672E0000002100240027002A83
:10152000002D003000330001010000040107010A12
:101530000100002200250028002B002E003100347D
:101540000002010000050108010B0100002000233A
:1015500000260029002C002F0032000001000003AB
:101560000106010901050505050705080808080227
:101570000202020A0A08080404040401010101012C
:101580000101010303030303030303040707070C1B
:101590000C0C0C0C0C0C0C020202020606060606D1
:1015A0000606060B0B0B0B0B0B0B0B01021020207E
:1015B00008081020401020408002010201080402A7
:1015C000010102040810204080804020100804021D
:1015D0000180040201804020100804020108040276
:1015E000010102040810204080010204081020407C
:1015F0008000000A0B02090C0D0E0807030401000D
:1016000000000000000000000000000000000000DA
:101610000000000000000000000000000012111097
:1016200000000000000000000000000000000000BA
:101630000000000000000023456E64206F66204D0E
:10164000756C746973656E736F72204379636C6532
:101650002300496E76616C6964206B657921000016
:1016600071AABEA911241FBECFEFD1E2DEBFCDBF4C
:1016700000E00CBF1BE0A0E0B2E0EEE5F9E701E01E
:101680000BBF02C007900D92AA3EB107D9F723E124
:10169000AAEEBBE001C01D92A23DB207E1F71BE03C
:1016A000C1E3DBE000E006C021970109802FFE01C5
:1016B0000E94CFB9C033D10780E00807A9F70E9484
:1016C000DBAC0C949DBC0C9400008091290D909192
:1016D0002A0D891B990B08950895DC0180E0615063
:1016E00090F09D919827E92FEF70F0E0E451F44FCE
:1016F0002491E92FE295EF70F0E0E450F44FE4918B
:10170000822F8E27ECCF08952091840C260F33274B
:10171000331F21323105ECF42091A30DFC0190E040
:1017200080E0243069F082E00895A091840C21913A
:10173000AC014C59534FA40FB52FB11D2C930196FA
:10174000861798F38091840C680F6093840C80E076
:10175000089581E00895089508950895E0912A0D6F
:101760008091290DE81730F4F0E0E75FF24F8081B7
:1017700090E008958FEF9FEF089590912A0D80914A
:10178000290D2FEF3FEF981748F4E92FF0E0E75FBE
:10179000F24F208130E09F5F90932A0DC901089598
:1017A000CF92DF92EF92FF920F931F93CF93DF932D
:1017B0007C01CB018A012091A90D222389F0EB0144
:1017C0006B01C40ED51ECC15DD0569F06991D701FA
:1017D000ED91FC910190F081E02DC7011995F3CFB7
:1017E000642F0E94840BC801DF91CF911F910F914C
:1017F000FF90EF90DF90CF900895CF93DF931F92EB
:10180000CDB7DEB769832091A90D2223F9F020918D
:10181000CB0D203258F021E030E0FC0133832283ED
:1018200090E080E00F90DF91CF9108958091AA0D14
:10183000E82FF0E0E555F24F998190838F5F809318
:10184000AA0D8093CB0D81E090E0ECCF61E0CE015A
:1018500001960E94840BF7CF90E080E00895AF924C
:10186000BF92CF92DF92EF92FF920F931F93CF938D
:10187000DF938C01EB0184E2FB0111928A95E9F779
:101880008EE10E94D98A83E090E00E94D48A0E946F
:10189000B49D66E08EE10E94CC9D10922A0D80934B
:1018A000290D8630F0F30E94E08DA82E0E94E08D75
:1018B000B82E0E94E08DE82E0E94E08DF82E0E9446
:1018C000E08DC82E0E94E08DD82E60E07A2D6B2925
:1018D000072E000C880B990B0E94ABB4F8016583AE
:1018E00076838783908760E07C2D6D29072E000C1E
:1018F000880B990B0E94ABB4F801618772878387CC
:10190000948760E07E2D6F29072E000C880B990BC1
:101910000E94ABB4F801658776878787908B118A20
:10192000128A138A148A84E290E0A0E0B0E08883EF
:101930009983AA83BB8385899689A789B08D8C8377
:101940009D83AE83BF8382E090E0A0E0B0E0888713
:101950009987AA87BB87188A198A1A8A1B8AC09016
:10196000E204D090E304E090E404F090E504A701E1
:10197000960165817681878190850E9423B720E05A
:1019800030E048EC52E40E940AB56C8B7D8B8E8B64
:101990009F8BA7019601F8016185728583859485E7
:1019A0000E9423B720E030E048EC52E40E940AB5E0
:1019B000688F798F8A8F9B8F2091DE043091DF04AE
:1019C0004091E0045091E104F801658576858785B2
:1019D00090890E9423B720E030E048EC52E40E9456
:1019E0000AB56C8F7D8F8E8F9F8F81E0DF91CF91B5
:1019F0001F910F91FF90EF90DF90CF90BF90AF902D
:101A00000895862F0C94E99B862F642F0C94129CCA
:101A1000862F642F0C94409C1F93CF93DF93EC018F
:101A2000162F60E0812F0E94409C612F70E0FB0127
:101A3000E555FA4EE491E883FB01EB59FA4EE49147
:101A4000F0E0EE0FFF1FE55BFA4E859194919A83CB
:101A500089831B861D861C861A86198618861F8216
:101A60001E821D821C821B82DF91CF911F910895DF
:101A7000EEE1F1E114A215A216A217A210A611A67A
:101A800012A613A681E084A729E130E036A725A796
:101A900087A780E090E0A0EAB0E480AB91ABA2AB76
:101AA000B3AB80E090E0A8EAB1E484AB95ABA6AB21
:101AB000B7AB8093DA049093DB04A093DC04B0937B
:101AC000DD0480E090E0A0E8BFE38093681190938C
:101AD0006911A0936A11B0936B118093D60490930F
:101AE000D704A093D804B093D90410929511109202
:101AF00094118BE090E090939711809396119093BE
:101B0000D5048093D4041092A5111092A41190E0F2
:101B100080E00C944B8D2F923F924F925F926F9288
:101B20007F928F929F92AF92BF92CF92DF92EF926D
:101B3000FF920F931F93CF93DF936C01CBE3D5E01C
:101B400085E9882E84E0982E0EE111E1EE24E394DD
:101B5000F12C22E1222E312C33E1432E512C40E195
:101B6000642E712C51E1A52EB12C80919504909199
:101B700096048E159F050CF4C9C021E0C216D1044D
:101B800009F0BDC0F80182AD93ADF4019383828367
:101B9000F40182819381009709F58A819B8190935A
:101BA000050280930402F4018281938184309105BF
:101BB000C1F52A813B8130930702209306028531CB
:101BC000910509F47BC08631910509F040C02A8156
:101BD0003B8130937C0420937B044EC0813091057F
:101BE00039F48A819B819093890480938804DBCFA8
:101BF0008230910539F48A819B819093030280930E
:101C00000202D1CF039779F68A819B8190930102DA
:101C10008093000264ED7BE089E093E10E942A95C5
:101C2000C2CF8530910539F42A813B8130937A0403
:101C300020937904C4CF8630910529F2873091052D
:101C4000B9F42A813B813093800420937F0487314B
:101C5000910591F42A813B8128303105B1F57092CC
:101C6000910460929004B0928F04A0928E0404C0FC
:101C70008A30910509F0A3CF9C012B5031092A30FD
:101C8000310590F42A813B813093010220930002B8
:101C900039E1389FB001399F700D1124685F7D4F85
:101CA00089E093E10E948D958FEFE81AF80A229659
:101CB000E2E08E0E911C0E5F1F4F57CF2A813B81B1
:101CC00030937E0420937D04D7CF2730310549F42B
:101CD000309291042092900450928F0440928E048E
:101CE000CBCF2630310541F621E030E0309391042E
:101CF0002093900410928F0410928E04BDCFF401B3
:101D000082819381F80193AF82AF42CFDF91CF916F
:101D10001F910F91FF90EF90DF90CF90BF90AF9009
:101D20009F908F907F906F905F904F903F902F90FB
:101D300008950F931F93CF93DF938C011092EB0BB9
:101D40001092EA0BC091EA0BD091EB0BC832D1058F
:101D5000A4F4809106020E947C9CCC0FDD1FC35D21
:101D6000D24F998388838091EA0B9091EB0B019677
:101D70009093EB0B8093EA0BE5CF0E94218B20E040
:101D800030E040EA50E40E940AB520E030E040E84C
:101D90005AE30E940AB50430110599F420E030E0BE
:101DA00040E650E40E940AB59B01AC0160E070E09F
:101DB00080E890E40E9444B6DF91CF911F910F918B
:101DC00008950A30110569F420E030E040E650E45F
:101DD0000E940AB59B01AC0160E070E080E291E4F2
:101DE000E9CF60E070E0CB01E7CF0F931F9360E095
:101DF000809190040E94129C83E090E00197F1F79B
:101E000061E0809190040E94129C83E290E001972F
:101E1000F1F760E0809190040E94129C80918E0402
:101E200090918F049927FC01E555FA4E6491FC01CD
:101E3000EB59FA4EE491F0E0EE0FFF1FE55BFA4E2E
:101E40008591949100E717E120E030E0462F0E9451
:101E500079A9611571058105910529F06F5F7F4FA3
:101E60008F4F9F4F9F700E94ABB420E030E44CE155
:101E700056E40E9423B72091080C3091090C409140
:101E80000A0C50910B0C0E940AB520E030E048E4A7
:101E900053E40E9423B71F910F910895DF92EF92B0
:101EA000FF920F931F93CF93DF937C018B01D42E6E
:101EB000DC011696ED91FC91138615861486128628
:101EC0001186108617821682158214821382C0E052
:101ED000B801F701868197810E949394D82F8823B7
:101EE00029F0DC1629F0CF5FDC1690F7D0E009C0AE
:101EF00067E0C8010E946D0BD80117969C91891369
:101F0000F2CF8D2FDF91CF911F910F91FF90EF9026
:101F1000DF900895DC012C911196ED91FC91F894DD
:101F20008181822B81839281322F309593239283FA
:101F300087E090E00197F1F781818323818383E239
:101F400090E00197F1F790817894EFECF0E0319711
:101F5000F1F7922381E009F480E00895FC0190817B
:101F60000180F281E02D292F209560FF14C0F894A4
:101F70008281822382838181892B8183A3E2B0E0E5
:101F80001197F1F78281982B9283789487ED90E0F6
:101F90000197F1F70895F8948281822382838181E9
:101FA000892B8183AFEFB0E01197F1F78281982BF5
:101FB000928378948FE090E0EBCFDF92EF92FF92E4
:101FC0000F931F93CF93DF93EC01D62EE42E08E0FE
:101FD00010E0FF24F39461E08D2D8F2109F460E07F
:101FE000CE010E94AE0FFF0C01501109A1F7E110C4
:101FF00010C0F894E981FA819181888180958923C4
:102000008183E981FA819281888180958923828305
:102010007894DF91CF911F910F91FF90EF90DF9017
:102020000895EF92FF920F931F93CF93DF938C014C
:102030007B0140E065E50E94DD0FE70188E0E80EE6
:10204000F11C699140E0C8010E94DD0FCE15DF054B
:10205000C1F7DF91CF911F910F91FF90EF900895FD
:10206000FC0190810180F281E02DF8948181292F7B
:1020700020958223818378943DE743E050E03150FE
:1020800029F1DA011197F1F780818923C1F3F894DE
:102090008281822382838181892B81837894ABE73B
:1020A000B7E01197F1F7F894818182238183A3E14E
:1020B000B1E01197F1F78081982381E009F080E089
:1020C0007894E3E6F6E03197F1F7089580E008951B
:1020D0008F929F92AF92BF92CF92DF92EF92FF9238
:1020E000CF93DF93EC018E819F810E94301040E0FE
:1020F0006CEC8E819F810E94DD0F488164E48E81AB
:102100009F810E94DD0F8A81882371F1E981E95066
:102110008EEEC82E82E0D82EE33038F4F0E0EE0FD9
:10212000FF1FED5AFA4FC080D1808B81882339F18F
:102130008881811124C00E948DA64B015C010D2C69
:10214000000CEE08FF088E819F810E948A0F81306B
:1021500059F00E948DA66C197D098E099F0968159A
:1021600079058A059B0578F3DF91CF91FF90EF9079
:10217000DF90CF90BF90AF909F908F900895B60161
:10218000DD0C880B990BDF91CF91FF90EF90DF90E2
:10219000CF90BF90AF909F908F900C94F19F6F92D3
:1021A0007F928F929F92AF92BF92CF92DF92EF92E7
:1021B000FF920F931F93CF93DF93EC017B018A0172
:1021C0008E819F810E943010811102C090E037C043
:1021D000B7018E819F810E94111040E06EEB8E81CD
:1021E0009F810E94DD0F7801680189E0C80ED11C33
:1021F000AE80BF8088E0882E912C712C6624639479
:10220000C5010E948A0F81117628660CE1E08E1AC2
:102210009108B1F7F70171927F01EC15FD0541F7C7
:102220008E819F810E943010813081F668E0C80164
:102230000E946D0B91E0F80120852813C7CF892FEC
:10224000DF91CF911F910F91FF90EF90DF90CF9092
:10225000BF90AF909F908F907F906F900895CF9395
:10226000DF9300D000D000D0CDB7DEB7AE014F5F16
:102270005F4F0E94CF10882331F08D818F33A9F0FA
:1022800020F48F31A1F080E007C08F3521F08F3727
:10229000D1F78CE001C08BE029960FB6F894DEBF31
:1022A0000FBECDBFDF91CF9108958AE0F5CF89E0D1
:1022B000F3CF0F931F93CF93DF93CDB7DEB7619723
:1022C0000FB6F894DEBF0FBECDBF8C01462FBE0106
:1022D000665F7F4F0E944E0F81110FC060E070E07B
:1022E0008EEF92EC61960FB6F894DEBF0FBECDBFB5
:1022F000DF91CF911F910F910895AE014F5F5F4F16
:10230000BE01665F7F4FC8010E94CF10882331F362
:102310006A8170E0762F6627770F770F770F298114
:1023200048E0249F90011124262B372B8A85803189
:10233000D1F4688570E08F81AB01481B5109CA0157
:102340009695982F8827979587950E94BBB9CB01C2
:102350004097B90153E0660F771F5A95E1F760780F
:102360009C01260F371F213854EE35070CF4B6CFE9
:10237000B901330F880B990B0E94ABB420E030E019
:1023800040E05CE30E940AB5ADCFEF92FF920F935D
:102390001F93CF93DF9300D000D01F921F92CDB731
:1023A000DEB78C01DC011696ED91FC911797138630
:1023B000158614861286118610861782168215825B
:1023C0001482138214961C92149715961C92EE2474
:1023D000E394BE016F5F7F4FF801868197810E9471
:1023E0009394882309F46FC067E0CE0101960E94A0
:1023F0006D0B98858913EDCFD8018C91811125C083
:1024000016968D919C910E943010BE016F5F7F4F98
:10241000F801868197810E94111040E064EBD80199
:1024200016968D919C910E94DD0FF801868197810F
:102430000E948A0FF82ED80116968D919C910E94C9
:102440003010F11002C0F801E082D8011196FC9022
:1024500089818031A1F1BE016F5F7F4FC8010E9469
:102460002F118F15D0F4F8018181D80111968C932A
:10247000119714968C9114978F5F14968C93898181
:10248000883231F0B0F4803119F0823209F0A1CFF6
:10249000F80185818F5F85839CCF8981803111F41C
:1024A0008CE0E3CFBE016F5F7F4FC8010E942F1108
:1024B000DCCF8B3369F3823409F08BCFE9CFFCE0BA
:1024C000FF1588F2EDCF28960FB6F894DEBF0FBE49
:1024D000CDBFDF91CF911F910F91FF90EF900895A5
:1024E0000F931F93CF938C01C62FFC0184810E9410
:1024F000D98AF80183858C2B90E00E94D48ACF91F1
:102500001F910F910C94B49D0F931F93CF938C0147
:10251000C62F0E9470126C2F6460C8010E94701256
:102520006C2F6B7FC8010E94701283EC90E00197C2
:10253000F1F7CF911F910F9108950F931F93CF93B0
:102540008C01C62F607F61600E94841280E1C89F69
:10255000B00111246160C8010E94841281E090E002
:10256000CF911F910F9108951F920F920FB60F9266
:1025700011240BB60F922F933F934F935F936F935A
:102580007F938F939F93AF93BF93EF93FF9380912C
:102590004D100E94E99B20915010309151102F5FF7
:1025A0003F4F309351102093501090914F1095361B
:1025B00018F096E090934C1090914C10943009F4E0
:1025C0006EC0F8F4923031F1933009F44CC0909120
:1025D0004E10992319F0811171C02F9AFF91EF913C
:1025E000BF91AF919F918F917F916F915F914F912B
:1025F0003F912F910F900BBE0F900FBE0F901F9029
:102600001895953009F457C0963009F791E09093EA
:102610001C114FC08111DBCF20915010309151100F
:102620002436310528F41092511010925010CFCF5B
:1026300010921C1110924F10E0914F1091E09E0FDC
:1026400090934F10F0E02091501030915110EE0F08
:10265000FF1FEE5AFF4E31832083109251101092CB
:10266000501093E019C0813009F0B1CFE0914F10C4
:1026700091E09E0F90934F10F0E020915010309118
:102680005110EE0FFF1FEE5AFF4E31832083109240
:1026900051101092501094E090934C1098CF8823D2
:1026A00059F220915010309151102536310508F41F
:1026B0008ECF95E0F1CF81118ACFB5CF2F988ECFF5
:1026C000CF92DF92EF92FF92CF93DF93EC01072E30
:1026D000000C880B990B0E94ABB46B017C0120E0CD
:1026E00030E040E45FE30E940AB520E030E048E4D7
:1026F00052E40E9423B70E94CFB7C617D707D4F081
:1027000020E030E040EA5FE3C701B6010E940AB56D
:1027100020E030E048E452E40E9423B720E030E0BB
:1027200040E85FE30E9445B60E94CFB721E06C17F6
:102730007D070CF420E0822F90E0DF91CF91FF9095
:10274000EF90DF90CF9008950F931F93CF93DF9377
:10275000082F6BE87BE083EA9FE00E94539AC7E072
:10276000D0E010E0B8010C2E02C0759567950A9470
:10277000E2F76170772742E050E083EA9FE00E9431
:10278000069A219778F7DF91CF911F910F910895C5
:102790001092A30D81E08093A20D10927D0D61E057
:1027A00084E10E94129C61E085E10E94129CE9EBA9
:1027B000F0E080818E7F808380818D7F808388E4BC
:1027C0008093B80085E48093BC000895CF93DF9395
:1027D00091E09093630C8823B9F0C091B800D09138
:1027E000BA008091BC008A7B8093BC0060E084E1E9
:1027F0000E94129C60E085E10E94129C0E94C81316
:10280000D093BA00C093B800DF91CF91089585EDC1
:102810008093BC008091A50D9091A60DA091A70D6D
:10282000B091A80D0796A11DB11D23E0B695A795FF
:10283000979587952A95D1F72091BC0024FD03C078
:102840001092A30D08954091A50D5091A60D609191
:10285000A70D7091A80D452B462B472B69F30097C8
:10286000A105B10541F025E32A95F1F70000019794
:10287000A109B109E1CF8091A40D0C94E6131F9238
:102880000F920FB60F9211240BB60F922F933F9316
:102890004F935F936F937F938F939F93AF93BF9368
:1028A000EF93FF938091B900887F803609F44DC083
:1028B00008F040C0883209F4A9C028F5803109F435
:1028C0009DC0C8F4882309F4FBC0883009F496C081
:1028D000FF91EF91BF91AF919F918F917F916F91F8
:1028E0005F914F913F912F910F900BBE0F900FBEB4
:1028F0000F901F901895883109F488C0803241F7F5
:102900008093A10D14C0803409F49DC040F480333D
:10291000B9F38833E9F68093A10D85ECB0C080351A
:1029200009F485C0883509F496C0883489F60E9478
:102930000714CECF883909F48CC038F5883729F0D0
:1029400050F4883611F0803719F683E08093A30D98
:102950001092A60C57C0883809F47BC0803919F052
:10296000803809F0B5CF8091A60C803208F071C094
:10297000E091A60C81E08E0F8093A60C8091BB00A5
:10298000F0E0EA57F34F80833DC0803B39F0E0F43C
:10299000803A09F479C0883A09F09ACF84E08093AC
:1029A000A30D1092850C1092840CE091070DF0910C
:1029B000080D19958091840C81110FC081E08093DE
:1029C000840C1092640C09C0803C09F4A6CF883CAA
:1029D00009F4A3CF883B09F07BCFE091850C81E01F
:1029E0008E0F8093850CF0E0EC59F34F808180933B
:1029F000BB009091850C8091840C29C080917E0D44
:102A00008093BB0085EC8093BC0062CF9091A00DB9
:102A100080919F0D981758F5E091A00D81E08E0FE1
:102A20008093A00DF0E0E158F24F8081E9CFE09172
:102A3000A00D81E08E0F8093A00D8091BB00F0E08F
:102A4000E158F24F80839091A00D80919F0D9817CF
:102A5000C8F285E8D8CFE091A00D81E08E0F809379
:102A6000A00D8091BB00F0E0E158F24F808380918F
:102A7000A20D81115CCF81E080937D0D84EA80936B
:102A8000BC001092A30D24CF85EC8093BC00109263
:102A9000A30D8091A60C803230F4E091A60CF0E0FA
:102AA000EA57F34F10826091A60C70E0E091050D9B
:102AB000F091060D86E89CE019951092A60C08CFBF
:102AC0001092A10D34CF23E333E948E853E40E9488
:102AD00023B720E030E040E85FE30E9445B60E9463
:102AE0004DB926E636EA45EA53E40E940AB56093FA
:102AF000080C7093090C80930A0C90930B0C0895AA
:102B0000CF92DF92EF92FF920E94F50E6B017C0153
:102B100020E030E040E050E40E942CB8181624F485
:102B20000E94F50E6B017C0120E030E040E050E4B3
:102B3000C701B6010E942CB8181624F40E94F50EA5
:102B40006B017C0120E030E040E050E4C701B601B9
:102B50000E942CB8181624F40E94F50E6B017C011B
:102B600020E030E040E050E4C701B6010E942CB8FC
:102B7000181624F40E94F50E6B017C0120E030E071
:102B800040E050E4C701B6010E942CB818162CF49E
:102B9000C12CD12CE12C80E4F82EC701B601FF90A6
:102BA000EF90DF90CF90089581E08093E7048091CB
:102BB0008704882341F088E08093C11360E086EBAE
:102BC00093E10C947012089580918704811110C0D4
:102BD00081E0809387048093E7048091BC13982F51
:102BE00094609093BC138C600E94E38A0C94D4157B
:102BF0008091E7048823D1F31092C11360E086EB43
:102C000093E10E9470121092E7048091BC138B7FB5
:102C10008093BC1388600E94E38A10928704089511
:102C20002F923F924F925F926F927F928F929F92DC
:102C3000AF92BF92CF92DF92EF92FF920F931F93CA
:102C4000CF93DF93CDB7DEB766970FB6F894DEBFAC
:102C50000FBECDBF1C0186E09FE00E94C28D40E800
:102C600055E260E070E086E09FE00E94865864E6EE
:102C700070E080E090E00E94F19F8CED95E0A0E094
:102C8000B0E080930A0F90930B0FA0930C0FB093BA
:102C90000D0F64E670E080E090E00E94F19F8FEFFE
:102CA0008A8781E08B8786E88C871D861E861F8633
:102CB000188A198A89E78A8BC101880F991F9E8B10
:102CC0008D8BD12CC12CF12CE12C412C512C3201BB
:102CD00086E09FE00E94F98708974CF049E050E0B9
:102CE000BE01665F7F4F86E09FE00E94B38765E08C
:102CF00070E080E090E00E94F19F10E000E0812C05
:102D0000912C540186E09FE00E942A88892B39F497
:102D1000F4E08F169104A104B1040CF04EC002300F
:102D200011050CF04AC086E09FE00E942A88892B9A
:102D300069F086E09FE00E940888E1E0F0E0EC0F97
:102D4000FD1FE00FF11F80830F5F1F4F65E070E0F4
:102D500080E090E00E94F19F0230110509F073C0FD
:102D600099818A8598136FC09A818C8598136BC05E
:102D7000FE013396FC8BEB8B86E09FE00E942A8855
:102D8000892B39F4F4E08F169104A104B1040CF0FE
:102D900053C00930110509F05CC08B8190E0982F79
:102DA00088272C81820F911D092E000CAA0BBB0BCA
:102DB000480E591E6A1E7B1E43C08FEFC81AD80AE0
:102DC000E214F30434F4ED89FE89EC15FD0509F0F5
:102DD0007FCF86E09FE00E94C28DE114F10409F4E8
:102DE0007101C301B2010E94ABB44B015C01B70198
:102DF000FF0C880B990B0E94ABB49B01AC01C50181
:102E0000B4010E9423B766960FB6F894DEBF0FBEDA
:102E1000CDBFDF91CF911F910F91FF90EF90DF9089
:102E2000CF90BF90AF909F908F907F906F905F906A
:102E30004F903F902F900895043011050CF0ADCFC6
:102E4000FFEFEF1AFF0A8FEF881A980AA80AB80A4C
:102E500059CF86E09FE00E940888EB89FC89819326
:102E6000FC8BEB8B0F5F1F4F87CF4F925F926F9260
:102E70007F929F92AF92BF92CF92DF92EF92FF929A
:102E80000F931F93CF93DF93982E8EE0A82EB12C33
:102E9000EE24EA9493E0F92E0FEF13E0D12CC12C2D
:102EA000D0E0C0E0412C512C3201892D0E947C9C45
:102EB000C817D90708F44AC0C816D90608F46C0127
:102EC0008017910708F444C08E159F0508F47C0113
:102ED000BC0190E080E00E94A9B49B01AC01C30159
:102EE000B2010E9445B62B013C0165E070E080E034
:102EF00090E00E94F19F81E0A81AB108B1F6BE01EE
:102F00006C0D7D1D6E0D7F1D600F711F90E080E0C8
:102F10000E94A9B49B01AC01C301B2010E9444B656
:102F200020E030E040E251E40E9423B7DF91CF91EE
:102F30001F910F91FF90EF90DF90CF90BF90AF90D7
:102F40009F907F906F905F904F900895EC01B8CF65
:102F50008C01BECF4F925F926F927F92AF92BF92E1
:102F6000CF92DF92FF920F931F93CF93DF9300D006
:102F700000D0CDB7DEB75C0186E09FE00E94C28D35
:102F800040E052EC61E070E086E09FE00E948658ED
:102F90008CED95E0A0E0B0E080930A0F90930B0FCA
:102FA000A0930C0FB0930D0F64E670E080E090E00A
:102FB0000E94F19FD12CC12CF12C65E070E080E0E3
:102FC00090E00E94F19F10E000E0412C512C320172
:102FD000F1103AC086E09FE00E942A88892B31F4E4
:102FE00085E1481651046104710474F5033011053C
:102FF0005CF586E09FE00E942A88892B69F086E0D4
:103000009FE00E940888E1E0F0E0EC0FFD1FE00F78
:10301000F11F80830F5F1F4F65E070E080E090E05C
:103020000E94F19F023011054CF089818B3B31F4F5
:10303000FF24F3948A818A3A09F0F12C8FEF481A21
:10304000580A680A780AC4CF8FEFC81AD80A64E60B
:1030500070E080E090E00E94F19FAC14BD0409F0A4
:10306000ACCF8F2D26960FB6F894DEBF0FBECDBF26
:10307000DF91CF911F910F91FF90DF90CF90BF9084
:10308000AF907F906F905F904F9008951F93CF9374
:10309000DF93182FCDE2DDE0812F0E947C9C899385
:1030A00099936CE370E080E090E00E94F19F8DE0E6
:1030B000CD37D80789F70E94218B20E030E040EA25
:1030C00050E40E940AB520E030E040E85AE30E9454
:1030D0000AB5DF91CF911F910895CF92DF92EF92C1
:1030E000FF920F931F93CF93DF9300D000D0CDB703
:1030F000DEB72091140C222309F4AAC02091390CC8
:1031000030913A0C263531050CF0A2C0409185046F
:1031100050918604493D5F400CF09AC07C012F5FBE
:103120003F4F30933A0C2093390C0E948DA60091AA
:103130000C0C10910D0C20910E0C30910F0C601B9B
:10314000710B820B930B0E94A9B420E030E04AE798
:1031500054E40E9423B76093100C7093110C809379
:10316000120C9093130C80918504909186048835FD
:10317000924034F488E592E090938604809385042D
:10318000809185049091860400E11CE09C0120510F
:103190003C406901C601800F911F9A838983F80121
:1031A00061918F01CE0101960E946D58FCE00431BF
:1031B0001F0781F78091850490918604049690936F
:1031C000860480938504B701CE0101960E94019880
:1031D000CE0101960E940997BC0185EB92E10E9405
:1031E0004E97CE0101960E949E974091B912509140
:1031F000BA124115510531F065E17CE085EB92E1B1
:103200000E94758D809185049091860429E3C22ED9
:103210002CE0D22E05E11CE09C0125513C407901B7
:10322000C701800F911F9A838983F80161918F01F3
:10323000CE0101960E946D58C016D10689F7809183
:1032400085049091860484969093860480938504E7
:1032500026960FB6F894DEBF0FBECDBFDF91CF919B
:103260001F910F91FF90EF90DF90CF900895AF9254
:10327000BF92CF92DF92EF92FF920F931F93CF9363
:10328000DF93CDB7DEB72C970FB6F894DEBF0FBE35
:10329000CDBF8091030D811102C00E94B85780916B
:1032A000930490919404029751F08091040C9091B2
:1032B000050C009709F4B4C1039709F4B1C163E5A3
:1032C00074E08FEA92E10E9429976FEA72E1CE01E1
:1032D00001960E94019844E150E070E060E0CE0168
:1032E00001960E948059CE0101960E949E9764E447
:1032F00074E08FEA92E10E9429976FEA72E1CE01B1
:1033000001960E94019844E150E06FEF7FEFCE01FB
:1033100001960E94FA57CE0101960E949E9787E07F
:103320000E94CC9F8C0186E00E94CC9FBC0190E063
:1033300080E00E94A9B42AE037ED43EA5CE30E94F2
:103340000AB523E333E948E853E40E9444B66B012D
:103350007C0184E0A82EB12C20E030E048EC52E45F
:10336000C701B6010E942CB818160CF05FC081E0AE
:10337000A81AB108E9F064E670E080E090E00E94ED
:10338000F19F86E00E94CC9FBC0190E080E00E940B
:10339000A9B42AE037ED43EA5CE30E940AB523E3CF
:1033A00033E948E853E40E9444B66B017C01D4CF72
:1033B00069E374E08FEA92E10E9429976FEA72E173
:1033C000CE0101960E9401984AE050E070E060E072
:1033D000CE0101960E948059CE0101960E949E97CF
:1033E00065EB75E0CE0101960E940A986FEA72E1E2
:1033F000CE0101960E94B896BC0185EB92E10E9435
:103400004E97CE0101960E949E978091040C909158
:10341000050C049721F41092050C1092040C81E025
:1034200090E09093940480939304D9C0B80190E005
:1034300080E00E94A9B42AE037ED43EA5CE30E94F1
:103440000AB523E333E948E853E40E9444B6AB01EC
:10345000BC0121E0CE0101960E94A69767EC75E0C1
:10346000CE0107960E940A98BE016F5F7F4FCE0182
:1034700007960E94B896BC0185EB92E10E944E9798
:10348000CE0107960E949E97CE0101960E949E97BC
:1034900065EB72E1CE0101960E94019842E350E093
:1034A0006FEF7FEFCE0101960E94FA57CE01019691
:1034B0000E949E9761ED75E0CE0101960E940A98E8
:1034C000CE0101960E94DC57CE0101960E949E9784
:1034D00060ED75E085EB92E10E94189721E0B7015D
:1034E000A601CE0101960E94A69766EF76E0CE0176
:1034F00007960E940A98BE016F5F7F4FCE01079624
:103500000E94B896BC018BEB92E10E944E97CE01CF
:1035100007960E949E97CE0101960E949E976CE5A9
:103520007AE0CE0101960E940A986BEB72E1CE011F
:1035300001960E94B896BC018FEA92E10E944E97D4
:10354000CE0101960E949E976FEA72E1CE0101962C
:103550000E9401984AE050E070E060E0CE010196E0
:103560000E94D658CE0101960E949E9761ED75E0AB
:10357000CE0101960E940A98CE0101960E94DC5766
:10358000CE0101960E949E9760ED75E08BEB92E173
:103590000E9418976BEB72E1CE0101960E94019890
:1035A0006CE57AE0CE0101960E94A29665EB72E18D
:1035B0000E94B896BC0185EB92E10E944E97CE0125
:1035C00001960E949E978091040C9091050C0397A0
:1035D00031F484E090E09093050C8093040C64E651
:1035E00070E080E090E00E94F19F8091030D8823BD
:1035F00031F060E273E080E090E00E94F19F2C9651
:103600000FB6F894DEBF0FBECDBFDF91CF911F91F3
:103610000F91FF90EF90DF90CF90BF90AF90089503
:1036200089E69EE00E94C28D64E670E080E090E052
:103630000E94F19F69E774E08FEA92E10E94299766
:103640006FEA72E1CE0101960E94019844E150E0D8
:1036500070E060E0CE0101960E948059CE01019693
:103660000E949E976AE674E08FEA92E10E94299791
:103670006FEA72E1CE0101960E94019844E150E0A8
:103680006FEF7FEFCE0101960E94FA57CE010196AF
:103690000E949E978CE40E94CBA66B017C0104E003
:1036A00010E0A7019601C701B6010E9491B98823D5
:1036B00009F449C00150110961F068EC70E080E044
:1036C00090E00E94F19F8CE40E94CBA66B017C01EC
:1036D000E8CF6FE574E08FEA92E10E9429976FEAE4
:1036E00072E1CE0101960E9401984AE050E070E03C
:1036F00060E0CE0101960E948059CE0101960E94A1
:103700009E9765EB75E0CE0101960E940A986FEADC
:1037100072E1CE0101960E94B896BC0185EB92E160
:103720000E944E97CE0101960E949E978091040CB4
:103730009091050C039721F41092050C1092040C43
:1037400082E090E06ECE21E0B701A601CE0107969F
:103750000E94A69767EC75E0CE0101960E940A9838
:10376000BE01695F7F4FCE0101960E94B896BC01F1
:1037700085EB92E10E944E97CE0101960E949E97A2
:10378000CE0107960E949E9765EB72E1CE010196ED
:103790000E94019842E350E06FEF7FEFCE01019667
:1037A0000E94FA57CE0101960E949E9761ED75E046
:1037B000CE0101960E940A98CE0101960E94DC5724
:1037C000CE0101960E949E9760ED75E085EB92E137
:1037D0000E94189786E60E94CBA66B017C0104E04C
:1037E00010E0A7019601C701B6010E9491B9882394
:1037F00081F00150110909F484C068EC70E080E0A8
:1038000090E00E94F19F86E60E94CBA66B017C01AE
:10381000E8CF21E0B701A601CE0107960E94A69746
:1038200066EF76E0CE0101960E940A98BE01695FBC
:103830007F4FCE0101960E94B896BC018BEB92E1BE
:103840000E944E97CE0101960E949E97CE01079648
:103850000E949E976CE57AE0CE0101960E940A983C
:103860006BEB72E1CE0101960E94B896BC018FEA23
:1038700092E10E944E97CE0101960E949E976FEAB8
:1038800072E1CE0101960E9401984AE050E06FEF8C
:103890007FEFCE0101960E94D658CE0101960E947C
:1038A0009E9761ED75E0CE0101960E940A98CE01C7
:1038B00001960E94DC57CE0101960E949E9760ED12
:1038C00075E08BEB92E10E9418976BEB72E1CE01F1
:1038D00001960E9401986CE57AE0CE0101960E9463
:1038E000A29665EB72E10E94B896BC0185EB92E16D
:1038F0000E944E97CE0101960E949E9783E090E031
:103900006ACE64ED7BE08BEB92E10E942A95DDCFDD
:10391000EF92FF920F931F93CF93DF93CDB7DEB754
:1039200068970FB6F894DEBF0FBECDBF8C016CE573
:103930007AE0CE010D960E940A9863ED75E0CE0103
:1039400043960E940A986AEB79E0C8010E94F897B2
:10395000BE016D5E7F4FC8010E94229761EB79E046
:10396000C8010E94CB968FEAE82E81E1F82EF7017C
:10397000608170E0CE0101960E946195BE016F5F8B
:103980007F4FCE0107960E940198BE01635F7F4F73
:10399000CE0107960E94B896BC01C8010E942297EA
:1039A000CE0107960E949E97CE0101960E949E9797
:1039B00064EA79E0C8010E94CB96F7016181062E86
:1039C000000C770BCE0101960E946195BE016F5FDE
:1039D0007F4FCE0107960E940198BE01635F7F4F23
:1039E000CE0107960E94B896BC01C8010E9422979A
:1039F000CE0107960E949E97CE0101960E949E9747
:103A00006AE979E0C8010E94CB96F7016281062E2F
:103A1000000C770BCE0101960E946195BE016F5F8D
:103A20007F4FCE0107960E940198BE01635F7F4FD2
:103A3000CE0107960E94B896BC01C8010E94229749
:103A4000CE0107960E949E97CE0101960E949E97F6
:103A500062E979E0C8010E94CB96F7016381748125
:103A6000CE0101960E946195BE016F5F7F4FCE012E
:103A700007960E940198BE016D5E7F4FCE010796AA
:103A80000E94B896BC01C8010E942297CE010796F9
:103A90000E949E97CE0101960E949E976BE779E067
:103AA000C8010E94CB96F70165817681CE0101960F
:103AB0000E946195BE016F5F7F4FCE0107960E9405
:103AC0000198BE01635F7F4FCE0107960E94B896B2
:103AD000BC01C8010E942297CE0107960E949E97C2
:103AE000CE0101960E949E9762E779E0C8010E948C
:103AF000CB96F7016781062E000C770B6F5F7F4F27
:103B0000CE0101960E946195BE016F5F7F4FCE018D
:103B100007960E940198BE01635F7F4FCE01079612
:103B20000E94B896BC01C8010E942297CE01079658
:103B30000E949E97CE0101960E949E9767E679E0CB
:103B4000C8010E94CB96F7016085062E000C770B0A
:103B5000CE0101960E946195BE016F5F7F4FC80143
:103B60000E942297CE0101960E949E97CE01439615
:103B70000E949E97CE010D960E949E97C80168965E
:103B80000FB6F894DEBF0FBECDBFDF91CF911F916E
:103B90000F91FF90EF9008954F925F926F927F92F6
:103BA0009F92AF92BF92CF92DF92EF92FF920F93CC
:103BB0001F93CF93DF93CDB7DEB7A8970FB6F894D6
:103BC000DEBF0FBECDBF63ED72E18DEC92E10E94CE
:103BD0004E970E94139563E076E0CE0101960E9415
:103BE0000A98BE016F5F7F4F8DEC92E10E9487962D
:103BF000182FCE0101960E949E97112309F4F7C059
:103C00008091D7129091D8124097B8F080E0A89692
:103C10000FB6F894DEBF0FBECDBFDF91CF911F91DD
:103C20000F91FF90EF90DF90CF90BF90AF909F905B
:103C30007F906F905F904F90089542E050E063ED69
:103C400072E1CE0101960E94CA58BE016F5F7F4F9C
:103C50008FEA92E10E946597CE0101960E949E979D
:103C60006FEA72E1CE0101960E940198CE010196A1
:103C70000E94825BCE0101960E949E978FEA92E19C
:103C80000E949C9520E030E048EC52E40E940AB586
:103C90000E94CFB7AB01BC014093C7045093C80446
:103CA0006093C9047093CA04CE0101960E943495B2
:103CB000CE0101960E94825BCE0101960E949E97E2
:103CC0006091C7047091C8048091C9049091CA049E
:103CD0008B019C0100591F452140310901341C49C9
:103CE00021053105C8F166ED75E0CE0101960E940F
:103CF0000A986FEA72E1CE0101960E94B89669EEC9
:103D000075E00E94A296BC0185EB92E10E944E975D
:103D1000CE0101960E949E9764ED75E0CE0101965A
:103D20000E940A9865EB72E1CE0101960E94B89656
:103D3000BC01CE0145960E940198CE0145960E9495
:103D40008457CE0145960E949E97CE0101960E940F
:103D50009E971092EC0489C01A821982FE01339654
:103D600026E0DF011D922A95E9F70E94ABB420E01E
:103D700030E048EC52E40E9423B78E010F5F1F4FE2
:103D800022E047E00E9400B0BC0185EB92E10E9476
:103D90008D9569EF75E0CE0145960E940A9865EB16
:103DA00072E1CE0145960E94B89666E076E00E94E8
:103DB000A296BC0185EB92E10E944E97CE014596FA
:103DC0000E949E978091C7049091C804A091C90455
:103DD000B091CA0480931E1190931F11A0932011DB
:103DE000B093211190E080E00E944B8D95CF61EF60
:103DF00078E0CE0101960E94F897BE016F5F7F4F79
:103E00008DEC92E10E948796182FCE0101960E94B8
:103E10009E97112389F142E050E063ED72E1CE01FB
:103E200001960E94CA58BE016F5F7F4F8FEA92E1F0
:103E30000E946597CE0101960E949E978FEA92E1BB
:103E40000E94A7956330710590F47093070C6093FE
:103E5000060C8091060C9091070C9093A51180930D
:103E6000A41190E080E00E944B8D81E0D0CE1092B2
:103E7000070C1092060CEDCF6CEE78E0CE010196A7
:103E80000E94F897BE016F5F7F4F8DEC92E10E9418
:103E90008796182FCE0101960E949E971123A1F1BB
:103EA00026E030E044E050E063ED72E1CE0101969F
:103EB0000E941B98BE016F5F7F4F8FEA92E10E94C4
:103EC0006597CE0101960E949E978FEA92E10E942B
:103ED000A79570939711609396117093D504609392
:103EE000D40463ED72E1CE0101960E940198CE01E7
:103EF00001960E94825BCE0101960E949E9790E0FF
:103F000080E00E944B8D25CF65EE78E0CE010196D2
:103F10000E94F897BE016F5F7F4F8DEC92E10E9487
:103F20008796182FCE0101960E949E971123A1F12A
:103F300046E050E063ED72E1CE0101960E94CA585E
:103F4000BE016F5F7F4F8FEA92E10E946597CE01BD
:103F500001960E949E978091B3129091B412892B82
:103F600061F08FEA92E10E949C9560938A047093BD
:103F70008B0480938C0490938D0463ED72E1CE01E9
:103F800001960E940198CE0101960E94825BCE01AB
:103F900001960E949E97DDCE6BE076E0CE01019601
:103FA0000E940A98BE016F5F7F4F8DEC92E10E94E4
:103FB0008796182FCE0101960E949E97112309F42F
:103FC000BEC061EE78E0CE0101960E94F897BE0176
:103FD0006F5F7F4F8DEC92E10E948796182FCE0184
:103FE00001960E949E971123D1F184E090E00E94F7
:103FF000990E6093AB047093AC048093AD049093DE
:10400000AE0461ED78E085EB92E10E942997409142
:10401000AB045091AC046091AD047091AE0422E009
:10402000CE0101960E94A697BE016F5F7F4F85EB80
:1040300092E10E942297CE0101960E949E97809164
:10404000AB049091AC04A091AD04B091AE04809308
:10405000421190934311A0934411B09345116EE027
:1040600076E0CE0101960E940A98BE016F5F7F4FF5
:104070008DEC92E10E948796182FCE0101960E9446
:104080009E971123F1F18AE090E00E94990E6093CF
:10409000A7047093A8048093A9049093AA0460ECE9
:1040A00078E085EB92E10E9429974091A704509116
:1040B000A8046091A9047091AA0422E0CE0101969F
:1040C0000E94A697BE016F5F7F4F85EB92E10E9431
:1040D0002297CE0101960E949E978091A70490910D
:1040E000A804A091A904B091AA04809346119093CA
:1040F0004711A0934811B093491190E080E00E94CD
:104100004B8D64ED75E0CE0101960E940A9865EB37
:1041100072E1CE0101960E94B896BC01CE0145968F
:104120000E940198CE0145960E948457CE01459683
:104130000E949E97CE0101960E949E9796CE63E1C3
:1041400076E0CE0101960E940A98BE016F5F7F4F14
:104150008DEC92E10E948796182FCE0101960E9465
:104160009E97112309F4BDC08091D7129091D81267
:104170000797F8F046E050E063ED72E1CE0101965A
:104180000E94CA58BE016F5F7F4F8FEA92E10E9482
:104190006597CE0101960E949E978FEA92E10E9458
:1041A0009C956093DA047093DB048093DC04909315
:1041B000DD0480917F049091800499270E94351737
:1041C0002DE038E643E55BE30E940AB56B017C0114
:1041D000209105053091060540910705509108058D
:1041E0000E94A4B418160CF460C06091ED047091A4
:1041F000EE048091EF049091F00420E030E048EC70
:1042000052E40E940AB56B017C0120E030E0A90174
:104210000E94A4B4181634F0C12CD12C38EAE32E35
:1042200031E4F32EC092DA04D092DB04E092DC0495
:10423000F092DD04C0925211D0925311E0925411C9
:10424000F09255118091040D882381F06EEA78E098
:1042500083EA9FE00E94759A6091DA047091DB0412
:104260008091DC049091DD040E94F79990E080E059
:104270000E944B8D64EA78E085EB92E10E942997D9
:104280004091DA045091DB046091DC047091DD040C
:1042900022E0CE0101960E94A697BE016F5F7F4F7C
:1042A00085EB92E10E942297A7C0209119053091D9
:1042B0001A0540911B0550911C05C701B6010E94CB
:1042C0002CB887FF05C0C701B6010E944B8C95CF63
:1042D000609101057091020580910305909104059C
:1042E0008CCF60EA78E0CE0101960E94F897BE017B
:1042F0006F5F7F4F8DEC92E10E948796182FCE0161
:1043000001960E949E97112309F47BC060E0809182
:104310007D040E94409C09E110E0C12CD12C760163
:1043200080917D040E947C9CBC01990F880B990BA5
:104330000E94ABB49B01AC01C701B6010E9445B617
:104340006B017C016AE070E080E090E00E94F19FE8
:104350000150110929F720E030E040EA50E4C7019C
:10436000B6010E940AB520E030EC4FE754E40E9409
:1043700023B720E030E048EC51E40E9423B760937B
:10438000D6047093D7048093D8049093D904609393
:1043900068117093691180936A1190936B1190E08A
:1043A00080E00E944B8D6DE878E085EB92E10E9401
:1043B00029974091D6045091D7046091D804709108
:1043C000D90422E0CE0101960E94A697BE016F5F3C
:1043D0007F4FCE0145960E94019869E176E0CE01BB
:1043E00045960E94A296BC0185EB92E10E9422971D
:1043F000CE0145960E949E97CE0101960E949E97FF
:1044000056C06CE176E0CE0101960E940A98BE018A
:104410006F5F7F4F8DEC92E10E948796182FCE013F
:1044200001960E949E97112309F44CC080914D1172
:10443000082E000C990B0197039798F589E390E0FB
:104440000E9435172AE137E64CE950E40E940AB58C
:1044500060934E1170934F118093501190935111AE
:1044600090E080E00E944B8D6CE678E085EB92E175
:104470000E94299740914E1150914F116091501117
:104480007091511122E0CE0101960E94A697BE01C3
:104490006F5F7F4FCE0145960E94019862E276E001
:1044A0009ECF66E478E085EB92E10E94299765EB68
:1044B00072E1CE0101960E940198CE0101960E9400
:1044C000845765CD62E478E0CE0101960E94F897AA
:1044D000BE016F5F7F4F8DEC92E10E948796182F8F
:1044E000CE0101960E949E97112309F43CC126E05B
:1044F00030E044E050E063ED72E1CE0101960E94AD
:104500001B98BE016F5F7F4F8FEA92E10E94659713
:10451000CE0101960E949E978FEA92E10E94A79594
:104520006B015B0166E679E0CE0101960E940A9874
:10453000BE016F5F7F4F83ED92E10E940F968E0167
:104540000B5E1F4FAC014F5F5F4F63ED72E1C8011F
:104550000E94CA58B8018FEA92E10E946597C8018B
:104560000E949E97CE0101960E949E9790907B0498
:104570008FEA92E10E949C952B013C018091040DF1
:104580008823B9F06BE577E083EA9FE00E94759A93
:104590004AE050E0B60183EA9FE00E94069A6CE58B
:1045A0007AE083EA9FE00E94539AC301B2010E941D
:1045B000F799692DC8010E940C0D18870F831D8281
:1045C0001E82198289E08A8381E08B838C831C8A16
:1045D0001B8ACE0101960E94C511CE0101960E9450
:1045E0006810CE0101960E94E1A20E8110E00B300E
:1045F000110514F00AE010E0BBE5CB16D10408F475
:104600004EC02BE3C22E2CE0D22E5601412C512C51
:104610003201F12CE12C0E151F05B9F06E2DCE01E3
:1046200001960E9459119B01AC01F5012193319330
:10463000419351935F01C301B2010E9445B62B0122
:104640003C01FFEFEF1AFF0AE6CFB7010F2C000C79
:10465000880B990B0E94ABB49B01AC01C301B20162
:104660000E9423B72B013C0110E000E0E016F106A8
:10467000B9F1D6012D913D914D915D916D015D0195
:10468000B4E0AB1AB108C301B2010E9444B6F5010F
:1046900060837183828393830F5F1F4FE7CF1A1468
:1046A0001B040CF041C00A151B050CF086010150DB
:1046B0001109602FCE0101960E9459119B01AC0196
:1046C000000F111F000F111F055C134FC301B20132
:1046D0000E9444B6D8016D937D938D939C9313975C
:1046E000EBE3FCE0ACE6B1E183E69CE04191519163
:1046F000619171914D935D936D937D938E179F079B
:10470000A9F790E080E00E944B8D61E278E085EBB4
:1047100092E10E94299744E050E063ED72E1CE01FE
:1047200001960E94CA58B9CDA114B104C9F68BE311
:10473000E82E8CE0F82E0A151B0591F26A2DCE01A9
:1047400001960E9459119B01AC01C301B2010E9464
:1047500044B6F70161937193819391937F01FFEFC9
:10476000AF1ABF0AE8CF65E276E0CE0101960E945B
:104770000A98BE016F5F7F4F8DEC92E10E94879691
:10478000182FCE0101960E949E97112309F423C190
:1047900027E030E046E050E063ED72E1CE010196A3
:1047A0000E941B98BE016F5F7F4F8FEA92E10E94CB
:1047B0006597CE0101960E949E978FEA92E10E9432
:1047C000A7957B0160934D1183ED92E10E94B29514
:1047D0006CE57AE0CE0101960E940A98BE016F5FF7
:1047E0007F4F83ED92E10E940F96AC014F5F5F4FC8
:1047F00063ED72E1CE0145960E94CA58CE014596FE
:104800000E949C9560934E1170934F1180935011AC
:1048100090935111CE0145960E949E97CE0101962C
:104820000E949E9760E178E085EB92E10E942997D3
:1048300044E0E416F1041CF582E0E816F1040CF003
:104840009FC0E114F10431F1EA94EF2809F471C03A
:1048500060914D11062E000C770BCE0145960E94FB
:10486000619567E376E0CE0101960E940A98BE0149
:104870006B5E7F4FCE0101960E94B8964CC0B4E0AB
:10488000EB16F10429F76FEE77E085EB92E10E94D9
:10489000CB9671C020E030E0A90160914E1170917B
:1048A0004F1180915011909151110E94A4B418168B
:1048B00064F080E090E0A0E8BFE380934E11909315
:1048C0004F11A0935011B093511120914E1130917E
:1048D0004F11409150115091511160E070E080EA09
:1048E00090E40E9423B7AB01BC0122E0CE014596C3
:1048F0000E94A6976CE276E0CE0101960E940A988B
:10490000BE016B5E7F4FCE0101960E94B89660E1BA
:104910007BE00E94A296BC0185EB92E10E94229767
:10492000CE0101960E949E97CE0145960E949E97C9
:1049300022C062E078E085EB92E10E94CB9620E015
:1049400030E048E453E460914E1170914F11809132
:104950005011909151110E94A4B4181664F080E097
:1049600090E4ACE1B5E480934E1190934F11A09385
:104970005011B093511190E080E00E944B8D97CD83
:1049800066EF77E085EB92E10E94CB968AE08E9D00
:10499000B0018F9D700D1124CE0101960E9461958A
:1049A000BE016F5F7F4FCE0145960E94019869E07E
:1049B0007BE0CE0145960E94A296BC0185EB92E178
:1049C0000E942297CE0145960E949E97CE010196A5
:1049D0000E949E97B4CF6EE376E0CE0101960E94CE
:1049E0000A98BE016F5F7F4F8DEC92E10E9487961F
:1049F000182FCE0101960E949E97112309F4CCC076
:104A000027E030E046E050E063ED72E1CE01019630
:104A10000E941B98BE016F5F7F4F8FEA92E10E9458
:104A20006597CE0101960E949E978FEA92E10E94BF
:104A3000A79560934A1183ED92E10E94B2958FEAA7
:104A400092E10E94A795611571058105910509F014
:104A500074C085E090E090934C1180934B1190E0EE
:104A600080E00E944B8D6EED77E085EB92E10E9435
:104A7000299780914A11833044F563ED77E085EB07
:104A800092E10E94CB9660914B1170914C11CE0136
:104A900001960E946195BE016F5F7F4FCE014596E2
:104AA0000E94019866E37AE0CE0145960E94A296A4
:104AB000BC0185EB92E10E942297CE0145960E94AF
:104AC0009E97CE0101960E949E9780914A11833055
:104AD0000CF4EDCC60914B1170914C11CE0183968A
:104AE0000E94619560914A11062E000C770BCE0151
:104AF00045960E94619567E376E0CE0101960E949B
:104B00000A98BE016B5E7F4FCE0101960E94B89657
:104B1000BE016D5D7F4F0E94B896BC0185EB92E1AE
:104B20000E942297CE0101960E949E97CE01459643
:104B30000E949E97CE01839661CC613071058105FC
:104B4000910519F489E190E086CF6CE57AE0CE0119
:104B500001960E940A98BE016F5F7F4F83ED92E13C
:104B60000E940F96AC014F5F5F4F63ED72E1CE0183
:104B700045960E94CA58CE0145960E94A79570930B
:104B80004C1160934B11CE0145960E949E97CE0129
:104B900001960E949E9763CF65E476E0CE01019670
:104BA0000E940A98BE016F5F7F4F8DEC92E10E94D8
:104BB0008796182FCE0101960E949E97112309F423
:104BC00068C08091790490917A040E94461860939D
:104BD000AF047093B0048093B1049093B2046093D7
:104BE000361170933711809338119093391180E00A
:104BF00090E5A3ECB7E48093B7049093B804A09336
:104C0000B904B093BA0480932E1190932F11A093FE
:104C10003011B09331118091040D882381F065EB40
:104C200077E083EA9FE00E94759A6091AF047091EB
:104C3000B0048091B1049091B2040E94F79990E081
:104C400080E00E944B8D4091AF045091B004609180
:104C5000B1047091B20422E0CE0145960E94A6975D
:104C600069E476E0CE0101960E940A98BE016B5E6F
:104C70007F4FCE0101960E94B896BC0185EB92E170
:104C80000E944E97CE0101960E949E97CE014596B6
:104C9000B5CB64E576E0CE0101960E940A98BE018C
:104CA0006F5F7F4F8DEC92E10E948796182FCE01A7
:104CB00001960E949E97112309F488C08091D71213
:104CC0009091D8120497F8F044E050E063ED72E15F
:104CD000CE0101960E94CA58BE016F5F7F4F8FEAD6
:104CE00092E10E946597CE0101960E949E978FEAFD
:104CF00092E10E949C956093BB047093BC048093E6
:104D0000BD049093BE048091BB049091BC04A0911B
:104D1000BD04B091BE0480932A1190932B11A093EF
:104D20002C11B0932D118091040D882389F06CE92A
:104D300077E083EA9FE00E94759A6091BB047091CE
:104D4000BC048091BD049091BE0442E00E9415997C
:104D50008091790490917A040E9446186093B3047C
:104D60007093B4048093B5049093B60460933211A9
:104D70007093331180933411909335118091040D09
:104D8000882381F062E977E083EA9FE00E94759AC8
:104D90006091B3047091B4048091B5049091B6040D
:104DA0000E94F79990E080E00E944B8D4091B304FF
:104DB0005091B4046091B5047091B60422E0CE0124
:104DC00045960E94A69768E576E04CCF60E676E0CF
:104DD000CE0101960E940A98BE016F5F7F4F8DEC55
:104DE00092E10E948796182FCE0101960E949E970D
:104DF000112311F40C94061E8091D7129091D812B1
:104E00000497F8F044E050E063ED72E1CE010196C2
:104E10000E94CA58BE016F5F7F4F8FEA92E10E94E5
:104E20006597CE0101960E949E978FEA92E10E94BB
:104E30009C956093B7047093B8048093B9049093E1
:104E4000BA048091B7049091B804A091B904B091CC
:104E5000BA0480932E1190932F11A0933011B09328
:104E600031118091040D882389F069E777E083EAA6
:104E70009FE00E94759A6091B7047091B804809188
:104E8000B9049091BA0442E00E9415998091790486
:104E900090917A040E9446186093AF047093B00416
:104EA0008093B1049093B2046093361170933711DC
:104EB00080933811909339118091040D882381F0EB
:104EC0006FE677E083EA9FE00E94759A6091AF04F5
:104ED0007091B0048091B1049091B2040E94F7994E
:104EE00090E080E00E944B8D4091AF045091B0045F
:104EF0006091B1047091B20461CFCF93DF93CDB7CD
:104F0000DEB72C970FB6F894DEBF0FBECDBF813051
:104F1000910509F06EC0909395118093941168E00B
:104F200076E0CE0101960E94F897CE0101960E948C
:104F3000825BCE0101960E949E9764E676E0CE01E8
:104F400001960E940A986AEA73E1CE0101960E94D6
:104F5000B896BC01CE0107960E94019848EC50E03B
:104F60006FEF7FEFCE0107960E948059CE01079622
:104F70000E949E97CE0101960E949E978CEC9DE028
:104F80000E94C28D40E052EC61E070E08CEC9DE04C
:104F90000E94865890E080E00E944B8D63E776E0A7
:104FA000CE0101960E940A9864EA73E1CE0101964F
:104FB0000E94B896BC01CE0107960E94019840ED70
:104FC00057E06FEF7FEFCE0107960E94FA57CE01B0
:104FD00007960E949E97CE0101960E949E9781E0BF
:104FE0002C960FB6F894DEBF0FBECDBFDF91CF91E8
:104FF00008950097E1F510929511109294116AEFBF
:1050000075E0CE0101960E94F897CE0101960E94AC
:10501000825BCE0101960E949E976AE676E0CE0101
:1050200001960E940A986AEA73E1CE0101960E94F5
:10503000B896BC01CE0107960E94019848EC50E05A
:105040006FEF7FEFCE0107960E948059CE01079641
:105050000E949E97CE0101960E949E978CEC9DE047
:105060000E94C28D40E855E260E070E08FCF823050
:105070009105A9F4909395118093941169EE75E0D0
:10508000CE0101960E94F897CE0101960E94825BA4
:10509000CE0101960E949E976EE676E0C0CF80E03A
:1050A0009FCF0F931F93CF93DF93CDB7DEB72C978E
:1050B0000FB6F894DEBF0FBECDBF8C0164ED7BE070
:1050C00083ED92E10E942A950830110509F0F8C09D
:1050D0006FED75E0CE0101960E94F89744E650E02E
:1050E0006FEF7FEFCE0101960E948059CE010196AD
:1050F0000E949E9763ED75E0CE0101960E94F8979D
:1051000044E650E070E060E0CE0101960E94FA575C
:10511000CE0101960E949E978CEC9DE00E94CD8866
:105120004CE251E061E070E0CE0107960E94BEA320
:105130008091040D8823D1F068E776E0CE010196D6
:105140000E940A98BE01695F7F4FCE0101960E94BE
:10515000B8966BE776E00E94A296BC0183EA9FE0D6
:105160000E94639ACE0101960E949E9769E07BE0BF
:10517000CE0101960E940A98BE016F5F7F4FCE015B
:1051800007960E948796182FCE0101960E949E973F
:10519000112309F478C06DE776E083ED92E10E9477
:1051A0002A9588E090E09093030C8093020C0E9473
:1051B000CC1D182F66EC75E0CE0101960E94F89781
:1051C00044E650E070E060E0CE0101960E94FA579C
:1051D000CE0101960E949E978CEC9DE00E94CD88A6
:1051E00048E552E061E070E0CE0101960E94BEA366
:1051F000BE016F5F7F4FCE0107960E946597CE017B
:1052000001960E949E978091040D8823D1F068E753
:1052100076E0CE0101960E940A98BE01695F7F4F39
:10522000CE0101960E94B8966BE776E00E94A296A6
:10523000BC0183EA9FE00E94639ACE0101960E941E
:105240009E976BE87BE0CE0101960E940A98BE0112
:105250006F5F7F4FCE0107960E948796082FCE0181
:1052600001960E949E97002371F062E876E083ED3C
:1052700092E10E942A950E94CC1D882321F069EBBF
:1052800075E0111102C062EB75E0CE0101960E943B
:10529000F89744E650E070E060E0CE0101960E948D
:1052A000FA57CE0101960E949E9764ED7BE083ED54
:1052B00092E10E942A95CE0107960E949E97A0C275
:1052C000093F2FEF120709F00CC168EA75E0CE0123
:1052D00001960E94F89744E650E06FEF7FEFCE0111
:1052E00001960E948059CE0101960E949E976AE91C
:1052F00075E0CE0101960E94F89744E650E070E018
:1053000060E0CE0101960E94FA57CE0101960E94FC
:105310009E978CEC9DE00E94CD884CE251E064E0C9
:1053200070E0CE0101960E94BEA38091040D8823F7
:10533000D1F068E776E0CE0107960E940A98BE0198
:105340006F5F7F4FCE0107960E94B8966BE776E0BD
:105350000E94A296BC0183EA9FE00E94639ACE015C
:1053600007960E949E9770E060E0CE0101960E9431
:105370007696082E000C990BC0970A9708F096C0F5
:1053800068E876E0CE0107960E940A98BE016F5F3A
:105390007F4FCE0107960E94B896BC0183ED92E143
:1053A0000E944E97CE0107960E949E9789EF9FEF2D
:1053B0009093030C8093020C0E94CC1D182F6CE874
:1053C00075E0CE0107960E94F89744E650E070E041
:1053D00060E0CE0107960E94FA57CE0107960E9420
:1053E0009E978CEC9DE00E94CD8848E552E065E0F8
:1053F00070E0CE0107960E94BEA3BE01695F7F4F99
:10540000CE0101960E946597CE0107960E949E9755
:105410008091040D8823D1F068E776E0CE010796ED
:105420000E940A98BE016F5F7F4FCE0107960E94CF
:10543000B8966BE776E00E94A296BC0183EA9FE0F3
:105440000E94639ACE0107960E949E9770E060E0EA
:10545000CE0101960E947696082E000C990BC097FB
:105460000A9720F56DE876E0CE0107960E940A982B
:10547000BE016F5F7F4FCE0107960E94B896BC01B8
:1054800083ED92E10E944E97CE0107960E949E976F
:1054900089EF9FEF9093030C8093020C0E94CC1D28
:1054A000882321F06FE775E0111102C068E775E00D
:1054B000CE0107960E94F89744E650E070E060E065
:1054C000CE0107960E94FA57CE0107960E949E973A
:1054D00064ED7BE083ED92E10E942A95CE01019676
:1054E000ECCE6EE675E0CE0101960E94F89744E698
:1054F00050E06FEF7FEFCE0101960E948059CE0100
:1055000001960E949E9764ED7BE083ED92E10E94FC
:105510002A95053F8FEF180709F044C062E976E04D
:1055200083ED92E10E942A9564E675E0CE01019632
:105530000E94F89744E650E06FEF7FEFCE010196AE
:105540000E94FA57CE0101960E949E978091D71231
:105550009091D812892B09F453C10E94CC1D882345
:1055600009F459C168EC70E080E090E00E94F19F7E
:1055700064EE74E0CE0101960E94F89744EF51E08A
:105580006FEF7FEFCE0101960E94FA57CE01019690
:105590000E949E971093030C0093020CC8010E9476
:1055A0005C742EC1063F2FEF120749F463E176E0E9
:1055B00083ED92E10E942A956AE575E0B7CF013F3D
:1055C0008FEF180749F46CE176E083ED92E10E94D9
:1055D0002A956BE475E0AACF023F2FEF120749F43A
:1055E00066E976E083ED92E10E942A956BE375E02F
:1055F0009DCF033F8FEF180709F04DC06FE275E0B4
:10560000CE0101960E94F89744E650E06FEF7FEFDD
:10561000CE0101960E948059CE0101960E949E976C
:1056200061E275E0CE0101960E94F89744E650E0F1
:105630006FEF7FEFCE0101960E94FA57CE010196DF
:105640000E949E9744EF51E062E070E0CE01019627
:105650000E94BEA3BE016F5F7F4F83ED92E10E9467
:105660006597CE0101960E949E9762EA76E0CE0190
:1056700001960E940A9863ED72E1CE0101960E94A4
:10568000B896BC0183ED92E10E944E97CE0101963F
:105690000E949E975BCF0230110509F094C065E12E
:1056A00075E0CE0101960E94F89744E650E06FEF56
:1056B0007FEFCE0101960E948059CE0101960E9493
:1056C0009E9765E075E0CE0101960E94F89744E64A
:1056D00050E06FEF7FEFCE0101960E94FA57CE01A6
:1056E00001960E949E9744EF51E066E070E0CE0183
:1056F00001960E94BEA3BE016F5F7F4F83ED92E1D2
:105700000E946597CE0101960E949E978091D712C4
:105710009091D8120597B0F070E060E083ED92E1CF
:105720000E947696082E000C990BC0970A9750F4A9
:1057300083ED92E10E94A795613523EC7207810504
:105740009105CCF467EF74E0CE0101960E94F897C2
:1057500048EE53E06FEF7FEFCE0101960E94FA57BB
:10576000CE0101960E949E9764ED7BE083ED92E16D
:105770000E942A95EBCE0E94ABB420E030E048ECCA
:1057800052E40E9423B7AB01BC0122E0CE01079690
:105790000E94A69763E076E0CE0101960E940A98E7
:1057A000BE01695F7F4FCE0101960E94B896BC0191
:1057B00083ED92E10E944E97CE0101960E949E9742
:1057C000CE010796C1CE6EEE74E0CE0101960E9426
:1057D000F89744E650E06FEF7FEFCE0101960E940C
:1057E000FA57CE0101960E949E9764ED7BE083ED0F
:1057F00092E10E942A950B3E8FEF180709F0A6CE82
:105800002C960FB6F894DEBF0FBECDBFDF91CF91BF
:105810001F910F91089568EC70E080E090E00E9485
:10582000F19F68ED74E0CE0101960E94F89744EF75
:1058300051E06FEF7FEFCE0101960E94FA574ECEF6
:10584000BF92CF92DF92EF92FF920F931F93CF936D
:10585000DF93CDB7DEB762970FB6F894DEBF0FBE09
:10586000CDBF8C016B016CE57AE0CE010D960E94F4
:105870000A9866ED74E0C8010E94F89776012FEF50
:10588000E21AF20AB701CE0101960E946195BE01AB
:105890006F5F7F4FCE0107960E94019861E776E027
:1058A000CE0107960E94A296BC01C8010E942297D1
:1058B000CE0107960E949E97CE0101960E949E9768
:1058C0008AE0B82EBE9CC001BF9C900D1124FC0143
:1058D000E155FE4E7F018081082E000C990B0E943D
:1058E0003EBC892B09F4B2C0B701CE0101960E94DB
:1058F0000A98BE016F5F7F4FCE0107960E94019804
:105900006BE879E0CE0107960E94A296BC01C8011F
:105910000E942297CE0107960E949E97CE01019683
:105920000E949E97BC9CC001BD9C900D11249C01BF
:1059300021553E4E7901F9016685062E000C770B44
:10594000CE0101960E946195BE016F5F7F4FCE012F
:1059500007960E94019869EA76E0CE0107960E94B8
:10596000A296BE01635F7F4F0E94B896BC01C8013A
:105970000E942297CE0107960E949E97CE01019623
:105980000E949E976FEC74E0C8010E94CB96F701CD
:105990006785062E000C770BCE0101960E9461955B
:1059A000BE016F5F7F4FCE0107960E940198BE0136
:1059B000635F7F4FCE0107960E94B896BC01C80175
:1059C0000E942297CE0107960E949E97CE010196D3
:1059D0000E949E9769EC74E0C8010E94CB96F70183
:1059E00060897189CE0101960E946195BE016F5F49
:1059F0007F4FCE0107960E940198BE01635F7F4FE3
:105A0000CE0107960E94B896BC01C8010E94229759
:105A1000CE0107960E949E97CE0101960E949E9706
:105A200064EC74E0C8010E94CB96F7016289738927
:105A3000CE0101960E946195BE016F5F7F4FC80144
:105A40000E942297CE0101960E949E97CE010D964C
:105A50000E949E97C80162960FB6F894DEBF0FBEF3
:105A6000CDBFDF91CF911F910F91FF90EF90DF900D
:105A7000CF90BF9008954F925F926F927F928F92D6
:105A80009F92AF92BF92CF92DF92EF92FF92CF930D
:105A9000DF93CDB7DEB768970FB6F894DEBF0FBEC1
:105AA000CDBF6B017C010E948DA66D877E878F879D
:105AB000988B89E69EE00E94C28D62E370E080E0F0
:105AC00090E00E94F19F61E0809190040E94409CD0
:105AD00060E080918E040E94409C64E670E080E06B
:105AE00090E00E94F19F60918A0470918B048091F4
:105AF0008C0490918D040E9463150E948015698B1F
:105B00007A8B8B8B9C8B0E949F9C4B015C016AE083
:105B100070E080E090E00E94F19F6BEA76E085EB18
:105B200092E10E942A9520E030E04AE754E4C70160
:105B3000B6010E940AB56D8B7E8B8F8B988F412C9E
:105B4000512C3201C12CD12C7601C701B6010E9423
:105B5000ABB42D893E894F89588D0E94A4B487FF2C
:105B600083C10E948DA62D853E854F855889621B75
:105B7000730B840B950B0E94A9B420E030E04AE738
:105B800054E40E9423B7AB01BC0123E0CE0101968F
:105B90000E94A697BE016F5F7F4F8FEA92E10E943D
:105BA0006597CE0101960E949E970E9480156B0119
:105BB0007C010E949F9C9B01AC01281939094A096C
:105BC0005B0949015A0131ED831637E09306A104C0
:105BD000B1049CF020E030E0A901C701B6010E94A9
:105BE0002CB8181674F426EA3BE944EC5BE3C701D1
:105BF000B6010E94A4B487FF0EC0812C912C5401E1
:105C00002CC026EA3BE944EC5BEBC701B6010E94DD
:105C10002CB8181694F3C501B40128EE33E040E027
:105C200050E00E94E1B5CA01B9010E94ABB44B013A
:105C30005C0129893A894B895C89C701B6010E94B8
:105C400044B620E030E04AE754E40E940AB5A501DA
:105C500094010E9423B74B015C016FEA72E1CE010F
:105C600001960E94019862ED76E0CE0101960E94B5
:105C7000A296BC018FEA92E10E944E97CE01019656
:105C80000E949E9723E0B701A601CE0101960E94D3
:105C9000A697BE016F5F7F4FCE0107960E940198C5
:105CA00069EC76E0CE0107960E94A296BC0189EAD3
:105CB00092E10E944E97CE0107960E949E97CE01D8
:105CC00001960E949E9722E0B501A401CE0107969D
:105CD0000E94A69764E87AE0CE0101960E940A9895
:105CE0006FEA72E1CE0101960E94B8966CEC76E004
:105CF0000E94A29669EA72E10E94B89669E27BE08E
:105D00000E94A296BE01695F7F4F0E94B89660ED27
:105D100076E00E94A296BC0185EB92E10E94229758
:105D2000CE0101960E949E97CE0107960E949E97F3
:105D300020E030E0A901C501B4010E942CB887FD24
:105D400006C06CE57AE089EA92E10E94189722E0A9
:105D5000B501A401CE0101960E94A697BE016F5F16
:105D60007F4FCE0107960E94019860ED76E0CE014C
:105D700007960E94A296BC0189EA92E10E942297AE
:105D8000CE0107960E949E97CE0101960E949E9793
:105D900065EB72E1CE0101960E940198CE01019659
:105DA0000E948457CE0101960E949E97C301B201C2
:105DB00025E030E040E050E00E94E1B5672B682B21
:105DC000692B21F56DEA74E0CE0101960E94F897E7
:105DD00045E050E070E060E0CE0101960E948059FD
:105DE000CE0101960E949E9769EA72E1CE0101966A
:105DF0000E94019845E050E06FEF7FEFCE010196E1
:105E00000E94FA57CE0101960E949E9764ED7BE0B6
:105E100085EB92E10E942A9565E070E080E090E0D9
:105E20000E94F19F0E948DA66B017C012D853E850D
:105E30004F855889C21AD30AE40AF50A0E948015D0
:105E4000698B7A8B8B8B9C8B0E949F9C4B015C0196
:105E50006AE070E080E090E00E94F19F3FEF431A1B
:105E6000530A630A730A71CE60E0809190040E9425
:105E7000409C68960FB6F894DEBF0FBECDBFDF9191
:105E8000CF91FF90EF90DF90CF90BF90AF909F9019
:105E90008F907F906F905F904F9008958F929F9218
:105EA000AF92BF92CF92DF92EF92FF920F931F9328
:105EB000CF93DF93CDB7DEB7EA970FB6F894DEBF86
:105EC0000FBECDBFF82E64ED7BE0CE01C5960E94DB
:105ED0000A988E010B5E1F4F6F2DC8010E940C0D9A
:105EE00018870F831D821E82198289E08A8381E0D0
:105EF0008B838C831C8A1B8ACE0101960E94C5115C
:105F0000CE0101960E946810CE0101960E94E1A286
:105F10000E8110E00330110509F488C163EA74E0D2
:105F2000CE01C5960E94299764ED7BE085EB92E156
:105F30000E942A95BE016B5C7F4FCE0183960E9422
:105F400001984AE050E070E060E0CE0183960E9444
:105F50008059CE0183960E949E9761E080E00E9466
:105F6000F48A66EF76E0CE01C5960E942A958BE30F
:105F7000C82E8CE0D82EF12CE12CE016F1060CF0A6
:105F8000F0C06E2DCE0101960E945911F6012191AB
:105F90003191419151916F010E9445B64B015C01D5
:105FA000FFEFEF1AFF0A20E030E04CEF52EC0E94C6
:105FB000A4B487FF33C0B701CE0189960E946195D2
:105FC00065E478E0CE0183960E940A98BE01675D81
:105FD0007F4FCE0183960E94B89664ED76E00E94D2
:105FE000A296BC0185EB92E10E942297CE01839696
:105FF0000E949E97CE0189960E949E9701301105BE
:1060000009F055C081E0E816F10409F0B6CF65EB60
:1060100072E1CE01C5960E944E97AFCF22E0B50146
:10602000A401CE018F960E94A697B701CE01899652
:106030000E94619565E478E0CE0183960E940A98FB
:10604000BE01675D7F4FCE0183960E94B89666E6DB
:1060500079E00E94A296BE01615D7F4F0E94B896D2
:10606000BC0189EA92E10E944E97CE0183960E947C
:106070009E97CE0189960E949E97CE018F960E9490
:106080009E9769EA72E1CE0183960E9401986CE5C1
:106090007AE0CE0183960E94A296BC0185EB92E144
:1060A0000E942297CE0183960E949E97A7CF02302E
:1060B000110511F522E0B501A401CE0183960E94DD
:1060C000A697BE016D5D7F4FCE0189960E94019813
:1060D0006CE57AE0CE0189960E94A296BC01CE01C1
:1060E000C5960E942297CE0189960E949E97CE0166
:1060F00083960E949E9741CF0330110509F43DCF4E
:1061000069EA72E1CE0183960E94019844E150E071
:106110006FEF7FEFCE0183960E94FA57CE018396F0
:106120000E949E9761ED75E0CE0183960E940A98C9
:10613000CE0183960E94DC57CE0183960E949E97E3
:1061400080918704882309F418CF8091E70488237D
:1061500009F413CF60ED77E080E090E00E94F19FBA
:106160000CCFCE01C5960E94B29585EB92E10E94BC
:10617000B2950115110579F560E974E085EB92E1BE
:106180000E94299765E874E0CE0183960E94F897F3
:106190004AE050E06FEF7FEFCE0183960E94FA57FE
:1061A000CE0183960E949E97CE01C5960E949E972F
:1061B000EA960FB6F894DEBF0FBECDBFDF91CF9148
:1061C0001F910F91FF90EF90DF90CF90BF90AF9015
:1061D0009F908F900895043011050CF5BE016B5C03
:1061E0007F4FCE0183960E9401984AE050E06FEF06
:1061F0007FEFCE0183960E94FA57CE0183960E94CC
:106200009E9761ED75E0CE0183960E940A98CE01BB
:1062100083960E94DC57CE0183960E949E9760EE83
:1062200076E085EB92E10E941897BECF63EF76E0AF
:10623000CE01C5960E942A95BE016B5C7F4FCE01B0
:1062400083960E9401984AE050E070E060E0CE0141
:1062500083960E948059CE0183960E949E9764ED9A
:106260007BE085EB92E10E942A9565EB72E1CE011D
:10627000C5960E944E9710E000E0602FCE01019677
:106280000E9459116B017C0122E0BC01A601CE01E4
:1062900083960115110509F077C00E94A697BE01EB
:1062A0006D5D7F4F86EB93E10E94559ACE018396F8
:1062B0000E949E9722E0B701A601CE0183960E941C
:1062C000A697BE016D5D7F4FCE0189960E94019811
:1062D0006CE57AE0CE0189960E94A296BC0185EB1E
:1062E00092E10E942297CE0189960E949E97CE014C
:1062F00083960E949E970F5F1F4F0330110509F090
:10630000BCCFCE01C5960E94B295BE016B5C7F4F9B
:10631000CE0183960E9401984AE050E06FEF7FEF34
:10632000CE0183960E94FA57CE0183960E949E97D3
:1063300061ED75E0CE0183960E940A98CE018396A6
:106340000E94DC57CE0183960E949E9785EB92E1D6
:106350000E94B29569EF76E0CE0183960E940A987A
:1063600065EB72E1CE0183960E94B89660EE76E00E
:106370000E94A296BC0185EB92E10E944E97CE014D
:1063800083960E949E9710CF0E94A697BE016D5DD6
:106390007F4FCE0189960E9401986CE57AE0CE018C
:1063A00089960E94A296BC01CE01C5960E942297B2
:1063B000CE0189960E949E9779CF8F929F92AF923D
:1063C000BF92CF92DF92EF92FF920F931F93CF93E2
:1063D000DF93CDB7DEB768970FB6F894DEBF0FBE78
:1063E000CDBF6C0180919411909195110197C9F0E6
:1063F00064ED7BE0C6010E940A98C60168960FB65C
:10640000F894DEBF0FBECDBFDF91CF911F910F91EA
:10641000FF90EF90DF90CF90BF90AF909F908F90C4
:10642000089563E077E0CE010D960E940A98BE01C0
:10643000635F7F4F8CEC9DE00E94559A6CE271E0A7
:1064400080E090E00E94F19FCE0143960E94FE6D95
:1064500064E670E080E090E00E94F19F10E000E0D0
:1064600085E0A82EB12C9AE0892E912C6EE077E081
:10647000CE0101960E940A98BE016F5F7F4FCE0148
:1064800043960E945B967C01CE0101960E949E97E6
:10649000A7014F5F5F4FBE016D5E7F4FCE0101963A
:1064A0000E94CA58BE016F5F7F4FCE010D960E94B9
:1064B0006597CE0101960E949E9789899A89892BBA
:1064C00009F170E060E0CE010D960E947696082EEC
:1064D000000C990BC0970A97A8F460E177E0CE0111
:1064E00001960E940A98BE016F5F7F4FCE010D9604
:1064F0000E948796E82ECE0101960E949E97FF2467
:10650000F394E110F12C64EB74E0CE0101960E944B
:10651000F89744E150E06FEF7FEFCE0101960E94C3
:10652000D658CE0101960E949E970F5F1F4F62E3DF
:1065300070E080E090E00E94F19FC801B5010E94E8
:10654000BBB90197C1F4CE0101960E94B16C8D8157
:106550009E81892B09F46AC0BE016F5F7F4F83ED76
:1065600092E10E944E970E94674BFF24F394CE0164
:1065700001960E949E97CE0101960E94FE6DBE017B
:106580006F5F7F4FCE0143960E946597CE010196C3
:106590000E949E9762E370E080E090E00E94F19F8D
:1065A0000436110519F0FF2009F460CF8091040D25
:1065B0008823F1F064ED75E0CE0101960E940A98FF
:1065C000BE01635F7F4FCE0101960E94B896BC0169
:1065D000CE0107960E940198CE0107960E9484572B
:1065E000CE0107960E949E97CE0101960E949E972B
:1065F00089899A89892B61F070E060E0CE010D965F
:106600000E947696082E000C990BC0970A9738F1D5
:1066100068E177E0C6010E940A98CE0143960E9485
:106620009E97CE010D960E949E97E7CE04311105EC
:106630000CF49DCFC801B4010E94BBB9892B09F0AD
:1066400096CFBE01635F7F4F8CEC9DE00E94559A10
:1066500068EC70E080E090E00E94F19F88CF60E1FC
:1066600077E0CE0101960E940A98BE016F5F7F4FCE
:10667000CE010D960E948796182FCE0101960E949A
:106680009E971111C5CFBE01635F7F4FC6010E9467
:10669000EF97C3CF2F923F924F925F926F927F926C
:1066A0008F929F92AF92BF92CF92DF92EF92FF9222
:1066B0000F931F93CF93DF93CDB7DEB76D970FB6D0
:1066C000F894DEBF0FBECDBF61E089E10E94409C1F
:1066D00061E089E10E94129C0E947C9464E277E070
:1066E00083EA9FE00E94C898F12CE12C17E2812FE9
:1066F0000E94D98A0E94B49D811195C160E377E020
:1067000083EA9FE00E94539A40E150E0612F83EAC0
:106710009FE00E94B1981093BA136CE477E083EA8B
:106720009FE00E94539A40E150E0612F83EA9FE08E
:106730000E94B1982FEFE21AF20A1F5F1034B9F6E7
:1067400061E877E0EF2811F067E977E083EA9FE0FE
:106750000E94C8980E9423A680E40E94E38A0CEC61
:1067600014E0D8016D918D0186EB93E10E949D129A
:10677000B4E0043D1B07A9F70E94B8570E94D41546
:106780008EE492E00E94CBB580932B0D8FE492E0D3
:106790000E94CBB580932C0D80912B0D90912C0DE8
:1067A0001816190664F41092CB04019741F4109264
:1067B0002C0D10922B0D8EE492E00E94F68C6BED66
:1067C0007BE0CE0101960E94F8974AE050E06FEF1F
:1067D0007FEFCE0101960E948059CE0101960E9462
:1067E0009E9740E052EC61E070E083EA9FE00E94F7
:1067F00086588091CB04882331F068EE73E080E006
:1068000090E00E94F19F83EA9FE00E9408888B8BB2
:106810006FEAE62E61E1F62E0CE211E0C8010E945B
:10682000CBB5F70181937F010F5F1F4F0632F2E076
:106830001F07A1F78091B011181624F42B892D366B
:1068400009F021C164ED7BE0CE010D960E940A980B
:106850001092AF1188E18093B01184E08093B11160
:106860001092B6111092B71165E17AE0CE010D9643
:106870000E942A9589EB91E1009739F044E050E0BD
:10688000BC01CE010D960E94758D81E08093BD11F3
:1068900083E08093BE1182E090E09093C0118093DA
:1068A000BF1185E090E09093C2118093C11162E125
:1068B0007AE0CE010D960E942A9583EC91E1009733
:1068C00039F044E050E0BC01CE010D960E94758D78
:1068D00082E08093C71183E08093C81182E090E04A
:1068E0009093CA118093C91185E090E09093CC11E8
:1068F0008093CB116FE07AE0CE010D960E942A952D
:106900008DEC91E1009739F044E050E0BC01CE01FC
:106910000D960E94758D83E08093D1118093D211E2
:1069200082E090E09093D4118093D31185E090E0C1
:106930009093D6118093D5116EE977E0CE010D9634
:106940000E942A9587ED91E1009739F044E050E0EC
:10695000BC01CE010D960E94758D85EF8093DB11F1
:1069600083E08093DC1182E090E09093DE118093CD
:10697000DD1185E090E09093E0118093DF118CE2CF
:1069800091E00E94988D8091040D882311F1CE0131
:1069900001960E94881CBE016F5F7F4F83EA9FE0D3
:1069A0000E94639ACE0101960E949E9768E17AE068
:1069B00083EA9FE00E94759A2AE04AE050E060E096
:1069C00070E083EA9FE00E94619883EA9FE00E9462
:1069D000AD986EED79E0CE0107960E94F897BE0162
:1069E000695F7F4F83EA9FE00E94639A10E000E0B6
:1069F0008091B111082E000C990B0817190724F586
:106A0000B801CE0101960E94202CBE016F5F7F4F1E
:106A100083EA9FE00E94639ACE0101960E949E97AE
:106A20000F5F1F4FE5CF843009F087CE66E677E031
:106A300083EA9FE00E94539A40E150E0612F83EA8D
:106A40009FE00E94B19879CECE0107960E949E9752
:106A50008091040D882399F068EF79E083EA9FE044
:106A60000E94759A2AE04AEF50E060E070E083EA05
:106A70009FE00E94619883EA9FE00E94AD98CE015A
:106A80000D960E949E978091B81181118091AF114F
:106A90008093AA110E948DA66093A6117093A711EE
:106AA0008093A8119093A9113B8910E0323709F423
:106AB00099C55EE1252E51E1352E710110E000E00F
:106AC000C8010E94CBB5D7018D937D010F5F1F4F89
:106AD00008381105A9F780911E1190911F11A091FE
:106AE0002011B091211185369105A105B1050CF455
:106AF0009BC18093C7049093C804A093C904B0932A
:106B0000CA048091221190912311A0912411B09177
:106B100025118093C3049093C404A093C504B0933B
:106B2000C6048091261190912711A0912811B0914F
:106B300029118093BF049093C004A093C104B09323
:106B4000C2046AE371E1CE0101960E940A98BE0177
:106B50006F5F7F4F80EB93E10E946597CE010196B6
:106B60000E949E9768E971E1CE0101960E940A9801
:106B7000BE016F5F7F4F8AEA93E10E946597CE0165
:106B800001960E949E9723E030E050E040E060EBE9
:106B900073E1CE0107960E941B9823E030E050E09D
:106BA00040E06AEA73E1CE0101960E941B982D81B4
:106BB0003E818B859C852817390709F589819A8143
:106BC0006F817885009759F06115710509F0F1C062
:106BD000232B09F4F1C0DC018C9190E00DC061150C
:106BE000710509F4E9C0232B09F4E6C0FB0180819B
:106BF00090E091958195910911E0892B09F010E0C1
:106C0000CE0101960E949E97CE0107960E949E9704
:106C1000111106C060EB73E18AEA93E10E944E977E
:106C200080912A1190912B11A0912C11B0912D11CE
:106C30008093BB049093BC04A093BD04B093BE04A6
:106C400080912E1190912F11A0913011B09131119E
:106C50008093B7049093B804A093B904B093BA0496
:106C60008091321190913311A0913411B09135116E
:106C70008093B3049093B404A093B504B093B60486
:106C80008091361190913711A0913811B09139113E
:106C90008093AF049093B004A093B104B093B20476
:106CA000E0919611F0919711FD8FEC8FF093D50440
:106CB000E093D4048091521190915311A0915411FA
:106CC000B09155118C8B9D8BAE8BBF8B8093DA046A
:106CD0009093DB04A093DC04B093DD0480916811F1
:106CE00090916911A0916A11B0916B11888F998F61
:106CF000AA8FBB8F8093D6049093D704A093D80417
:106D0000B093D904409042115090431160904411C7
:106D1000709045114092AB045092AC046092AD0467
:106D20007092AE048090461190904711A090481147
:106D3000B09049118092A7049092A804A092A9044F
:106D4000B092AA040091A4111091A511B801012ECE
:106D5000000C880B990B0E94ABB46B017C01AC0159
:106D60009B010E9491B9811104C01093070C0093FC
:106D7000060C209195043091960490E080E028174D
:106D80003907E4F0D101D8964D915C91D99757FF1E
:106D90000BC0FC01EE0FFF1FEB56FB4F40815181F2
:106DA000D9965C934E93D8970196B2E02B0E311C86
:106DB000E6CF0E9456BC20CF11E022CFA301920162
:106DC000C301B2010E9491B9811109C0A5019401CA
:106DD000C501B4010E9491B9882309F472C30E94CD
:106DE000380D3CE6A32E31E1B32E0BE31CE0D501B8
:106DF000CD90DD90ED90FD905D01A7019601C7015A
:106E0000B6010E9491B9811105C0F801C082D182FA
:106E1000E282F3820C5F1F4FFCE003361F0739F755
:106E200081E090E00E948B0D1B891257113009F40C
:106E3000D9C32B892E3609F4D4C380911E119091A9
:106E40001F11A0912011B091211185369105A10546
:106E5000B1050CF4C7C380919411909195118D7F69
:106E6000892B41F440E855E260E070E08CEC9DE055
:106E70000E9486588091941190919511019741F448
:106E800040E052EC61E070E08CEC9DE00E9486589E
:106E900064E670E080E090E00E94F19F80919411A0
:106EA00090919511892B09F0B8C02B892E3671F07D
:106EB00080911E1190911F11A0912011B09121116C
:106EC00085369105A105B1050CF0A7C064ED7BE006
:106ED000CE0107960E940A9866EA77E0CE010196F5
:106EE0000E940A986AEA73E1CE0101960E94B89660
:106EF000BC01CE0107960E944E97CE0101960E94DA
:106F00009E97BE01695F7F4F8CEC9DE00E94559A71
:106F100068EB7BE080E090E00E94F19FBE01695F3A
:106F20007F4FCE0101960E940198CE0101960E94EA
:106F3000825BCE0101960E949E976CE271E080E038
:106F400090E00E94F19F4091AE135091AF134250D8
:106F500051096AEA73E1CE0101960E94CA58BE0146
:106F60006F5F7F4FCE0107960E946597CE01019615
:106F70000E949E97BE01695F7F4FCE0101960E94DD
:106F80000198BE01695F7F4FCE0101960E94B896BD
:106F9000BC01CE0107960E944E97CE0101960E9439
:106FA0009E976EEA77E0CE0101960E940A98BE0194
:106FB000695F7F4FCE0101960E94B896BC01CE0159
:106FC00007960E944E97CE0101960E949E97BE01A1
:106FD000695F7F4F8CEC9DE00E94559A68EB7BE0E7
:106FE00080E090E00E94F19FBE01695F7F4FCE017B
:106FF00001960E940198CE0101960E94825BCE010B
:1070000001960E949E976CE271E080E090E00E9401
:10701000F19FCE0107960E949E9764E670E080E0A3
:1070200090E00E94F19FF89482E08093B0008093FA
:10703000B10094E69093B3001092B2008093700078
:10704000789480934C1010924F1080914D1060E016
:107050000E94409C65EB7BE0CE0101960E94F89770
:107060004AE050E06FEF7FEFCE0101960E94805919
:10707000CE0101960E949E9764ED7BE085EB92E144
:107080000E942A958091941190919511892B31F449
:107090006AE676E085EB92E10E942A958091941150
:1070A00090919511019731F464E676E085EB92E1D9
:1070B0000E942A958091941190919511029731F434
:1070C0006EE676E085EB92E10E942A958091B912F6
:1070D0009091BA12892BC1F06AEA73E185EB92E1D3
:1070E0000E94229765EB72E1CE0101960E94019801
:1070F0004AE050E06FEF7FEFCE0101960E94FA5711
:10710000CE0101960E949E978091941190919511C5
:10711000019709F05CC0CE0107960E94DD318B8596
:107120009C85009709F449C0EF81F88520812223CE
:1071300009F443C0079708F440C062EA7BE085EB9E
:1071400092E10E942997BE01695F7F4F85EB92E132
:107150000E94229765EB72E1CE0101960E94019890
:10716000CE0101960E948457CE0101960E949E97FF
:1071700069E97BE0CE0101960E94F89748EC50E067
:107180006FEF7FEFCE0101960E94D658CE01019697
:107190000E949E97BE01695F7F4FCE0101960E94BB
:1071A000019848EC50E06FEF7FEFCE0101960E940E
:1071B000FA57CE0101960E949E9768EE73E080E038
:1071C00090E00E94F19FCE0107960E949E976DE786
:1071D0007BE085EB92E10E94299764ED75E0CE019A
:1071E00001960E940A986AEA73E1CE0101960E9414
:1071F000B89665EB72E10E94B896BC0185EB92E10E
:107200000E944E97CE0101960E949E9765EB72E117
:10721000CE0101960E940198CE0101960E948457EA
:10722000CE0101960E949E9764ED7BE085EB92E192
:107230000E942A9564E670E080E090E00E94F19F51
:107240000E947C9464E670E080E090E00E94F19FF0
:1072500083E20E94D98A81E090E00E94D48A0E9451
:10726000B49D83E090E09093050C8093040C8CE433
:107270000E94CBA66B017C0162E370E080E090E0AD
:107280000E94F19FA7019601C701B6010E9491B922
:107290008823B9F086E60E94CBA66B017C0162E3ED
:1072A00070E080E090E00E94F19FA7019601C70185
:1072B000B6010E9491B9882321F01092050C10921A
:1072C000040C8091040C9091050C039709F08CC27A
:1072D00068E67BE0CE0101960E94F897CE01019608
:1072E0000E94825BCE0101960E949E9783E080936C
:1072F000D9120E947C9480ED0E94A29E853509F0EF
:1073000096C28AEA0E94BF9E9093DB128093DA12A3
:107310008CEA0E94BF9E9093DD128093DC128EEA6D
:107320000E94BF9E9093DF128093DE1280EB0E943A
:10733000BF9E9093EB128093EA1282EB0E94BF9E55
:107340009093ED128093EC1284EB0E94BF9E909379
:10735000EF128093EE1286EB0E94BF9E9093E11293
:107360008093E01288EB0E94BF9E9093E31280937B
:10737000E2128AEB0E94BF9E9093E5128093E41282
:107380008CEB0E94BF9E9093E7128093E6128EEBE7
:107390000E94BF9E9093E9128093E8126FE27BE017
:1073A00085EB92E10E9429970E9491A00E94ABB4C4
:1073B0000E94CFB70E94ABB420E030E048EC52E42A
:1073C0000E9423B7AB01BC0122E0CE0101960E94CE
:1073D000A697BE016F5F7F4FCE0107960E9401986E
:1073E00067E076E0CE0107960E94A296BC0185EB8D
:1073F00092E10E942297CE0107960E949E97CE01AD
:1074000001960E949E9765EB72E1CE0101960E9463
:107410000198CE0101960E94825BCE0101960E94E6
:107420009E9769E17BE085EB92E10E94299760914C
:10743000C7047091C8048091C9049091CA040E9445
:10744000ABB420E030E048EC52E40E9423B7AB013B
:10745000BC0122E0CE0101960E94A697BE016F5F9B
:107460007F4FCE0107960E94019867E076E0CE013B
:1074700007960E94A296BC0185EB92E10E9422979A
:10748000CE0107960E949E97CE0101960E949E977C
:1074900065EB72E1CE0101960E940198CE01019642
:1074A0000E94825BCE0101960E949E973B893136F5
:1074B00009F04EC281E00E94AE5B81E00E946861EB
:1074C000C6C100914A11602F002E000C770B880B6B
:1074D000990B0E94ABB49B01AC010E9491B9811140
:1074E0007ECC60904B1170904C11B301072C000CB6
:1074F000880B990B0E94ABB49B01AC010E9491B91F
:1075000081116DCC10914D11612F012E000C770B64
:10751000880B990B0E94ABB49B01AC010E9491B9FE
:1075200081115DCC80904E1190904F11A090501120
:10753000B0905111A5019401C501B4010E9491B907
:1075400081114DCC2C893D894E895F89CA01B901D1
:107550000E9491B9811143CC288D398D4A8D5B8D64
:10756000CA01B9010E9491B9811139CC609194117D
:1075700070919511072E000C880B990B0E94ABB4EB
:107580009B01AC010E9491B9811129CCEC8DFD8D3C
:10759000BF01FF0F880B990B0E94ABB49B01AC019C
:1075A0000E9491B981111BCCA7019601C701B601B8
:1075B0000E9491B9811113CC04300CF010CC15301D
:1075C0000CF00DCCFBEF6F1671040CF008CC20E032
:1075D00030E0A901C501B4010E94A4B487FDFFCB2E
:1075E00000CC1CEF8091C7049091C804A091C904FD
:1075F000B091CA0480931E1190931F11A093201183
:10760000B09321118091C3049091C404A091C5044A
:10761000B091C6048093221190932311A09324115A
:10762000B09325118091BF049091C004A091C10432
:10763000B091C2048093261190932711A093281132
:10764000B09329113B89333751F160E080EB93E12E
:107650000E94F59660E08AEA93E10E94F5964091D7
:10766000B4135091B5134115510549F08AE391E1E6
:10767000009729F0BC0180EB93E10E94758D409149
:10768000AE135091AF134115510549F088E991E1CE
:10769000009729F0BC018AEA93E10E94758D8091E0
:1076A000BB049091BC04A091BD04B091BE04809332
:1076B0002A1190932B11A0932C11B0932D1180912E
:1076C000B7049091B804A091B904B091BA04809322
:1076D0002E1190932F11A0933011B09331118091FE
:1076E000B3049091B404A091B504B091B604809312
:1076F000321190933311A0933411B09335118091CE
:10770000AF049091B004A091B104B091B204809301
:10771000361190933711A0933811B093391190E03E
:1077200080E00E944B8DEBE3FCE0ACE6B1E183E648
:107730009CE041915191619171914D935D936D9355
:107740007D938E179F07A9F765EC7BE0CE0101962C
:107750000E94F897CE0101960E94825BCE010196AD
:107760000E949E9795E9C92E94E0D92E26E5A22E77
:1077700021E1B22EF12CE12C809195049091960498
:107780008E159F054CF1D6018D919D916D01F501EE
:10779000819391935F018091040D8823C9F064ED7A
:1077A00075E083EA9FE00E94539A4AE050E0B701F7
:1077B00083EA9FE00E94069A61EA77E083EA9FE00D
:1077C0000E94539AF6013297808191810E94409ADB
:1077D000FFEFEF1AFF0AD0CF123008F03CCB90E059
:1077E00080E00E944B8D37CB86E00E94CC9FBC018D
:1077F00090E080E00E94A9B42AE037ED43EA5CE320
:107800000E940AB523E333E948E853E40E9444B6F2
:1078100020E030E048E453E40E94A4B487FF66CD42
:1078200082E090E090939404809393045FCD62E4AF
:107830007BE0CE0101960E94F897CE0101960E944E
:107840008457CE0101960E949E971092920464E69E
:1078500070E080E090E00E94F19F8091040C909194
:10786000050C892BA1F461E0809190040E94409C5A
:1078700060E080918E040E94409C60918A04709127
:107880008B0480918C0490918D040E94631560E0BC
:10789000809190040E94409C8091CB04882331F019
:1078A00068EE73E080E090E00E94F19F62E17AE090
:1078B00081EC92E10E942A9582E090E09093030C83
:1078C0008093020C8091CB04882309F494C16FED5E
:1078D0007AE0CE0101960E94F8974CE251E06FEFFA
:1078E0007FEFCE0101960E94FA57CE0101960E94C9
:1078F0009E9760918804709189048091D40490913E
:10790000D5040E94475584E1C82ED12CE12CF12CDE
:1079100010E000E00F5F1F4FC701B6010E94F19F0A
:1079200060918804709189048091D4049091D50469
:107930000E944755033011052CF00A301105DCF484
:10794000892BE1F044E1C40ED11CE11CF11CE2CF13
:1079500083EA9FE00E940888182F64E670E080E0C8
:1079600090E00E94F19F113609F4A4CD80E00E94BE
:10797000AE5B80E0A3CD892B09F0EDC18091D404EA
:107980009091D5048B30910509F095C18091131326
:1079900090911413A0911513B09116138093FE0BC0
:1079A0009093FF0BA093000CB093010C80910F13E8
:1079B00090911013A0911113B09112138093FA0BB0
:1079C0009093FB0BA093FC0BB093FD0B4091FE0B2F
:1079D0005091FF0B6091000C7091010C21E0CE01E1
:1079E00001960E94A69766EF76E0CE0107960E9468
:1079F0000A98BE016F5F7F4FCE0107960E94B8962E
:107A0000BC0185EB92E10E944E97CE0107960E9441
:107A10009E97CE0101960E949E974091FA0B50913D
:107A2000FB0B6091FC0B7091FD0B21E0CE010196E8
:107A30000E94A69765EB77E0CE0107960E940A9810
:107A4000BE016F5F7F4FCE0107960E94B896BC01C2
:107A500085EB92E10E942297CE0107960E949E97A5
:107A6000CE0101960E949E976FE47BE085EB92E148
:107A70000E94189764ED7BE0CE0101960E940A985F
:107A800044E150E070E060E0CE0101960E94805930
:107A9000CE0101960E949E97C090FE0BD090FF0BE6
:107AA000E090000CF090010C20E030E0A901C7014B
:107AB000B6010E942CB820E030E040E05FE387FD93
:107AC0001AC1C701B6010E9445B60E94CFB7AB01EB
:107AD000BC01CE0101960E943495BE016F5F7F4FBD
:107AE0008FEA92E10E946597CE0101960E949E97CF
:107AF00060E087E00E94F48A6FEA72E186EB93E12E
:107B00000E94559A6FED86EB93E10E94DA986BEB39
:107B100077E086EB93E10E94539A6091FA0B7091A3
:107B2000FB0B8091FC0B9091FD0B0E94CFB74AE0BC
:107B300050E086EB93E10E94069A6FE47BE086EBCF
:107B400093E10E94539A64E670E080E090E00E9426
:107B5000F19FC090FE0BD090FF0BE090000CF090D6
:107B6000010C20E030E040EF51E4C701B6010E9473
:107B70002CB860ED7AE087FF28C020E030E040EDCF
:107B800051E4C701B6010E942CB887FDB9C060EC72
:107B90007AE0CE0101960E94F8974AE050E06FEF3C
:107BA0007FEFCE0101960E94FA57CE0101960E9406
:107BB0009E978091CB04882331F06CED75E080E0D6
:107BC00090E00E94F19F60EB7AE0CE0101960E9466
:107BD000F8974AE050E06FEF7FEFCE0101960E94E8
:107BE000FA57CE0101960E949E9762E370E080E012
:107BF00090E00E94F19F61E07BE085EB92E10E94C2
:107C0000299764ED75E0CE0101960E940A986AEA10
:107C100073E1CE0101960E94B89665EB72E10E9475
:107C2000B896BC0185EB92E10E944E97CE01019679
:107C30000E949E9765EB72E1CE0101960E94019829
:107C4000CE0101960E948457CE0101960E949E9714
:107C50006DEE7AE085EB92E10E94299765EB72E187
:107C6000CE0101960E940198CE0101960E94845790
:107C7000CE0101960E949E9764ED7BE085EB92E138
:107C80000E942A956D960FB6F894DEBF0FBECDBF49
:107C9000DF91CF911F910F91FF90EF90DF90CF90E8
:107CA000BF90AF909F908F907F906F905F904F901C
:107CB0003F902F9008958631910509F467CE0C9777
:107CC00009F084CE8091F10B9091F20BA091F30B0F
:107CD000B091F40B8093FE0B9093FF0BA093000CDC
:107CE000B093010C8091ED0B9091EE0BA091EF0BF6
:107CF000B091F00B63CEC701B6010E9444B6E5CE49
:107D000020E030E040EB51E4C701B6010E942CB8FE
:107D100062EA7AE087FF59CF63E97AE0CE01019603
:107D20000E94F8974AE050E06FEF7FEFCE01019696
:107D30000E94FA57CE0101960E949E978091CB0433
:107D4000882331F06CED75E080E090E00E94F19FB7
:107D500065E87AE03ACF0E94B8576EE170E080E0C3
:107D600090E00E94F19F0E943CA06B017C0164E6C0
:107D700070E080E090E00E94F19F66EF76E085EB96
:107D800092E10E942A9521E0B701A601CE01019659
:107D90000E94A697BE016F5F7F4F85EB92E10E9424
:107DA0002297CE0101960E949E9765EB72E1CE016B
:107DB00001960E9401984AE050E070E060E0CE0138
:107DC00001960E948059CE0101960E949E97809153
:107DD0008704882379F08091E704882359F06FEDB8
:107DE00086EB93E10E94DA9861ED75E086EB93E112
:107DF0000E94539A60ED75E085EB92E10E9418971E
:107E0000C092FE0BD092FF0BE092000CF092010C9E
:107E100020E030E040EF51E4C701B6010E942CB8E9
:107E200065E77AE087FF28C020E030E040ED51E4CC
:107E3000C701B6010E942CB887FD3EC065E67AE016
:107E4000CE0101960E94F8974AE050E06FEF7FEF75
:107E5000CE0101960E94FA57CE0101960E949E978C
:107E60008091CB04882331F06CED75E080E090E0E8
:107E70000E94F19F65E57AE0CE0101960E94F89795
:107E80004AE050E06FEF7FEFCE0101960E94FA5773
:107E9000CE0101960E949E976CE271E080E090E036
:107EA0000E94F19F8091CB04882309F4A4CE68EE50
:107EB00073E080E090E09DCE20E030E040EB51E4C4
:107EC000C701B6010E942CB867E47AE087FFD4CFDF
:107ED00068E37AE0CE0101960E94F8974AE050E00C
:107EE0006FEF7FEFCE0101960E94FA57CE01019607
:107EF0000E949E978091CB04882331F06CED75E051
:107F000080E090E00E94F19F6AE27AE0B5CF3F9274
:107F10004F925F926F927F928F929F92AF92BF9299
:107F2000CF92DF92EF92FF920F931F93CF93DF9345
:107F3000CDB7DEB7E4970FB6F894DEBF0FBECDBF66
:107F400063ED72E18DEC92E10E944E970E941395D1
:107F50006EEB77E0CE0101960E940A98BE016F5F3A
:107F60007F4F8DEC92E10E948796182FCE010196EB
:107F70000E949E97112309F48FC026E030E045E06F
:107F800050E063ED72E1CE0101960E941B98BE01A4
:107F90006F5F7F4F8FEA92E10E946597CE01019655
:107FA0000E949E978FEA92E10E94A7956B0166E678
:107FB00079E0CE0101960E940A98BE016F5F7F4F63
:107FC00083ED92E10E940F96AC014F5F5F4F63ED2E
:107FD00072E1CE010B960E94CA58BE01655F7F4FC9
:107FE0008FEA92E10E946597CE010B960E949E97C0
:107FF000CE0101960E949E978FEA92E10E94A7957A
:108000009B01E5E9F4E041E050E0A0919504B091D6
:108010009604A417B5075CF0A281B381A217B30739
:1080200011F4138212824F5F5F4F3296EECFF6014A
:10803000EE0FFF1FEB56FB4F7183608382E090E0F1
:108040000E948B0D63ED72E1CE0101960E940198B2
:10805000CE0101960E94825BCE0101960E949E97FE
:1080600090E080E00E944B8D1092EC041091EC04A3
:10807000112311F40C94654B63ED72E1CE0101966E
:108080000E940198CE0101960E94825BCE0101966A
:108090000E949E970C944C4B64EC77E0CE010196C5
:1080A0000E940A98BE016F5F7F4F8DEC92E10E94A3
:1080B0008796182FCE0101960E949E971123F1F00A
:1080C000E5E9F4E081E090E0209195043091960498
:1080D0002817390774F0863091052CF49383828336
:1080E00001963296F1CF9C012E5F3F4F338322835E
:1080F000F7CF82E090E00E948B0DB2CF6AEC77E080
:10810000CE0101960E940A98BE016F5F7F4F8DECF1
:1081100092E10E948796182FCE0101960E949E97A9
:108120001123D1F080912B0D90912C0D892B81F48E
:1081300081E090E090932C0D80932B0D8EE492E0E3
:108140000E94F68C68EC70E080E090E00E94F19F65
:10815000F0E0E0E019958ACF61ED77E0CE0101967D
:108160000E940A98BE016F5F7F4F8DEC92E10E94E2
:108170008796182FCE0101960E949E97112399F1A0
:1081800069ED77E0CE0101960E940A9864EA73E1F6
:10819000CE0101960E94B896BC0185EB92E10E9447
:1081A0004E97CE0101960E949E9764ED75E0CE0138
:1081B00001960E940A9865EB72E1CE0101960E9439
:1081C000B896BC01CE010B960E940198CE010B9689
:1081D0000E948457CE010B960E949E97CE01019675
:1081E0000E949E9741CF63EE77E0CE0101960E94F8
:1081F0000A98BE016F5F7F4F8DEC92E10E948796D7
:10820000182FCE0101960E949E97112369F069E50F
:1082100079E085EB92E10E9429976AEA73E185EBA8
:1082200092E10E942297C1CF6AEE77E0CE010196DB
:108230000E940A98BE016F5F7F4F8DEC92E10E9411
:108240008796182FCE0101960E949E97112309F15F
:1082500066E379E085EB92E10E94299765EB72E194
:10826000CE0101960E940198CE0101960E9484578A
:10827000CE0101960E949E970E94380D1092EC0448
:1082800060EF77E083ED92E10E942A950E94674BB0
:10829000EDCE64EF77E0CE0101960E940A98BE0110
:1082A0006F5F7F4F8DEC92E10E948796182FCE0171
:1082B00001960E949E97112309F495C066E679E025
:1082C000CE0101960E940A98BE016F5F7F4F83ED39
:1082D00092E10E940F96AC014F5F5F4F63ED72E138
:1082E000CE010B960E94CA58BE01655F7F4F8FEA90
:1082F00092E10E946597CE010B960E949E97CE0157
:1083000001960E949E978FEA92E10E94A7958B01A9
:1083100069E279E085EB92E10E9429978091AF11A3
:10832000882331F06DE179E085EB92E10E94299795
:108330000115110559F465EB72E1CE0101960E9419
:108340000198CE0101960E94845704C7CE01019680
:108350000E94881CCE0101960E948457CE0101968E
:108360000E949E97023011050CF47ECE6EED79E0EE
:10837000CE010B960E94F897BE01655F7F4FCE013C
:1083800001960E940198CE0101960E948457CE0169
:1083900001960E949E97F12CE12C8091B111082E3C
:1083A000000C990BE816F9068CF4B701CE01019682
:1083B0000E94202CCE0101960E948457CE01019686
:1083C0000E949E97FFEFEF1AFF0AE7CFCE010B96B0
:1083D0000E949E970230110509F446CE8CE291E08E
:1083E0000E94988D41CE6BEF77E0CE0101960E94FE
:1083F0000A98BE016F5F7F4F8DEC92E10E948796D5
:10840000182FCE0101960E949E97112309F482C372
:1084100063ED72E1CE018F960E94019866E679E0E5
:10842000CE0101960E940A98BE016F5F7F4FCE0178
:108430008F960E940F96AC014F5F5F4FBE01615D4A
:108440007F4FCE0189960E94CA58CE0101960E94A4
:108450009E97BE01615D7F4FCE0101960E940198FB
:10846000CE0101960E94825BCE0101960E949E97EA
:108470006FEF77E0CE0101960E940A98BE016F5F10
:108480007F4FCE0189960E945B968C01CE010196AA
:108490000E949E9764ED7BE0CE0183960E940A982D
:1084A00064ED7BE0CE014D960E940A9810161106ED
:1084B0000CF099C1A8014F5F5F4F8DA59EA548178D
:1084C000590790F4BE01675D7F4FCE0101960E946F
:1084D000CA58BE016F5F7F4FCE0183960E94659799
:1084E000CE0101960E949E97980150E040E0BE01A7
:1084F000675D7F4FCE0101960E941B98BE016F5FA2
:108500007F4FCE014D960E946597CE0101960E9445
:108510009E9789A19AA1892B09F418C2CE014D9684
:108520000E94A7956B0121E0C21AD108860138E1AB
:10853000C316D10414F007E110E017FF02C00FEFDB
:108540001FEFB801CE010B960E94619561E078E0C3
:10855000CE0141960E940A98BE01655F7F4FCE0111
:1085600041960E94B896BC01CE0101960E940198E6
:10857000CE0101960E94825BCE0101960E949E97D9
:10858000CE0141960E949E97CE010B960E949E9727
:10859000BE016D5D7F4FCE0189960E944E976FEFB1
:1085A00077E0CE0101960E940A98BE016F5F7F4F6F
:1085B000CE0189960E945B967C01CE0101960E94B5
:1085C0009E9764ED7BE0CE0183960E942A9564ED30
:1085D0007BE0CE014D960E942A951E141F040CF0DC
:1085E00010C1A7014F5F5F4F8DA59EA54817590782
:1085F00090F4BE01675D7F4FCE0101960E94CA587C
:10860000BE016F5F7F4FCE0183960E946597CE01BA
:1086100001960E949E97970150E040E0BE01675D81
:108620007F4FCE0101960E941B98BE016F5F7F4F66
:10863000CE014D960E946597CE0101960E949E97AD
:10864000A8014F5F5F4F8AE0849F9001859F300DA6
:108650001124A90141555E4E5A01FE0131963F0198
:10866000F12CE12C809F9001819F300D1124A901F4
:1086700043545E4E2A013AE2332E89A19AA1892BF6
:1086800009F4E8C0CE014D96E114F10409F0CEC022
:10869000D7FCCCC00E94B295A114B10439F044E0DB
:1086A00050E0B501CE014D960E94758DB501CE0109
:1086B00041960E940A9866E078E0CE0147960E94B3
:1086C0000A98BE016F5E7F4FCE0147960E94B89612
:1086D000BC01CE010B960E940198CE010B960E9420
:1086E000825BCE010B960E949E97CE0147960E9418
:1086F0009E97CE0141960E949E9789A19AA10297CA
:1087000008F48DC061E070E0CE014D960E9476962F
:10871000082E000C990B803391050CF44C96E32D38
:10872000E81B8E2FF2018083FFEFEF1AFF0ABE01D4
:108730006D5D7F4FCE0189960E944E976FEF77E077
:10874000CE010B960E940A98BE01655F7F4FCE0155
:1087500089960E945B964C01CE010B960E949E97D3
:1087600064ED7BE0CE0183960E942A9564ED7BE068
:10877000CE014D960E942A95181419040CF05CC085
:10878000A4014F5F5F4F8DA59EA54817590790F430
:10879000BE01675D7F4FCE010B960E94CA58BE0195
:1087A000655F7F4FCE0183960E946597CE010B9641
:1087B0000E949E97940150E040E0BE01675D7F4FAC
:1087C000CE010B960E941B98BE01655F7F4FCE01C4
:1087D0004D960E946597CE010B960E949E9752E09F
:1087E000650E711C4ACF64ED7BE0CE0183960E943A
:1087F0002A95BE01675D7F4FCE014D960E944E9730
:1088000088CE64ED7BE0CE0183960E942A95BE015E
:10881000675D7F4FCE014D960E944E9711CFCE01DE
:108820004D960E94A795F20160837ECF0E94A79586
:10883000F3017183608378CF64ED7BE0CE01839692
:108840000E942A95BE01675D7F4FCE014D960E9422
:108850004E97C5CFD7FE8BC06FEF77E0CE010B965A
:108860000E940A98BE01655F7F4FCE0183960E94E9
:108870005B968C01CE010B960E949E9717FF66C0F7
:1088800009811A810931110514F008E110E0101670
:10889000110614F001E010E00093B111B801CE010F
:1088A00041960E94619564E178E0CE0147960E946E
:1088B0000A98BE016F5E7F4FCE0147960E94B89620
:1088C000BC01CE010B960E940198CE010B960E942E
:1088D000825BCE010B960E949E97CE0147960E9426
:1088E0009E97CE0141960E949E97E114F10451F1AA
:1088F0008B819C8197FF02C090E080E09093B31140
:108900008093B21121E0E216F104E1F08D819E81A5
:10891000081719070CF4C8011816190614F081E09D
:1089200090E081508093B61132E0E316F10451F0EB
:108930008F8198851816190614F081E090E0815017
:108940008093B7118CE291E00E94218DCE014D966B
:108950000E949E97CE0183960E949E97CE01899693
:108960000E949E97CE018F960E949E977FCB80910A
:10897000B011082E000C990B081719070CF083C0D2
:10898000B701CE0141960E9461956EE178E0CE017B
:1089900047960E940A98BE016F5E7F4FCE014796B0
:1089A0000E94B896BC01CE010B960E940198CE01A0
:1089B0000B960E94825BCE010B960E949E97CE0181
:1089C00047960E949E97CE0141960E949E978AE00C
:1089D000809FF001819FF00D1124E155FE4E81E052
:1089E000878783E090E0918B808B938B828BE1145F
:1089F000F10409F4ABCF8B819C818038910514F090
:108A00008FE790E080384FEF940714F480E89FEFF1
:108A1000878751E0E516F10409F498CF8AE0809F3A
:108A2000F001819FF00D1124E155FE4E8D819E8154
:108A300097FF02C090E080E0918B808B82E0E81687
:108A4000F10409F483CF8AE0809FF001819FF00D4B
:108A50001124E155FE4E8F81988597FF02C090E06A
:108A600080E0938B828B8091B111082E000C990BC2
:108A7000081719071CF00F5F0093B1118CE291E009
:108A80000E94988D63CFBE016D5D7F4FCE014796EA
:108A90000E9401986091B011062E000C770BCE0158
:108AA0000B960E94619566E278E0CE0141960E94A5
:108AB0000A98BE01695E7F4FCE0141960E94B8962A
:108AC00067E378E00E94A296BE01655F7F4F0E9437
:108AD000B896BC01CE0147960E944E97CE014196B2
:108AE0000E949E97CE010B960E949E97BE01695EE2
:108AF0007F4FCE010B960E940198CE010B960E94EB
:108B00008457CE010B960E949E97CE0147960E94F5
:108B10009E971CCF6BE378E0CE0101960E940A98E5
:108B2000BE016F5F7F4F8DEC92E10E948796182FF8
:108B3000CE0101960E949E971123C9F166E679E065
:108B4000CE0101960E940A98BE016F5F7F4F83EDB0
:108B500092E10E940F96AC014F5F5F4F63ED72E1AF
:108B6000CE010B960E94CA58BE01655F7F4F8FEA07
:108B700092E10E946597CE010B960E949E97CE01CE
:108B800001960E949E978FEA92E10E94A795611537
:108B9000710531F481E0809387040E94E41564CA72
:108BA0006130710509F060CA10928704F6CF60E465
:108BB00078E0CE0101960E940A98BE016F5F7F4F58
:108BC0008DEC92E10E948796182FCE0101960E94AB
:108BD0009E97112309F43AC143E050E063ED72E13E
:108BE000CE0101960E94CA58BE016F5F7F4F8FEA87
:108BF00092E10E946597CE0101960E949E976FEACE
:108C000072E1CE0101960E940198CE0101960E9468
:108C1000825BCE0101960E949E976FEA72E1CE01BF
:108C200001960E940198CE0101960E940997BC010D
:108C300080EB93E10E944E97CE0101960E949E9791
:108C40006FEA72E1CE0101960E940198CE01019671
:108C50000E940997BC018AEA93E10E944E97CE01D7
:108C600001960E949E974091B4135091B5134115FF
:108C7000510549F08AE391E1009729F0BC0180EBAE
:108C800093E10E94758D4091AE135091AF13411541
:108C9000510549F088E991E1009729F0BC018AEA81
:108CA00093E10E94758D90E080E00E944B8D66EA12
:108CB00077E0CE0101960E940A986FEA72E1CE0138
:108CC00001960E94B896BC01CE0141960E9401987F
:108CD000CE0101960E949E978091941190919511DA
:108CE000892B39F4BE016F5E7F4F8CEC9DE00E94B2
:108CF000559A68EB7BE080E090E00E94F19F8091C4
:108D0000941190919511029709F087C06FEA72E172
:108D1000CE0147960E94019864E478E0CE01019666
:108D20000E940A98CE0101960E94EEA9CE010196FA
:108D30000E949E9764EF71E080E090E00E94F19FB6
:108D400067E478E0CE0101960E940A98CE01019670
:108D50000E94EEA9CE0101960E949E976CED75E0EF
:108D600080E090E00E94F19F60E578E0CE010196FE
:108D70000E940A98CE0101960E94EEA9CE010196AA
:108D80000E949E9764EF71E080E090E00E94F19F66
:108D90006EE578E0CE0101960E940A98CE01019618
:108DA0000E94EEA9CE0101960E949E9764EF71E0A9
:108DB00080E090E00E94F19F66EA77E0CE010196A4
:108DC0000E940A98BE01695E7F4FCE0101960E9403
:108DD000B896BC01CE010B960E940198CE01019677
:108DE0000E949E97CE010B960E94B295BE01655FD0
:108DF0007F4FCE0101960E940198CE0101960E94FC
:108E0000EEA9CE0101960E949E97CE010B960E947C
:108E10009E97CE0147960E949E9768EB7BE080E08C
:108E200090E00E94F19F6AE371E1CE0101960E94F9
:108E30000A98CE0101960E94825BCE0101960E94A3
:108E40009E971092EC04CE0141968ECD6CE678E0B0
:108E5000CE0101960E940A98BE016F5F7F4F8DEC94
:108E600092E10E948796182FCE0101960E949E974C
:108E7000112309F487C044E050E063ED72E1CE01B4
:108E800001960E94CA58BE016F5F7F4F8FEA92E140
:108E90000E946597CE0101960E949E976EEA77E048
:108EA000CE0101960E940A986FEA72E1CE01019606
:108EB0000E94B896BC01CE010B960E940198CE018B
:108EC00001960E949E978091941190919511892B03
:108ED00069F4BE01655F7F4F8CEC9DE00E94559A5E
:108EE00068E873E180E090E00E94F19F8091941126
:108EF00090919511029759F561E778E0CE010196BE
:108F00000E940A988091B3129091B412892B21F596
:108F10006AE778E0CE0101960E942A95BE01655F5E
:108F20007F4FCE0141960E940198CE0141960E944A
:108F3000EEA9CE0141960E949E9760ED77E080E019
:108F400090E00E94F19FCE0101960E949E971092A0
:108F5000EC04CE010B9608CDBE016F5F7F4FCE01B2
:108F600041960E940198CE0141960E94EEA9CE0141
:108F700041960E949E9760ED77E080E090E00E942D
:108F8000F19FCCCF63E878E0CE0101960E940A9869
:108F9000BE016F5F7F4F8DEC92E10E948796182F84
:108FA000CE0101960E949E97112309F462C063EDE1
:108FB00072E18FEA92E10E944E9781E08093EC0487
:108FC00063ED72E1CE0101960E940198CE010196F7
:108FD0000E94825BCE0101960E949E97809194111F
:108FE00090919511029709F16FEA72E18CEC9DE086
:108FF0000E94559A68EB7BE080E090E00E94F19F30
:10900000CE0101960E94FE6DBE016F5F7F4F83ED22
:1090100092E10E946597CE0101960E949E9760EDB5
:1090200077E080E090E00E94F19F80919411909110
:109030009511029771F46FEA72E1CE0101960E94D8
:109040000198CE0101960E94EEA9CE0101960E94E0
:109050009E978091D7129091D812892B09F404C859
:1090600064ED75E0CE0101960E940A9863ED72E10D
:10907000A4C867E878E0CE0101960E940A98BE0174
:109080006F5F7F4F8DEC92E10E948796182FCE0183
:1090900001960E949E97112309F462C08091941159
:1090A00090919511019711F00C943440CE010196E6
:1090B0000E94DD318D819E81009709F44BC0E981CA
:1090C000FA812081222309F445C0079708F442C0A1
:1090D00064E179E0CE010B960E94F89748EC50E0ED
:1090E0006FEF7FEFCE010B960E94D658CE010B9604
:1090F0000E949E97BE016F5F7F4FCE010B960E942C
:10910000019840ED57E06FEF7FEFCE010B960E9484
:10911000FA57CE010B960E949E976DE878E0CE013B
:109120000B960E940A9863ED72E1CE010B960E94A5
:10913000B896BC01CE0141960E940198CE0141969D
:109140000E948457CE0141960E949E97CE010B96B5
:109150000E949E97CE0101960E949E970C943440E7
:109160006BE978E0CE0101960E940A98BE016F5F1C
:109170007F4F8DEC92E10E948796182FCE010196C9
:109180000E949E97112361F125E030E044E050E019
:1091900063ED72E1CE0101960E941B98BE016F5FE4
:1091A0007F4F8FEA92E10E946597CE0101960E945F
:1091B0009E9763ED72E1CE0101960E940198CE0167
:1091C00001960E94825BCE0101960E949E978FEAD3
:1091D00092E10E94A795CB010E947D270C94344018
:1091E00060EA78E0CE0101960E940A98BE016F5FA6
:1091F0007F4F8DEC92E10E948796182FCE01019649
:109200000E949E97112361F127E030E046E050E094
:1092100063ED72E1CE0101960E941B98BE016F5F63
:109220007F4F8FEA92E10E946597CE0101960E94DE
:109230009E978FEA92E10E94A795672B69F410929E
:10924000040D63ED72E1CE0101960E940198CE01FA
:1092500001960E94825B7ECF81E08093040DF1CF66
:1092600067EA78E0CE0101960E940A98BE016F5F1E
:109270007F4F8DEC92E10E948796182FCE010196C8
:109280000E949E97112309F4BBC08091390C9091E4
:109290003A0C1816190614F00C94364088E592E042
:1092A000909386048093850483EA9FE00E94CD8892
:1092B000198A1A8A1B8A1C8ACC24C394D12C28EDC3
:1092C000422E2FE0522E5E0191E1A90EB11C3E010B
:1092D000E5E16E0E711C8091390C90913A0C8C1561
:1092E0009D0514F40C943640809185049091860479
:1092F000893D9F4024F0509286044092850400915D
:10930000850410918604750148018A189B08C401E0
:109310008E0D9F1D0E94CBB5F70181937F01E6154D
:10932000F705A9F7C80104969093860480938504F5
:1093300085E1E82E8CE0F82E01511C40C8018E0D0D
:109340009F1D0E94CBB5F70181937F01F9E3EF16D2
:10935000FCE0FF0699F749895A896B897C8923E0EB
:10936000CE0101960E94A697BE016F5F7F4FCE018E
:109370000B960E94019860E979E0CE010B960E945D
:10938000A296BC0185EB92E10E944E97CE010B960E
:109390000E949E97CE0101960E949E9765E17CE017
:1093A000CE0101960E940A98BE016F5F7F4F85EB48
:1093B00092E10E942297CE0101960E949E9765EB52
:1093C00072E1CE0101960E940198CE0101960E94A1
:1093D0008457CE0101960E949E97809185049091BA
:1093E00086048496909386048093850464E170E0FB
:1093F00080E090E00E94F19F2FEFC21AD20A6BCF5B
:109400006BEA78E0CE0101960E940A98BE016F5F78
:109410007F4F8DEC92E10E948796182FCE01019626
:109420000E949E971123D1F126E030E045E050E004
:1094300063ED72E1CE0101960E941B98BE016F5F41
:109440007F4F8FEA92E10E946597CE0101960E94BC
:109450009E978FEA92E10E94A795672B21F41092C4
:10946000140C0C94364081E08093140C10923A0C4A
:109470001092390C1092100C1092110C1092120CC8
:109480001092130C0E948DA660930C0C70930D0C1F
:1094900080930E0C90930F0C0C94364061EB78E0A7
:1094A000CE0101960E940A98BE016F5F7F4F8DEC3E
:1094B00092E10E948796182FCE0101960E949E97F6
:1094C000112309F478C08091D7129091D812079790
:1094D00010F40C94364046E050E063ED72E1CE01AA
:1094E00001960E94CA58BE016F5F7F4F8FEA92E1DA
:1094F0000E946597CE0101960E949E978FEA92E1A5
:109500000E949C956093E8047093E9048093EA04B8
:109510009093EB0464E079E085EB92E10E94299757
:109520004091E8045091E9046091EA047091EB04E1
:1095300021E0CE0101960E94A697BE016F5F7F4F8A
:10954000CE010B960E94019862ED76E0CE010B965B
:109550000E94A296BC0185EB92E10E942297CE0167
:109560000B960E949E97CE0101960E949E9765EBF6
:1095700072E1CE0101960E940198CE0101960E94EF
:109580008457CE0101960E949E970E948DA628EED8
:1095900033E040E050E00E9413B6CA01B9010E94D6
:1095A000A9B46093FF0C7093000D8093010D90930C
:1095B000020D0C94364068EB78E0CE0101960E94D3
:1095C0000A98BE016F5F7F4F8DEC92E10E948796F3
:1095D000182FCE0101960E949E97112309F456C0C0
:1095E0008091D7129091D812079710F40C943640BE
:1095F00046E050E063ED72E1CE0101960E94CA5848
:10960000BE016F5F7F4F8FEA92E10E946597CE01A6
:1096100001960E949E978FEA92E10E949C9560932A
:10962000810470938204809383049093840464EF94
:1096300078E085EB92E10E94299740918104509156
:109640008204609183047091840421E0CE0101962C
:109650000E94A697BE016F5F7F4FCE010B960E94BE
:10966000019862ED76E0CE010B960E94A296BC01B5
:1096700085EB92E10E942297CE010B960E949E9765
:10968000CE0101960E949E970C949B410E94CC1D96
:10969000182F81110C943640812FE4960FB6F89460
:1096A000DEBF0FBECDBFDF91CF911F910F91FF9015
:1096B000EF90DF90CF90BF90AF909F908F907F9072
:1096C0006F905F904F903F90089511E0E5CFAF927B
:1096D000BF92CF92DF92EF92FF920F931F93CF939F
:1096E000DF93CDB7DEB7A4970FB6F894DEBF0FBEF9
:1096F000CDBF8091EC0B882399F01092EC0BA496CF
:109700000FB6F894DEBF0FBECDBFDF91CF911F9192
:109710000F91FF90EF90DF90CF90BF90AF900895A2
:109720008091D7129091D812049708F040C06BE84E
:1097300078E0CE0101960E940A98BE016F5F7F4FCC
:109740008DEC92E10E948796182FCE0101960E941F
:109750009E97112361F161E070E083ED92E10E9438
:10976000769680330CF4845E6AE270E0681B7109BF
:1097700087FD7395CE0101960E946195BE016F5FD2
:109780007F4F83ED92E10E946597CE0101960E9482
:109790009E9763ED72E181EC92E10E944E9783ED1A
:1097A00092E10E94A795CB010E945C74A8CF6CEE59
:1097B00077E0CE0101960E940A98BE016F5F7F4F4D
:1097C0008DEC92E10E948796182FCE0101960E949F
:1097D0009E97112309F4AFC36FEB78E0CE01019699
:1097E0000E940A98CE0101960E948457CE010196EC
:1097F0000E949E976BEC78E0CE0107960E940A9833
:109800006AEA73E1CE0107960E94B896BC01CE01C8
:1098100001960E940198CE0101960E948457CE01C4
:1098200001960E949E97CE0107960E949E97609196
:10983000C7047091C8048091C9049091CA040E9421
:10984000ABB420E030E048EC52E40E9423B7AB0117
:10985000BC0122E0CE0107960E94A69761EE78E057
:10986000CE010D960E940A98BE01695F7F4FCE011E
:109870000D960E94B89667E076E00E94A296BC0121
:10988000CE0101960E940198CE0101960E94845754
:10989000CE0101960E949E97CE010D960E949E9742
:1098A000CE0107960E949E974091C3045091C40434
:1098B0006091C5047091C60424E0CE0107960E9411
:1098C000A69766EF78E0CE010D960E940A98BE0139
:1098D000695F7F4FCE010D960E94B896BC01CE0104
:1098E00001960E940198CE0101960E948457CE01F4
:1098F00001960E949E97CE010D960E949E97CE01E2
:1099000007960E949E974091B7045091B8046091C9
:10991000B9047091BA0422E0CE0107960E94A6977E
:109920004091AF045091B0046091B1047091B204C1
:1099300023E0CE010D960E94A6974091BB04509162
:10994000BC046091BD047091BE0422E0CE01439638
:109950000E94A6974091B3045091B4046091B5045D
:109960007091B60423E0CE0149960E94A69763E168
:1099700079E0CE014F960E940A98BE01675E7F4F44
:10998000CE014F960E94B89668E279E00E94A296B6
:10999000BE016D5E7F4F0E94B8966BE279E00E9437
:1099A000A296BE01635F7F4F0E94B89668E279E09D
:1099B0000E94A296BE01695F7F4F0E94B89661E344
:1099C00079E00E94A296BC01CE0101960E94019806
:1099D000CE0101960E948457CE0101960E949E9767
:1099E000CE014F960E949E97CE0149960E949E9767
:1099F000CE0143960E949E97CE010D960E949E979F
:109A0000CE0107960E949E976AE477E0CE014996C0
:109A10000E94F897F0904D110F2D0F2C000C110B98
:109A20000115110509F07EC120914E1130914F11A1
:109A3000409150115091511160E070E080EA90E443
:109A40000E9423B7AB01BC0122E0CE0101960E9427
:109A5000A6976CE276E0CE0107960E940A98BE01B6
:109A60006F5F7F4FCE0107960E94B89660E17BE062
:109A70000E94A296BC01CE0149960E942297CE0177
:109A800007960E949E97CE0101960E949E97C8015C
:109A90000297029738F58F2D9AE08902B0011124C0
:109AA000CE0101960E94619566E379E0CE010796AA
:109AB0000E940A98BE016F5F7F4FCE0107960E94F9
:109AC000B89669E07BE00E94A296BC01CE0149965F
:109AD0000E942297CE0107960E949E97CE01019682
:109AE0000E949E976AE277E00430110519F034F085
:109AF00062E277E0CE0149960E94CB96BE01675E96
:109B00007F4FCE0101960E940198CE0101960E94DE
:109B10008457CE0101960E949E9762E479E0CE01BF
:109B200049960E942A9580914A1160914B1170913B
:109B30004C1183300CF08DC3CE0101960E946195CB
:109B40006DE379E0CE0107960E940A98BE016F5F2F
:109B50007F4FCE0107960E94B89666E37AE00E9496
:109B6000A296BC01CE0149960E942297CE0107968B
:109B70000E949E97CE0101960E949E97BE01675E4D
:109B80007F4FCE0101960E940198CE0101960E945E
:109B90008457CE0101960E949E9740915211509198
:109BA0005311609154117091551122E0CE01079626
:109BB0000E94A69762E579E0CE010D960E940A9870
:109BC000BE01695F7F4FCE010D960E94B89668E690
:109BD00079E00E94A296BC01CE0101960E940198F4
:109BE000CE0101960E948457CE0101960E949E9755
:109BF000CE010D960E949E97CE0107960E949E97D9
:109C0000409168115091691160916A1170916B11C6
:109C100022E0CE0107960E94A6976FE679E0CE017A
:109C20000D960E940A98BE01695F7F4FCE010D9686
:109C30000E94B89669E176E00E94A296BC01CE012E
:109C400001960E940198CE0101960E948457CE0190
:109C500001960E949E97CE010D960E949E97CE017E
:109C600007960E949E9785E9E82E84E0F82E01E091
:109C700010E099E1C92EE2E0EE0EF11C809195040E
:109C800090919604801791070CF457C0F701A080BB
:109C9000B180B501CE0107960E946195B801CE0151
:109CA0000D960E94619562E879E0CE0143960E948C
:109CB0000A98BE01635F7F4FCE0143960E94B8961B
:109CC0006AE879E00E94A296BE01695F7F4F0E9418
:109CD000B8966DE879E00E94A296CA9CB001CB9C30
:109CE000700D1124685F7D4F0E94A296BC01CE01C9
:109CF00001960E940198CE0101960E948457CE01E0
:109D000001960E949E97CE0143960E949E97CE0197
:109D10000D960E949E97CE0107960E949E970F5F18
:109D20001F4FA9CF0130110509F0B1CE6CE377E0E8
:109D3000CE0149960E94CB96AACE80919411909123
:109D40009511892B71F463E979E0CE0101960E94A7
:109D50000A98CE0101960E948457CE0101960E9476
:109D60009E978091941190919511019771F462EAF8
:109D700079E0CE0101960E940A98CE0101960E94D8
:109D80008457CE0101960E949E97809194119091E4
:109D90009511029771F46CEA79E0CE0101960E9468
:109DA0000A98CE0101960E948457CE0101960E9426
:109DB0009E976091D4047091D504CE0107960E94BD
:109DC00061956EEB79E0CE010D960E940A98BE0176
:109DD000695F7F4FCE010D960E94B896BC01CE01FF
:109DE00001960E940198CE0101960E948457CE01EF
:109DF00001960E949E97CE010D960E949E97CE01DD
:109E000007960E949E974091E8045091E904609162
:109E1000EA047091EB0422E0CE0107960E94A69717
:109E20006BED79E0CE010D960E940A98BE01695F44
:109E30007F4FCE010D960E94B89662ED76E00E94AB
:109E4000A296BC01CE0101960E940198CE01019616
:109E50000E948457CE0101960E949E97CE010D96D6
:109E60000E949E97CE0107960E949E974091810482
:109E700050918204609183047091840422E0CE01A9
:109E800007960E94A6976BEE79E0CE010D960E9490
:109E90000A98BE01695F7F4FCE010D960E94B89669
:109EA00062ED76E00E94A296BC01CE0101960E946E
:109EB0000198CE0101960E948457CE0101960E941E
:109EC0009E97CE010D960E949E97CE0107960E9406
:109ED0009E976EE177E0CE0101960E94F897CE0141
:109EE00001960E94A157CE0101960E949E97609113
:109EF000060C7091070CCE0101960E946195CE016F
:109F000001960E94A157CE0101960E949E976FEF85
:109F100076E0CE0101960E94F897CE0101960E944C
:109F20008457CE0101960E949E971092EC04CE01B8
:109F300049960E949E978091D7129091D8128330B3
:109F4000910508F083C18130910509F061C070E08E
:109F500060E083ED92E10E947696D82E8D2DDD0C87
:109F6000990B0E9427BC892BB1F00E94D4150E9446
:109F7000B8576CE57AE0CE0101960E940A984AE053
:109F800050E070E060E0CE0101960E94D658CE010C
:109F900001960E949E9763ED72E1CE0107960E94A2
:109FA000019870E060E0CE0107960E9476968234B8
:109FB00009F405C10CF097C0803309F429C10CF0F5
:109FC00081C0833209F412C18A3209F418C1BE017A
:109FD000695F7F4F81EC92E10E944E9770E060E0F4
:109FE00081EC92E10E947696082E000C990BC097A6
:109FF0000A9738F481EC92E10E94A795CB010E9468
:10A000005C7464E670E080E090E00E94F19FB1C073
:10A01000029709F0A3CF6BE878E0CE0101960E9489
:10A020000A98BE016F5F7F4F8DEC92E10E94879688
:10A03000182FCE0101960E949E97112309F48ECF0E
:10A0400061E070E083ED92E10E947696682FCE0188
:10A0500001960E94D697BE016F5F7F4F81EC92E11F
:10A060000E946597CE0101960E949E9770E060E085
:10A0700083ED92E10E947696D82E8091040D88237C
:10A0800009F46CCF6BEF79E0CE0101960E940A983B
:10A0900063ED72E1CE0101960E94B8966CE57AE01C
:10A0A0000E94A296BC0183EA9FE00E94559ACE01CD
:10A0B00001960E949E9761EC72E183EA9FE00E9404
:10A0C000639A4CCF813309F4B2C0813409F07FCF59
:10A0D00068E07AE083ED92E10E942A958091020C7B
:10A0E0009091030C44C0813699F30CF061C0833425
:10A0F00009F470C0843409F06ACF8091C512909140
:10A10000C612892BB1F161E070E0CE0107960E9482
:10A110007696182F8091040D882361F061E07AE033
:10A1200083EA9FE00E94539A61EC72E183EA9FE028
:10A130000E94639A10330CF4145E6AE270E0611BB3
:10A14000710917FD7395CE0101960E946195BE01BC
:10A150006F5F7F4F81EC92E10E946597CE0101967F
:10A160000E949E9781EC92E10E94A795CB010E94EC
:10A170005C74CE0107960E949E970E948DA6609304
:10A18000FB0C7093FC0C8093FD0C9093FE0C0E94D2
:10A190008DA66093FB0C7093FC0C8093FD0C909348
:10A1A000FE0C64ED7BE083ED92E10E942A95A7CA44
:10A1B000833681F024F0843609F49FCF08CF6BE01A
:10A1C0007AE083ED92E10E942A951092030D8CEFC4
:10A1D0009FEFCDCF6EE07AE083ED92E10E942A9569
:10A1E00081E08093030D8DEF9FEFC1CF61E17AE0B5
:10A1F00083ED92E10E942A958EEF9FEFB8CF64E144
:10A200007AE083ED92E10E942A958FEF9FEFAFCF26
:10A2100066E177E081EC92E10E942A9566E177E0C1
:10A2200083ED92E10E942A9590E080E0A0CF65E165
:10A230007AE081EC92E10E942A9565E17AE083ED73
:10A2400092E10E942A9581E090E091CF0E94873FA1
:10A250009ECFCE0101960E94619567E17AE0CE0122
:10A2600007960E940A98BE016F5F7F4FCE01079646
:10A270000E94B89676CCCF92DF92EF92FF920F9326
:10A280001F93CF93DF93CDB7DEB7E0970FB6F89467
:10A29000DEBF0FBECDBF8E01015E1F4F8130910525
:10A2A00009F0B7C060E27AE0CE0101960E940A98F8
:10A2B00063E27AE0CE0107960E940A9866E27AE0AD
:10A2C000CE010D960E940A9861EF76E0C8010E94C7
:10A2D000F89744E650E06FEF7FEFC8010E94805985
:10A2E000C8010E949E9766EE76E083ED92E10E949F
:10A2F00029976091D4047091D504CE0185960E946F
:10A30000619563ED72E1C8010E940198BE016B5D29
:10A310007F4FC8010E94B896BC01CE018B960E9467
:10A32000019840ED57E06FEF7FEFCE018B960E94D2
:10A33000FA57CE018B960E949E97C8010E949E9765
:10A34000CE0185960E949E9767ED76E0C8010E9437
:10A35000F89744E650E06FEF7FEFC8010E94805904
:10A36000C8010E949E9767ED79E0C8010E940A9893
:10A3700023E030E0A801BE016F5F7F4FCE018596DC
:10A380000E9491A4BE016B5D7F4F83ED92E10E941C
:10A390006597CE0185960E949E97C8010E949E9760
:10A3A0008091D7129091D812892B09F4E3C270E002
:10A3B00060E083ED92E10E947696082E000C990BE6
:10A3C000C0970A9708F0D6C283ED92E10E94A79544
:10A3D0006B0169E27AE0C8010E940A9886E08C9DD0
:10A3E000B0018D9D700D112481E090E08C0F9D1FB8
:10A3F000680F791FC8010E94B896BC0183ED92E1F5
:10A400000E944E97C8010E949E970E94873F182F76
:10A41000E2C08A3F2FEF920709F023C16EE27AE093
:10A42000CE0101960E940A9868E37AE0CE01079671
:10A430000E940A9860E47AE0CE010D960E940A9884
:10A4400068E47AE0CE0143960E940A9868EC76E0D0
:10A45000C8010E94F89744E650E06FEF7FEFC80113
:10A460000E948059C8010E949E9762EC76E083EDBD
:10A4700092E10E94299780914A11EE24E394F12CF5
:10A48000EC0EFD1E96E08902E00CF11C112463ED38
:10A4900072E1C8010E940198B701C8010E94B896F4
:10A4A000BC01CE0185960E94019840ED57E06FEF08
:10A4B0007FEFCE0185960E94FA57CE0185960E94C5
:10A4C0009E97C8010E949E9762EB76E0C8010E94A9
:10A4D000F89744E650E06FEF7FEFC8010E94805983
:10A4E000C8010E949E976EE47AE0C8010E940A9813
:10A4F00024E030E0A801BE016F5F7F4FCE0185965A
:10A500000E9491A4BE016B5D7F4F83ED92E10E949A
:10A510006597CE0185960E949E97C8010E949E97DE
:10A520008091D7129091D812892B09F498C070E0CD
:10A5300060E083ED92E10E947696082E000C990B64
:10A54000C0970A9708F08BC083ED92E10E94A7950F
:10A5500062307105810591050CF46EC066EA76E003
:10A56000C8010E94F89744E650E06FEF7FEFC80102
:10A570000E94FA57C8010E949E9744EF51E063E0A1
:10A5800070E0CE0185960E94BEA364E57AE0C80122
:10A590000E940A9863ED72E1C8010E94B8966BE5CB
:10A5A0007AE00E94A296BE016B5D7F4F0E94B89632
:10A5B000BC0183ED92E10E944E97C8010E949E97D4
:10A5C000CE0185960E949E970E94873F182FCE014C
:10A5D00043960E949E97CE010D960E949E97CE01B3
:10A5E00007960E949E97CE0101960E949E9760E278
:10A5F00076E0111102C061E176E0CE0101960E9481
:10A60000F89748EC50E06FEF7FEFCE0101960E9483
:10A61000FA57CE0101960E949E97E0960FB6F894E5
:10A62000DEBF0FBECDBFDF91CF911F910F91FF9085
:10A63000EF90DF90CF90089564E57AE0C8010E9422
:10A640000A9863ED72E1C8010E94B896BC0183EDDF
:10A6500092E10E944E97C8010E949E97B5CF10E0EC
:10A66000B6CF0F9609F0ECC0CE0101967C0164EDE7
:10A670007BE0C7010E940A9896E0E90EF11C0E15D6
:10A680001F05A9F76EE57AE0CE0101960E942A9592
:10A6900080914D11811130C020914E1130914F1198
:10A6A000409150115091511160E070E080EA90E4C7
:10A6B0000E9423B7AB01BC0122E0CE0185960E9427
:10A6C000A69764E67AE0C8010E940A98BE016B5D15
:10A6D0007F4FC8010E94B89669E07BE00E94A29675
:10A6E000BC01CE0101960E942297C8010E949E974C
:10A6F000CE0185960E949E976BE976E0CE01079683
:10A700000E9429976FE876E0CE010D960E94299766
:10A7100063E876E0CE0143960E94299767E776E0EA
:10A72000CE0149960E94299761E776E0C8010E9410
:10A73000299762E676E0C8010E94F89744E650E067
:10A740006FEF7FEFC8010E948059C8010E949E9759
:10A7500064ED7BE083ED92E10E942A9580914D119A
:10A7600061E070E06C0F7D1F26E08202600D711DBC
:10A770001124C8010E94019840ED57E06FEF7FEF70
:10A78000C8010E94FA57C8010E949E9763E576E0CF
:10A79000C8010E94F89744E650E06FEF7FEFC801D0
:10A7A0000E948059C8010E949E9763ED72E1C80122
:10A7B0000E94019825E030E0A801BE016F5F7F4F45
:10A7C000CE0185960E9491A4BE016B5D7F4F83ED03
:10A7D00092E10E946597CE0185960E949E97C801DE
:10A7E0000E949E978091D7129091D812892B31F1B7
:10A7F00070E060E083ED92E10E947696082E000CF6
:10A80000990BC0970A97D0F465E276E0C8010E94E0
:10A810000A9863ED72E1C8010E94B896BC0183ED0D
:10A8200092E10E944E97C8010E949E970E94873F26
:10A83000182FCE0149960E949E97C9CE10E0F9CFFD
:10A8400067E67AE0CE0101960E940A9867EA79E00D
:10A85000CE0107960E940A986AE67AE0CE010D962C
:10A860000E940A9863E476E0C8010E94F89744E6E3
:10A8700050E06FEF7FEFC8010E948059C8010E942D
:10A880009E976DE376E083ED92E10E942997809197
:10A8900094119091951126E0289F7001299FF00C4A
:10A8A000112481E090E08C0F9D1FE80EF91E63EDEE
:10A8B00072E1C8010E940198B701C8010E94B896D0
:10A8C000BC01CE0185960E94019840ED57E06FEFE4
:10A8D0007FEFCE0185960E94FA57CE0185960E94A1
:10A8E0009E97C8010E949E976DE276E0C8010E9483
:10A8F000F89744E650E06FEF7FEFC8010E9480595F
:10A90000C8010E949E9763ED72E1C8010E94019800
:10A9100023E030E0A801BE016F5F7F4FCE01859636
:10A920000E9491A4BE016B5D7F4F83ED92E10E9476
:10A930006597CE0185960E949E97C8010E949E97BA
:10A940008091D7129091D812892BA1F070E060E02D
:10A9500083ED92E10E947696082E000C990BC09729
:10A960000A9740F483ED92E10E94A795CB010E94E3
:10A970007D274DCD10E02FCECF92DF92EF92FF9248
:10A98000CF93C0914D11C4304CF4C1300CF04BC08A
:10A99000CC2359F160E070E0CB013FC0C430D1F767
:10A9A0000E94351720E030E040EA50E40E940AB5EA
:10A9B00020E030EC4FE754E40E9423B720E030E081
:10A9C00040EA50E40E9423B720E030E040E851E440
:10A9D0000E940AB520E030E040E850E40E9445B60D
:10A9E00020E030E04AE754E416C00E94351720E02A
:10A9F00030E040EA50E40E940AB520E030EC4FE736
:10AA000054E40E9423B720914E1130914F11409190
:10AA10005011509151110E9423B7CF91FF90EF90A8
:10AA2000DF90CF9008950E9435172AE137E64CE970
:10AA300050E40E940AB520914E1130914F1140917F
:10AA40005011509151110E9444B66B017C01EC2FC2
:10AA5000EE0FFF0BE75AFA4F60817181072E000C51
:10AA6000880B990B0E94ABB49B01AC01C701B601E6
:10AA7000D2CF80918704882349F08091E70488230E
:10AA800029F060E086EB93E10C949D1208958F927B
:10AA90009F92AF92BF92CF92DF92EF92FF920F936D
:10AAA0001F93CF93DF938C01862F0B30110509F094
:10AAB00092C090911C13992309F0F89462E10E94CE
:10AAC00056A2EC0180911C13882309F078942097FA
:10AAD00001F180E090ECA9E7B4EC80930F13909320
:10AAE0001013A0931113B093121380931313909328
:10AAF0001413A0931513B0931613CE3F8FEFD807FE
:10AB000009F49DC0CF3FDC0709F4EBC1CCEFDFEFC8
:10AB100024C1C0911713E09018136E2D70E090E0DF
:10AB200080E00E94ABB42DEC3CEC4CEC5DE30E9469
:10AB30000AB54B015C016C2F70E090E080E00E9450
:10AB4000ABB49B01AC01C501B4010E9445B6609352
:10AB50000F13709310138093111390931213D091CD
:10AB60001913F0901A136D2F6F7770E090E080E06A
:10AB70000E94ABB44B015C016F2D70E090E080E06F
:10AB80000E94ABB42DEC3CEC4CEC5DE30E940AB5AA
:10AB90009B01AC01C501B4010E9445B6D7FD19C0A7
:10ABA00060931313709314138093151390931613DB
:10ABB000CE0DCD0FCF0D81E090E020911B13C2137D
:10ABC00002C090E080E0892B09F487C0CFEFDFEF6F
:10ABD00088C19058E5CFCFEFDFEF0631110509F0BE
:10ABE000BCC090911C13992309F0F89461E00E9475
:10ABF00056A2EC0180911C13882309F078942097C9
:10AC000009F180E090ECA9E7B4EC80930F139093E6
:10AC10001013A0931113B0931213809313139093F6
:10AC20001413A0931513B0931613CF3FDC0709F448
:10AC300058C1209709F451C0229609F067CFCEEF92
:10AC4000DFEF8BC0C0911813D091171360911713C9
:10AC50007091181376276727762790E080E00E948E
:10AC6000A9B42DEC3CEC4CEC5DE30E940AB560937A
:10AC70000F13709310138093111390931213E0909D
:10AC80001A13F09019136F2D6F77762F6E2D90E0B9
:10AC900080E00E94A9B42DEC3CEC4CEC5DE30E94FA
:10ACA0000AB5F7FC18C060931313709314138093C4
:10ACB0001513909316138C2F8D0F8E0D8F0DC1E0F1
:10ACC000D0E090911B13891302C0D0E0C0E0D19571
:10ACD000C195D109AACF9058E6CFC0900F13D0905C
:10ACE0001013E0901113F090121320E030E048ECC4
:10ACF00052E4C701B6010E942CB8D0E0C0E018169B
:10AD000014F4CBEFDFEF20E030E0A901C701B6017A
:10AD10000E94A4B487FF02C0CAEFDFEFC0901313F4
:10AD2000D0901413E0901513F090161320E030E04B
:10AD300048EC52ECC701B6010E94A4B487FF02C0E0
:10AD4000C9EFDFEF20E030E040EF52E4C701B60189
:10AD50000E942CB818160CF4BFC00C30110509F075
:10AD6000C0C08CE50E94D98A90E080E00E94D48A1D
:10AD70000E94B49D65E08CE50E94CC9D10922A0D46
:10AD80008093290DC82FD0E0209709F4A8C0C530C2
:10AD9000D1050CF4B6C00DEE1BE00E94E08DF80169
:10ADA00080870F5F1F4FC8018D5E9B408C179D07EA
:10ADB000A4F3C091F50B0091F60B602F70E090E0CA
:10ADC00080E00E94ABB42DEC3CEC4CEC5DE30E94C7
:10ADD0000AB56B017C016C2F70E090E080E00E946E
:10ADE000ABB49B01AC01C701B6010E9445B66B0133
:10ADF0007C01C092ED0BD092EE0BE092EF0BF09243
:10AE0000F00BD091F70B1091F80B6D2F6F7770E06E
:10AE100090E080E00E94ABB44B015C01612F70E0D8
:10AE200090E080E00E94ABB42DEC3CEC4CEC5DE398
:10AE30000E940AB59B01AC01C501B4010E9445B650
:10AE4000D7FD5DC06093F10B7093F20B8093F30B11
:10AE50009093F40BC00FCD0FC10F8091F90BC81365
:10AE6000B5CE20E030E048EC52E4C701B6010E94C4
:10AE70002CB8D0E0C0E0181614F4CBEFDFEF20E0E0
:10AE800030E040EA50E4C701B6010E94A4B487FF55
:10AE900002C0CAEFDFEFC090F10BD090F20BE09050
:10AEA000F30BF090F40B20E030E040EF51ECC701E1
:10AEB000B6010E94A4B487FF02C0C9EFDFEF20E013
:10AEC00030E040EF52E4C701B6010E942CB81816DA
:10AED00044F4C8EFDFEF05C0C8EFDFEF3ECFCEEFA1
:10AEE000DFEFCE01DF91CF911F910F91FF90EF9097
:10AEF000DF90CF90BF90AF909F908F900895905823
:10AF0000A1CFCDEFDFEFEDCFCF93DF93FC01248115
:10AF10003581232B99F0EC01BC018CEC9DE00E9463
:10AF2000639A6EE170E080E090E00E94F19FBE01C4
:10AF300083EA9FE0DF91CF910C94639ADF91CF91E8
:10AF40000895CF93DF93FC0124813581232B69F091
:10AF5000EC01BC0183EA9FE00E94559ABE018CEC93
:10AF60009DE0DF91CF910C94559ADF91CF91089598
:10AF7000809187048823F9F08091E7048823D9F031
:10AF800081E00E94E38A8BE39FE10197F1F760E0A3
:10AF900080E00E94F48A6CE17DE086EB93E10E9400
:10AFA000759A61E080E00E94F48A6CE07DE086EBB7
:10AFB00093E10C94759A0895CF93DF9320918704C1
:10AFC0002223A9F02091E704222389F0EC016FED00
:10AFD00086EB93E10E94DA988C819D81892B39F070
:10AFE000BE0186EB93E1DF91CF910C94559ADF91EE
:10AFF000CF910895EF92FF920F931F93CF93DF931A
:10B0000020918704222309F461C02091E7042223C0
:10B0100009F45CC08A01EB017C01209719F1C0950D
:10B02000D09561E08C2F0E94F48AB70186EB93E102
:10B030000E94559A6BEF7CE086EB93E10E94759A33
:10B04000F701848161E08C0F0E94F48AB801110F2E
:10B05000880B990BDF91CF911F910F91FF90EF908B
:10B060000C94F19F0E948DA6AB01BC018091B70C9E
:10B070009091B80CA091B90CB091BA0C8C599F4F1B
:10B08000AF4FBF4F84179507A607B707F8F461E0E5
:10B0900080E00E94F48AB70186EB93E10E94559A02
:10B0A0006AEE7CE086EB93E10E94759A61E0F7011D
:10B0B00084810E94F48A0E948DA66093B70C7093DD
:10B0C000B80C8093B90C9093BA0CC0CFDF91CF919C
:10B0D0001F910F91FF90EF900895FF920F931F9390
:10B0E000CF93DF93EC01F62E08811981C8010E94ED
:10B0F000CBB5F81621F06F2DC8010E94D3B5CE0153
:10B10000DF91CF911F910F91FF900895CF93DF931F
:10B11000EC019A01AB01E889F98982E0808321156D
:10B1200081EE38074105510581F160E079E08DE35A
:10B1300090E00E9413B621503109410951095695FA
:10B14000479537952795EC85FD851082EE85FF851F
:10B150002083188EEC89FD8986E08083EA89FB894B
:10B16000808180618083EA89FB8980818860808317
:10B17000EA89FB89808180688083EA89FB898081F4
:10B180008F7D8083DF91CF910895E889F9891082BE
:10B1900020E1D9CFCF93DF93EC01FB0124813581EE
:10B1A0000E941B98CE01DF91CF910895CF92DF923C
:10B1B000EF92FF920F931F93CF93DF93CDB7DEB73C
:10B1C00062970FB6F894DEBF0FBECDBF2091870403
:10B1D000222309F446C02091E704222309F441C048
:10B1E0008A016B017C010E948DA6AB01BC0180919C
:10B1F000B30C9091B40CA091B50CB091B60C8C59D5
:10B200009F4FAF4FBF4F84179507A607B70748F565
:10B2100060E0CD20C094A1F580E00E94F48AD12C9A
:10B22000B70186EB93E10E94559A69ED7CE086EBCD
:10B2300093E10E94759AF701848160E08D0D0E9470
:10B24000F48A0E948DA66093B30C7093B40C809323
:10B25000B50C9093B60CB801110F880B990B0E9496
:10B26000F19F62960FB6F894DEBF0FBECDBFDF919F
:10B27000CF911F910F91FF90EF90DF90CF900895A5
:10B2800080E00E94F48A0E948DA628EE33E040E020
:10B2900050E00E94E1B5CA01B90120E831E541E082
:10B2A00050E00E94E1B5AB01BC01CE0101960E94C5
:10B2B0003495BE016F5F7F4FCE0107960E940198C3
:10B2C00060E979E0CE0107960E94A296BC01CE010A
:10B2D0000D960E940198CE0107960E949E97CE017E
:10B2E00001960E949E97BE01635F7F4F86EB93E1BC
:10B2F0000E94559AD988CE010D960E949E9790CFB4
:10B30000BF92CF92DF92EF92FF920F931F93CF9352
:10B31000DF93CDB7DEB762970FB6F894DEBF0FBEEE
:10B32000CDBF6C018B017A0180918704882369F17C
:10B330008091E704882349F177FF37C00095109585
:10B3400060E0802F0E94F48AB60186EB93E10E94B0
:10B35000559A68EC7CE086EB93E10E94759AF601C1
:10B36000848160E0800F0E94F48A0E948DA6609321
:10B37000B30C7093B40C8093B50C9093B60CB701DA
:10B38000FF0C880B990B0E94F19F62960FB6F89400
:10B39000DEBF0FBECDBFDF91CF911F910F91FF9008
:10B3A000EF90DF90CF90BF90089560E080E00E9422
:10B3B000F48A0E948DA628EE33E040E050E00E941F
:10B3C000E1B5CA01B90120E831E541E050E00E9451
:10B3D000E1B5AB01BC01CE0101960E943495BE01DE
:10B3E0006F5F7F4FCE0107960E94019860E979E078
:10B3F000CE0107960E94A296BC01CE010D960E9436
:10B400000198CE0107960E949E97CE0101960E9458
:10B410009E97BE01635F7F4F86EB93E10E94559A32
:10B42000B98860E08B2D0E94F48A0115110531F472
:10B430000B2DCE010D960E949E9786CF60E0802F47
:10B440000E94F48AF6CFCF93DF93EC01483085E079
:10B4500058076105710509F448C008F099C04934DE
:10B4600081E058076105710509F4B2C008F040C0D9
:10B47000443481E058076105710509F476C000F590
:10B48000413481E058076105710509F456C048F45C
:10B49000403451406105710509F4E4C064ED7BE07E
:10B4A000E3C0423481E058076105710509F409C120
:10B4B000433451406105710589F76FE07AE0D4C0EB
:10B4C000463481E058076105710509F40CC108F4A0
:10B4D0009FC0473481E058076105710509F455C0E4
:10B4E0004834514061057105C9F662E77AE0BCC095
:10B4F000423085E058076105710509F4E2C000F5A6
:10B50000443781E058076105710509F4F2C040F441
:10B51000423751406105710509F669E07BE0A4C03E
:10B52000411585E058076105710509F49BC041305C
:10B5300055406105710509F0B1CF65E17AE094C02D
:10B54000453085E058076105710509F461C080F454
:10B55000433085E058076105710509F4AECF4430EA
:10B5600055406105710509F099CF6CE07AE07CC027
:10B57000463085E058076105710509F4B4C04730CD
:10B5800055406105710509F089CF60E77AE06CC02C
:10B590004D3B82E458078FEF6807710509F4AFC08F
:10B5A00008F048C04F3E80E158078FEF68077105EB
:10B5B00061F3F8F4423385E058076105710509F439
:10B5C000ACCF48F4493055406105710509F066CFAC
:10B5D00064E77AE049C0443385E0580761057105A6
:10B5E00009F487C04D3F52406F4F710509F495CF64
:10B5F00055CF4D3D82E258078FEF6807710509F47A
:10B6000078C048F4473E58416F4F710509F046CF66
:10B6100069E07AE029C04F3C80E358078FEF680764
:10B62000710509F4A2CF473C58436F4F710509F4E7
:10B630005CCF34CF473988E658078FEF680771052C
:10B6400009F47BCF48F54D3A82E558078FEF68073C
:10B65000710509F451C078F4453B5A446F4F7105A8
:10B6600009F01CCF66E177E0CE010E940A98CE0176
:10B67000DF91CF910895453A8AE558078FEF680723
:10B68000710509F4A5CF4D3952466F4F710509F088
:10B6900005CF61ED75E0E8CF473588EA58078FEFB1
:10B6A0006807710519F180F445388AE758078FEF6C
:10B6B00068077105C1F0473658496F4F710509F0A9
:10B6C000EDCE62E17AE0D0CF4F3480EB58078FEFB8
:10B6D0006807710509F4F1CE4D33524C6F4F710577
:10B6E00009F41BCFDBCE6EE67AE0BECF6BE878E0E4
:10B6F000BBCF6BE87BE0B8CF64ED75E0B5CF66E714
:10B700007AE0B2CF0F931F93CF93DF9300D000D096
:10B71000CDB7DEB72091040D2223A9F08C0164ED92
:10B7200075E0CE0101960E940A98B801CE010196FB
:10B730000E94B896BC0183EA9FE00E94639ACE0102
:10B7400001960E949E9726960FB6F894DEBF0FBE14
:10B75000CDBFDF91CF911F910F9108954F925F92CE
:10B760006F927F929F92AF92BF92CF92DF92EF92B1
:10B77000FF920F931F93CF93DF93CDB7DEB7A997B7
:10B780000FB6F894DEBF0FBECDBF982E882351F0C0
:10B790008091040D882331F064ED7BE083EA9FE023
:10B7A0000E94C8980E947C9460E08DE20E94B79D40
:10B7B00060E18DE20E94B79D68E08DE20E94B79D36
:10B7C00040901F135090201360902113709022130B
:10B7D000498E5A8E6B8E7C8EC0902313D09024138A
:10B7E000E0902513F0902613CD8EDE8EEF8EF8A21A
:10B7F0008091271390912813A0912913B0912A13B7
:10B800008EA39FA3A8A7B9A789A39AA3ABA3BCA300
:10B810009920C9F18091040D8823A9F166EF74E1A4
:10B82000CE0101960E94F897CE0101960E94825B9C
:10B83000CE0101960E949E978E01075E1F4F5E010A
:10B8400095E2A90EB11CD8016D917D918D919D91CC
:10B850008D0146E00E9415996CE57AE083EA9FE04D
:10B860000E94539AA016B10671F764ED7BE0CE01F9
:10B8700001960E940A98CE0101960E94825BCE0139
:10B8800001960E949E9723E938E144E85FE3C301F3
:10B89000B2010E940AB52B013C014D865E866F867F
:10B8A000788A22E430E645E85FE3C701B6010E94EA
:10B8B0000AB56B017C01C98ADA8AEB8AFC8A25E821
:10B8C0003BEE41E95FE36EA17FA188A599A50E94A7
:10B8D0000AB56D8B7E8B8F8B988F40921F13509281
:10B8E00020136092211370922213C0922313D092DE
:10B8F0002413E0922513F09226136093271370937C
:10B9000028138093291390932A13992009F4A0C037
:10B910008091040D882309F49BC069EE74E1CE0187
:10B9200001960E94F897CE0101960E94825BCE019B
:10B9300001960E949E978E01035F1F4F6E01B9E131
:10B94000CB0ED11C7801F801619171918191919197
:10B950008F0142E00E9415996CE57AE083EA9FE04E
:10B960000E94539AC016D10671F764ED7BE0CE01B8
:10B9700001960E940A98CE0101960E94825BCE0138
:10B9800001960E949E974BE253E166E070E082E3ED
:10B990000E94E49EA0902B13B0902C13C0902D1306
:10B9A000D0902E1300912F13109130136CED74E191
:10B9B00083EA9FE00E94759A4AE050E0B50183EA6D
:10B9C0009FE00E94069A6CE57AE083EA9FE00E947D
:10B9D000539A4AE050E0B60183EA9FE00E94069A3B
:10B9E0006CE57AE083EA9FE00E94539A4AE050E0D7
:10B9F000B80183EA9FE00E94069A64ED7BE083EA47
:10BA00009FE00E94C898CE0101960E94639F63ED5B
:10BA100074E183EA9FE00E94759A8E010F5F1F4FC9
:10BA2000D8016D917D918D919D918D014AE00E948B
:10BA300015996CE57AE083EA9FE00E94539A0E150F
:10BA40001F0571F764ED7BE083EA9FE00E94C898D0
:10BA500061E08DE10E94B79D9920B1F08091040DC5
:10BA6000882391F06FEB74E183EA9FE00E94759A5E
:10BA7000AE014B5D5F4F61E070E08DE10E94E49E9E
:10BA80008DA190E00E94409A62E08EE10E94B79DF5
:10BA900063E08FE10E94B79D64E080E20E94B79D61
:10BAA000992009F450C08091040D882309F44BC0FB
:10BAB00063EA74E183EA9FE00E94759AAE014B5DF0
:10BAC0005F4F61E070E08EE10E94E49ECDA0D12C3A
:10BAD000AE014B5D5F4F61E070E08FE10E94E49E3C
:10BAE000EDA0F12CAE014B5D5F4F61E070E080E2B4
:10BAF0000E94E49E0DA110E04AE050E0B60183EA06
:10BB00009FE00E94069A6CE57AE083EA9FE00E943B
:10BB1000539A4AE050E0B70183EA9FE00E94069AF8
:10BB20006CE57AE083EA9FE00E94539A4AE050E095
:10BB3000B80183EA9FE00E94069A64ED7BE083EA05
:10BB40009FE00E94C89865E081E20E94B79D99201D
:10BB5000B1F08091040D882391F060E974E183EAEB
:10BB60009FE00E94759AAE014B5D5F4F61E070E00F
:10BB700081E20E94E49E8DA190E00E94409A66E0DE
:10BB800082E20E94B79D9920B1F08091040D882334
:10BB900091F068E774E183EA9FE00E94759AAE0134
:10BBA0004B5D5F4F61E070E082E20E94E49E8DA1F8
:10BBB00090E00E94409A67E083E20E94B79D99203E
:10BBC000B1F08091040D882391F062E674E183EA7C
:10BBD0009FE00E94759AAE014B5D5F4F61E070E09F
:10BBE00083E20E94E49E8DA190E00E94409A68E06A
:10BBF00084E20E94B79D9920B1F08091040D8823C2
:10BC000091F06AE474E183EA9FE00E94759AAE01C4
:10BC10004B5D5F4F61E070E084E20E94E49E8DA185
:10BC200090E00E94409A69E085E20E94B79D9920C9
:10BC3000B1F08091040D882391F060E374E183EA10
:10BC40009FE00E94759AAE014B5D5F4F61E070E02E
:10BC500085E20E94E49E8DA190E00E94409A6AE0F5
:10BC600086E20E94B79D9920B1F08091040D88234F
:10BC700091F06AE174E183EA9FE00E94759AAE0157
:10BC80004B5D5F4F61E070E086E20E94E49E8DA113
:10BC900090E00E94409A6BE088E20E94B79D992054
:10BCA000B1F08091040D882391F061E074E183EAA2
:10BCB0009FE00E94759AAE014B5D5F4F61E070E0BE
:10BCC00088E20E94E49E8DA190E00E94409A6CE080
:10BCD00089E20E94B79D992009F479C08091040DF2
:10BCE000882309F474C069EE73E183EA9FE00E943F
:10BCF000759AAE014B5D5F4F61E070E089E20E9492
:10BD0000E49E8DA190E00E94409A62ED73E183EA87
:10BD10009FE00E94759A66E070E087E20E941D9F96
:10BD200090E00E94409A6BEB73E183EA9FE00E94EF
:10BD3000759A65E070E087E20E941D9F90E00E9486
:10BD4000409A64EA73E183EA9FE00E94759A64E096
:10BD500070E087E20E941D9F90E00E94409A6BE88D
:10BD600073E183EA9FE00E94759A62E070E087E2E7
:10BD70000E941D9F90E00E94409A62E773E183EA6F
:10BD80009FE00E94759A61E070E087E20E941D9F2B
:10BD900090E00E94409A69E573E183EA9FE00E9487
:10BDA000759A70E060E087E20E941D9F90E00E941B
:10BDB000409A68E473E183EA9FE00E94759A63E029
:10BDC00070E087E20E941D9F90E00E94409A41E04F
:10BDD00067E070E087E20E94389F41E063E070E036
:10BDE00087E20E94389F41E063E070E08AE20E94AF
:10BDF000389F992091F08091040D882371F06FE2B3
:10BE000073E183EA9FE00E94759A63E070E08AE242
:10BE10000E941D9F90E00E94409A40E063E070E025
:10BE20008AE20E94389F992091F08091040D882326
:10BE300071F065E173E183EA9FE00E94759A63E027
:10BE400070E08AE20E941D9F90E00E94409A41E0CB
:10BE500062E070E08AE20E94389F992091F0809120
:10BE6000040D882371F069EF72E183EA9FE00E947C
:10BE7000759A62E070E08AE20E941D9F90E00E9445
:10BE8000409A40E062E070E08AE20E94389F992088
:10BE900091F08091040D882371F06CED72E183EADA
:10BEA0009FE00E94759A62E070E08AE20E941D9F06
:10BEB00090E00E94409A41E061E070E08AE20E94D6
:10BEC000389F992091F08091040D882371F060ECE7
:10BED00072E183EA9FE00E94759A61E070E08AE275
:10BEE0000E941D9F90E00E94409A40E061E070E057
:10BEF0008AE20E94389F992091F08091040D882356
:10BF000071F063EA72E183EA9FE00E94759A61E052
:10BF100070E08AE20E941D9F90E00E94409A41E0FA
:10BF200070E060E08AE20E94389F992091F0809151
:10BF3000040D882371F067E872E183EA9FE00E94B4
:10BF4000759A70E060E08AE20E941D9F90E00E9476
:10BF5000409A40E070E060E08AE20E94389F9920B9
:10BF600091F08091040D882371F06AE672E183EA12
:10BF70009FE00E94759A70E060E08AE20E941D9F37
:10BF800090E00E94409A41E066E070E087E20E9403
:10BF9000389F41E065E070E087E20E94389F41E011
:10BFA00064E070E087E20E94389F40E062E070E069
:10BFB00087E20E94389F40E061E070E087E20E94E3
:10BFC000389F40E070E060E087E20E94389F99204F
:10BFD00009F475C08091040D882309F470C062E5EE
:10BFE00072E183EA9FE00E94759A66E070E08BE25E
:10BFF0000E941D9F90E00E94409A64E372E183EAF0
:10C000009FE00E94759A65E070E08BE20E941D9FA0
:10C0100090E00E94409A66E172E183EA9FE00E940C
:10C02000759A64E070E08BE20E941D9F90E00E9490
:10C03000409A6DEF71E183EA9FE00E94759A62E099
:10C0400070E08BE20E941D9F90E00E94409A64EE97
:10C0500071E183EA9FE00E94759A61E070E08BE2F3
:10C060000E941D9F90E00E94409A6BEC71E183EA70
:10C070009FE00E94759A70E060E08BE20E941D9F35
:10C0800090E00E94409A68EB71E183EA9FE00E9491
:10C09000759A63E070E08BE20E941D9F90E00E9421
:10C0A000409A63EA71E183EA9FE00E94759A64E036
:10C0B00070E08CE20E941D9F90E00E94409A40E058
:10C0C00064E070E08CE20E94389FAE014B5D5F4FF0
:10C0D00061E070E08CE20E94E49E6DA1607F66608A
:10C0E0008CE20E94B79D992009F45EC08091040DF6
:10C0F000882309F459C06FE871E183EA9FE00E9448
:10C10000759AAE014B5D5F4F61E070E08CE20E947A
:10C11000E49E6DA16F706650770B072E000C880BA4
:10C12000990B0E94ABB49B01AC0160E070E080E031
:10C1300090E40E94F7B820E030E048EC50E40E9420
:10C140000AB50E94F79968E771E183EA9FE00E94CF
:10C15000759AAE014B5D5F4F61E070E080E30E9435
:10C16000E49E6DA14AE050E083EA9FE00E94B1980E
:10C1700060E671E183EA9FE00E94759A61E070E0F9
:10C1800080E30E941D9F90E00E94409A67E471E165
:10C1900083EA9FE00E94759A61E070E08FE20E945E
:10C1A0001D9F90E00E94409A41E061E070E08FE2C4
:10C1B0000E94389F992091F08091040D882371F09E
:10C1C0006FE271E183EA9FE00E94759A61E070E09E
:10C1D0008EE20E941D9F90E00E94409A41E061E043
:10C1E00070E08EE20E94389F40E067E070E081E3FB
:10C1F0000E94389F992009F455C08091040D88232E
:10C2000009F450C06CE171E183EA9FE00E94759AE5
:10C2100067E070E081E30E941D9F90E00E94409AD9
:10C2200068E77AE083EA9FE00E94539AAE014B5D93
:10C230005F4F61E070E080E00E94E49E8DA10E946B
:10C24000A41364ED7BE083EA9FE00E94C8980DE1AF
:10C2500010E069E477E083EA9FE00E94539A40E1AE
:10C2600050E0B80183EA9FE00E94069A6CE77AE00A
:10C2700083EA9FE00E94539AAE014B5D5F4F61E0FD
:10C2800070E0802F0E94E49E8DA10E94A41364EDB3
:10C290007BE083EA9FE00E94C8980F5F1F4F0A333C
:10C2A0001105B9F6A9960FB6F894DEBF0FBECDBF43
:10C2B000DF91CF911F910F91FF90EF90DF90CF9082
:10C2C000BF90AF909F907F906F905F904F90089538
:10C2D0001F93CF93DF93CDB7DEB7A8970FB6F8942F
:10C2E000DEBF0FBECDBF182F0E947C948EE10E944E
:10C2F000D98A62E080E490E10E94FD0B60E080E476
:10C3000090E10E94FD0B0E94B49D8EE10E94D98AAB
:10C3100061E080E490E10E94FD0B60E280E490E146
:10C320000E94FD0B0E94B49D80E290E09093F41275
:10C330008093F31280E090E8A9E8B4E48093E204EB
:10C340009093E304A093E404B093E50480E090E0CC
:10C35000A5E7B4E48093DE049093DF04A093E004A7
:10C36000B093E104BE016F5F7F4F80EF92E10E94C6
:10C37000878A112309F484C062E97CE083EA9FE0A4
:10C380000E94759A83EA9FE00E94AD9862E87CE083
:10C3900083EA9FE00E94759ABE016F5F7F4F83EA38
:10C3A0009FE00E94C89862E77CE083EA9FE00E94D9
:10C3B000759A6D857E858F8598890E94E19862E6E1
:10C3C0007CE083EA9FE00E94759A69897A898B896B
:10C3D0009C890E94E19862E57CE083EA9FE00E94EC
:10C3E000759A20E030E040E251E4698D7A8D8B8DC2
:10C3F0009C8D0E940AB542E00E9415996FE77AE091
:10C4000083EA9FE00E94C89862E47CE083EA9FE0B0
:10C410000E94759A20E030E040E251E46D8D7E8DFF
:10C420008F8D98A10E940AB542E00E9415996FE78E
:10C430007AE083EA9FE00E94C89862E37CE083EAA6
:10C440009FE00E94759A20E030E040E251E469A14B
:10C450007AA18BA19CA10E940AB542E00E94159985
:10C460006FE77AE083EA9FE00E94C8986CE07CE086
:10C4700083EA9FE00E94759A83EA9FE00E94AD984C
:10C4800064EF71E080E090E00E94F19FA8960FB603
:10C49000F894DEBF0FBECDBFDF91CF911F910895FD
:10C4A0002F923F924F925F926F927F928F929F92C4
:10C4B000AF92BF92CF92DF92EF92FF920F931F93B2
:10C4C000CF93DF93CDB7DEB7C854D1090FB6F89438
:10C4D000DEBF0FBECDBF2B013C012DA73EA74FA74E
:10C4E00058AB28EE421623E052066104710434F082
:10C4F00030E9432E55245394612C712CCDA4DEA435
:10C50000EFA4F8A820E1C21627E2D206E104F10464
:10C5100054F020E1C22E27E2D22EE12CF12CCDA640
:10C52000DEA6EFA6F8AA8091030D882341F0C12C66
:10C53000D12C7601C394CDA6DEA6EFA6F8AA0E9460
:10C540008DA625966CAF7DAF8EAF9FAF25970E94CD
:10C550008DA66DAB7EAB8FAB98AF25966CAD7DADE8
:10C560008EAD9FAD259728EE33E040E050E00E946D
:10C57000E1B529962CAF3DAF4EAF5FAF299721E0D3
:10C580002DA319A61AA61BA61CA68E01035F1F4F7A
:10C59000CC24DD247601C418D508E608F708C9AA1A
:10C5A000DAAAEBAAFCAA6DA97EA98FA998AD259657
:10C5B000CCACDDACEEACFFAC25976C197D098E09D7
:10C5C0009F09CDA4DEA4EFA4F8A86C157D058E0507
:10C5D0009F050CF0C2C30E94ABB420E030E04AE7F4
:10C5E00054E40E9423B7AB01BC0123E0C8010E94C0
:10C5F000A697B8018FEA92E10E946597C8010E9450
:10C600009E97A70196012A303105410551058CF40A
:10C6100029964CAD5DAD6EAD7FAD2997C8010E94E6
:10C620003495B8018FEA92E10E946597C8010E9493
:10C630009E978091030D882309F463C264ED7BE02B
:10C640008FEA92E10E942A95CE0101960E94639F93
:10C6500064ED7BE085EB92E10E942A95AE014F5F8D
:10C660005F4F1A01812C912C5401D101CD90DD90A6
:10C67000ED90FD901D01A7019601C701B6010E9432
:10C680000AB59B01AC01C501B4010E9445B64B013E
:10C690005C0123E0B701A601C8010E94A697B8017A
:10C6A000CE0143960E9401986CE57AE0CE01439654
:10C6B0000E94A296BC0185EB92E10E942297CE01D6
:10C6C00043960E949E97C8010E949E9720163106AD
:10C6D00061F6C501B4010E944DB94B015C01BDE298
:10C6E0004B16B1E05B066104710434F00E94B85748
:10C6F00060E080E00E94F48A23E0B501A401CE014D
:10C7000043960E94A69763E87AE0C8010E940A98BF
:10C710006FEA72E1C8010E94B89666E87AE00E946A
:10C72000A296BE016D5E7F4F0E94B8966BE87AE0DC
:10C730000E94A296BC0185EB92E10E942297C8015B
:10C740000E949E97CE0143960E949E972AE939E95E
:10C7500049E55FE3C501B4010E942CB818160CF03E
:10C76000E7C123E333E343E95FE3C501B4010E947A
:10C77000A4B4880F880BCDA0C822CDA28091060C4E
:10C780009091070C8130910509F4E7C1029721F0DF
:10C79000DDA0DD2009F4E1C189849A84AB84BC84E6
:10C7A000C980DA80EB80FC80CDA2DEA2EFA2F8A6E1
:10C7B000CD80DE80EF80F88420E030E0A901C50163
:10C7C000B4010E94A4B4882309F4B4C12DA13EA1F0
:10C7D0004FA158A5CA01B9010E940AB569AF7AAF45
:10C7E0008BAF9CAFA7019601C701B6010E940AB5A5
:10C7F0009B01AC0169AD7AAD8BAD9CAD0E9445B695
:10C800000E944DB9A50194010E94C4B620EE3EE2FB
:10C8100045E652E40E940AB569AF7AAF8BAF9CAF90
:10C8200020E030E0A901C701B6010E94A4B488232A
:10C8300009F485C12DA13EA14FA158A5CA01B90196
:10C840000E940AB521966CAF7DAF8EAF9FAF219746
:10C85000A5019401C501B4010E940AB59B01AC0178
:10C8600021966CAD7DAD8EAD9FAD21970E9445B6F2
:10C870000E944DB9A70196010E94C4B620EE3EE287
:10C8800045E652E40E940AB521966CAF7DAF8EAFAB
:10C890009FAF219720E030E0A9016DA17EA18FA17B
:10C8A00098A50E94A4B4882309F44EC1A50194015F
:10C8B000C501B4010E940AB54B015C01A7019601B4
:10C8C000C701B6010E940AB59B01AC01C501B401C4
:10C8D0000E9445B60E944DB92DA13EA14FA158A579
:10C8E0000E94C4B66B017C016FEA72E1C8010E942C
:10C8F00001986EE87AE0C8010E94A296BC0185EB1F
:10C9000092E10E944E97C8010E949E9765EB72E1EA
:10C91000C8010E940198C8010E94A157C8010E9445
:10C920009E9721E049AD5AAD6BAD7CADCE014F96DF
:10C930000E94A69721E021964CAD5DAD6EAD7FAD16
:10C940002197CE0149960E94A69720EE3EE245E649
:10C9500052E4C701B6010E940AB5AB01BC0121E057
:10C96000C8010E94A697B801CE0143960E94019883
:10C970006CE57AE0CE0143960E94A296BE01675E06
:10C980007F4F0E94B8966CE57AE00E94A296BE01A5
:10C99000615E7F4F0E94B896BC0185EB92E10E94D8
:10C9A0004E97CE0143960E949E97C8010E949E9783
:10C9B000CE0149960E949E97CE014F960E949E9767
:10C9C00065EB72E189EA92E10E944E9765EB72E1B4
:10C9D000C8010E940198C8010E948457C8010E94A2
:10C9E0009E972DE2421621E05206610471047CF408
:10C9F00069A57AA58BA59CA525E030E040E050E034
:10CA00000E94E1B5672B682B692B09F044C06CE0EC
:10CA100075E18FEA92E10E9429976FEA72E1C801FD
:10CA20000E94019845E050E06FEF7FEFC8010E943F
:10CA3000D658C8010E949E9766EA7AE0C8010E9413
:10CA40000A9845E050E061EF7FEFC8010E948059ED
:10CA5000C8010E949E9764ED7BE0C8010E940A987D
:10CA6000C8010E94DC57C8010E949E9765EB72E1E5
:10CA7000C8010E94019845E050E070E060E0C80104
:10CA80000E94FA57C8010E949E9764ED7BE085EBF7
:10CA900092E10E942A95B201C30177FE04C069A900
:10CAA0007AA98BA99CA90E94F19F31E03DA30E9425
:10CAB0008DA66B017C012DA93EA94FA958ADC21AC4
:10CAC000D30AE40AF50AC9A6DAA6EBA6FCA6C414A2
:10CAD000D504E604F70444F4C301B2016C197D09DE
:10CAE0008E099F090E94F19F0E948DA66DAB7EABBF
:10CAF0008FAB98AF64ED7BE085EB92E10E942A95C5
:10CB000052CD64E87AE0C8010E940A986FEA72E1A7
:10CB1000C8010E94B89660E979E00E94A296BC0123
:10CB20008FEA92E10E944E97C8010E949E978CCD99
:10CB30001DA224CE6BED7FE089EC9FE367CE6BED09
:10CB40007FE089EC9FE39ACE8BEDC82E8FE0D82E44
:10CB500089ECE82E8FE3F82EC7CE68EA7AE0C801A8
:10CB60000E940A9865EB72E1C8010E94B896BC0168
:10CB700085EB92E10E944E97C8010E949E9765EB5B
:10CB800072E1C8010E940198C8010E948457C8013F
:10CB90000E949E9765EB72E1C8010E940198C8014E
:10CBA0000E946D18C8010E949E9723E0B501A40160
:10CBB000CE0143960E94A69768E87AE0C8010E94D9
:10CBC0000A98BE016D5E7F4FC8010E94B8966BE85F
:10CBD0007AE00E94A296BC0185EB92E10E944E97FA
:10CBE000C8010E949E97CE0143960E949E9765EBD6
:10CBF00072E1C8010E940198C8010E946D18C80125
:10CC00000E949E976FEA72E1C8010E94019865EB4D
:10CC100072E1C8010E94B896BC0185EB92E10E94C6
:10CC20004E97C8010E949E9765EB72E1C8010E9471
:10CC30000198C8010E948457C8010E949E974981AB
:10CC40005A816B817C8123E0CE0143960E94A69796
:10CC500065EB7AE0C8010E940A98BE016D5E7F4FC5
:10CC6000C8010E94B8966CE87AE00E94A296BC01C6
:10CC70008FEA92E10E942297C8010E949E97CE01FE
:10CC800043960E949E9749855A856B857C8523E053
:10CC9000CE0149960E94A6974D815E816F8178856D
:10CCA00023E0C8010E94A697B801CE0143960E94D6
:10CCB000019869EB7AE0CE0143960E94A296BE01EC
:10CCC000675E7F4F0E94B8966CE87AE00E94A29659
:10CCD000BC0189EA92E10E944E97CE0143960E94E0
:10CCE0009E97C8010E949E97CE0149960E949E97EA
:10CCF0004DE2441641E054066104710474F469A5E0
:10CD00007AA58BA59CA525E030E040E050E00E948C
:10CD1000E1B5672B682B692BF1F46FEA72E1C8016A
:10CD20000E9401984AE050E06FEF7FEFC8010E9437
:10CD3000D658C8010E949E9769EA72E1C8010E9414
:10CD400001984AE050E070E060E0C8010E94FA57A4
:10CD5000C8010E949E971DA2AACE6FEA72E1CE0181
:10CD60000D960E9401984AE050E06FEF7FEFCE01F0
:10CD70000D960E948059CE010D960E949E97CDA0DF
:10CD8000CC20B1F166EA7AE0CE010D960E940A98B5
:10CD900045E050E061EF7FEFCE010D960E94805993
:10CDA000CE010D960E949E978091030D882391F0ED
:10CDB00064E075E1CE010D960E94F89745E050E0E1
:10CDC00070E060E0CE010D960E948059CE010D9674
:10CDD0000E949E9764ED7BE0CE010D960E940A981A
:10CDE000CE010D960E94DC57CE010D960E949E97B3
:10CDF00069EA72E1CE010D960E9401984AE050E086
:10CE00006FEF7FEFCE010D960E94FA57CE010D967F
:10CE10000E949E97C85BDF4F0FB6F894DEBF0FBE2F
:10CE2000CDBFDF91CF911F910F91FF90EF90DF90D9
:10CE3000CF90BF90AF909F908F907F906F905F90BA
:10CE40004F903F902F9008954F925F926F927F92F4
:10CE50008F929F92AF92BF92CF92DF92EF92FF920A
:10CE6000CF93DF93CDB7DEB72C970FB6F894DEBF24
:10CE70000FBECDBF0E94B8570E9491A02B013C016C
:10CE80000E943CA04B015C016091C7047091C804F2
:10CE90008091C9049091CA040E94ABB46B017C01DB
:10CEA0000E9491A00E94ABB4A70196010E9423B7F3
:10CEB00021E03EED42E45EE30E94F7B89B01AC0145
:10CEC00060E070E080E89FE30E9444B620E03AE230
:10CED0004DE257E40E940AB56B017C01C301B20127
:10CEE0000E94ABB420E030E048EC52E40E9423B74B
:10CEF000AB01BC0122E0CE0101960E94A697BE01C3
:10CF00006F5F7F4F89EA92E10E946597CE0101969B
:10CF10000E949E9767E076E089EA92E10E94189766
:10CF200069EA72E18FEA92E10E944E9763E076E04F
:10CF3000CE0101960E940A9869EA72E1CE0101963B
:10CF40000E94B896BC0189EA92E10E944E97CE01F8
:10CF500001960E949E9766EF76E085EB92E10E9433
:10CF60002A9521E0B501A401CE0101960E94A69761
:10CF7000BE016F5F7F4F85EB92E10E942297CE0149
:10CF800001960E949E976CEB7AE085EB92E10E94FD
:10CF9000189721E0B701A601CE0101960E94A6973D
:10CFA000BE016F5F7F4FCE0107960E94019862E439
:10CFB0007BE0CE0107960E94A296BC0185EB92E130
:10CFC0000E942297CE0107960E949E97CE0101965D
:10CFD0000E949E9769EA72E1CE0101960E94019833
:10CFE0006CE57AE0CE0101960E94A29665EB72E1B3
:10CFF0000E94B896BC0185EB92E10E944E97CE014B
:10D0000001960E949E9721E0B501A401CE010196F0
:10D010000E94A697BE016F5F7F4F8BEB92E10E944B
:10D020006597CE0101960E949E976BEB72E1CE014F
:10D0300001960E9401984AE050E070E060E0CE0165
:10D0400001960E948059CE0101960E949E9765E04C
:10D0500070E080E090E00E94F19F61ED75E0CE010C
:10D0600001960E940A98CE0101960E94DC57CE01DB
:10D0700001960E949E976FEA72E1CE0101960E948E
:10D0800001984AE050E06FEF7FEFCE0101960E94D9
:10D09000FA57CE0101960E949E9720E0B701A601A3
:10D0A000CE0101960E94A697BE016F5F7F4FCE0111
:10D0B00007960E94019862E47BE0CE0107960E94E9
:10D0C000A296BC018BEB92E10E944E97CE0107968F
:10D0D0000E949E97CE0101960E949E976BEB72E193
:10D0E000CE0101960E9401984AE050E064EF7FEF84
:10D0F000CE0101960E94FA57CE0101960E949E979A
:10D1000065E070E080E090E00E94F19F8091030D67
:10D11000882331F068E572E080E090E00E94F19FA2
:10D120002C960FB6F894DEBF0FBECDBFDF91CF9126
:10D13000FF90EF90DF90CF90BF90AF909F908F9037
:10D140007F906F905F904F9008954F925F926F9293
:10D150007F928F929F92AF92BF92CF92DF92EF9287
:10D16000FF920F931F93CF93DF93CDB7DEB7CA54CF
:10D17000D1090FB6F894DEBF0FBECDBF8C0164EDB0
:10D180007BE0CE01C7960E940A9864ED7BE0CE0159
:10D19000CD960E940A98BE016F5F7F4F80EF92E1AB
:10D1A0000E942F0CCD88DE88EF88F88C20E030E0DC
:10D1B00040E251E4C701B6010E940AB52B013C01CF
:10D1C000898D9A8DAB8DBC8D2B968CAF9DAFAEAFFC
:10D1D000BFAF2B9720E030E040E251E4BC01CD012D
:10D1E0000E940AB54B015C0120E030E040E251E4CE
:10D1F0006D8D7E8D8F8D98A10E940AB527966CAF9C
:10D200007DAF8EAF9FAF2797C701B60190582B9681
:10D210002CAD3DAD4EAD5FAD2B970E94C4B62BED4E
:10D220003FE049EC5FE30E9445B62091C304309192
:10D23000C4044091C5045091C6040E9445B66B01D8
:10D240007C0120E030E0A9010E94A4B487FDCFC298
:10D25000C092AF0CD092B00CE092B10CF092B20C34
:10D26000C090AF0CD090B00CE090B10CF090B20C2C
:10D270002BED3FE049EC50E4C701B6010E942CB809
:10D28000181684F42BED3FE049EC50E4C701B601D9
:10D290000E9444B66093AF0C7093B00C8093B10CB5
:10D2A0009093B20C20E030E044E353E46091AF0C83
:10D2B0007091B00C8091B10C9091B20C0E940AB5A3
:10D2C0002BED3FE049E450E40E9423B76093AB0CA0
:10D2D0007093AC0C8093AD0C9093AE0C0E94CFB7C2
:10D2E000CE018B960E94619562EC7AE0CE01859624
:10D2F0000E940A98BE01655D7F4FCE0185960E940F
:10D30000B8966CEC7AE00E94A296BC018BEB92E19D
:10D310000E944E97CE0185960E949E97CE018B96D5
:10D320000E949E97C090AB0CD090AC0CE090AD0CDE
:10D33000F090AE0C20E030E044EB52E4C701B601BF
:10D340000E94A4B418160CF463C220E030E040E060
:10D350005FE3C701B6010E9445B60E94CFB7CE0178
:10D360008B960E94619563ED7AE0CE0185960E94CE
:10D370000A98BE01655D7F4FCE0185960E94B896E2
:10D38000BC01CE01C7960E944E97CE0185960E94A1
:10D390009E97CE018B960E949E976CEB79E0CE0112
:10D3A000CD960E942A95BE01695C7F4FCE0185967D
:10D3B0000E9401984AE050E070E060E0CE0185965E
:10D3C0000E948059CE0185960E949E970E948DA64C
:10D3D000AB01BC018091B30C9091B40CA091B50C41
:10D3E000B091B60C8C599F4FAF4FBF4F8417950724
:10D3F000A607B70708F091C264ED7BE0CE018596E1
:10D400000E940A98CE0185960E94DC57CE0185962F
:10D410000E949E97BE01635C7F4F86EB93E10E9462
:10D42000559A6CE57AE0CE0185960E940A98BE0175
:10D43000635C7F4FCE0185960E94B896BC01CE01F9
:10D44000C7960E942297CE0185960E949E970E94C1
:10D450008DA6C090BF0CD090C00CE090C10CF09095
:10D46000C20C6C197D098E099F090E94A9B420E0A5
:10D4700030E04AE754E40E9423B7AB01BC0123E04B
:10D48000CE018B960E94A69764E87AE0CE0185963D
:10D490000E940A98BE01655D7F4FCE0185960E946D
:10D4A000B89660E979E00E94A296BC0189EA92E10F
:10D4B0000E944E97CE0185960E949E97CE018B9634
:10D4C0000E949E9769EA72E1CE0185960E940198BA
:10D4D0006BEB72E1CE0185960E94B896BE01695C45
:10D4E0007F4F0E94B896BC01CE01C7960E944E970E
:10D4F000CE0185960E949E976DEB7CE085EB92E1D4
:10D500000E94299721E0B301A201CE0185960E94D5
:10D51000A697BE016B5D7F4F85EB92E10E9422973B
:10D52000CE0185960E949E9721E027964CAD5DAD79
:10D530006EAD7FAD2797CE01C1960E94A69721E0E0
:10D54000B501A401CE018B960E94A6976CE57AE006
:10D55000CE0185960E940A98BE01655D7F4FCE017F
:10D5600085960E94B8966CE57AE00E94A296BE016C
:10D570006F5C7F4F0E94B8966BED7AE00E94A29696
:10D58000BC0185EB92E10E942297CE0185960E9414
:10D590009E97CE018B960E949E97CE01C1960E94C7
:10D5A0009E97A3019201C301B2010E940AB56B01CB
:10D5B0007C01A5019401C501B4010E940AB59B013B
:10D5C000AC01C701B6010E9445B66B017C012796EC
:10D5D0002CAD3DAD4EAD5FAD2797CA01B9010E949C
:10D5E0000AB59B01AC01C701B6010E9445B60E9475
:10D5F0004DB96093A70C7093A80C8093A90C9093DD
:10D60000AA0C6FED7AE085EB92E10E9418974091A9
:10D61000A70C5091A80C6091A90C7091AA0C21E064
:10D62000CE0185960E94A697BE016B5D7F4FCE010D
:10D630008B960E94019860E87AE0CE018B960E945A
:10D64000A296BC018BEB92E10E944E97CE018B9685
:10D650000E949E97CE0185960E949E976BEB72E189
:10D6600085EB92E10E942297C090A70CD090A80C65
:10D67000E090A90CF090AA0C20E030E04AE754E4D6
:10D68000C701B6010E942CB887FD29C020E030E018
:10D690004AE754E4C701B6010E9423B7AB01BC01BD
:10D6A00023E0CE0185960E94A697BE016B5D7F4F59
:10D6B000CE018B960E94019861E87AE0CE018B96AC
:10D6C0000E94A296BC018BEB92E10E944E97CE0184
:10D6D0008B960E949E97CE0185960E949E9720E091
:10D6E00030E64AE656E46091A70C7091A80C809150
:10D6F000A90C9091AA0C0E94A4B4BE01695C7F4F52
:10D7000087FF2AC1CE0185960E94019863E87AE0DE
:10D71000CE0185960E94A29665EB72E10E94B896B2
:10D72000BC0185EB92E10E944E97CE0185960E9446
:10D730009E9703301105A1F465EB72E1CE01859649
:10D740000E940198CE0185960E948457CE0185964D
:10D750000E949E9764ED7BE085EB92E10E942A9502
:10D7600063EE7AE0CE0185960E940A986BEB72E137
:10D77000CE0185960E94B896BC01CE018B960E9480
:10D7800001984AE050E06FEF7FEFCE018B960E9448
:10D79000FA57CE018B960E949E97CE0185960E94E5
:10D7A0009E976AE070E080E090E00E94F19FCE01D9
:10D7B000CD960E949E97CE01C7960E949E97C65B0B
:10D7C000DF4F0FB6F894DEBF0FBECDBFDF91CF9114
:10D7D0001F910F91FF90EF90DF90CF90BF90AF908F
:10D7E0009F908F907F906F905F904F9008952BED5A
:10D7F0003FE049EC50E4C701B6010E9445B6609392
:10D80000AF0C7093B00C8093B10C9093B20C28CDF8
:10D8100020E030E044E353E4C701B6010E94A4B421
:10D820001816CCF0A701960160E070E884E393E459
:10D830000E9444B66093AB0C7093AC0C8093AD0C1B
:10D840009093AE0C0E94CFB7CE018B960E9461954B
:10D8500066ED7AE08ACD20E030E047E853E4C70186
:10D86000B6010E94A4B41816CCF120E030E044E3E5
:10D8700053E4C701B6010E9444B620E030E040E026
:10D880005FE30E9445B66093AB0C7093AC0C809341
:10D89000AD0C9093AE0C0E94CFB7CE018B960E9438
:10D8A000619566ED7AE0CE0185960E940A98BE01E8
:10D8B000655D7F4FCE0185960E94B896BC01CE0172
:10D8C000C7960E944E97CE0185960E949E97CE01E4
:10D8D0008B960E949E9769ED7AE061CDA701960133
:10D8E00060E070E084EB93E40E9444B620E030E016
:10D8F00040E05FE30E9445B66093AB0C7093AC0CC4
:10D900008093AD0C9093AE0C0E94CFB7CE018B9656
:10D910000E94619563ED7AE0C6CF0E948DA60E94B9
:10D92000A9B46B017C016091B30C7091B40C80912F
:10D93000B50C9091B60C0E94ABB420E030E048ECFE
:10D9400051E40E9445B69B01AC01C701B6010E949B
:10D95000A4B487FD51CD65CD85EB92E10E944E9731
:10D9600020CFDF92EF92FF920F931F93CF93DF931D
:10D97000CDB7DEB762970FB6F894DEBF0FBECDBF4E
:10D980008C011092F80C64ED7BE0CE010D960E94A4
:10D990000A98FF24F39483EA9FE00E942A8820914A
:10D9A000F80C181619067CF521112DC083EA9FE0AA
:10D9B0000E9408888A3009F07EC089899A89892B5B
:10D9C00009F481C0F092F80C6CEE7AE0CE01019679
:10D9D0000E940A98BE01635F7F4FCE0101960E94AC
:10D9E000B896BC01CE0107960E940198CE01079619
:10D9F0000E94825BCE0107960E949E97CE010196FF
:10DA00000E949E9760C0F12CE12CDD24D394222348
:10DA100009F460C089899A89019709F045C062EDCF
:10DA200076E0CE0107960E940A98BE01695F7F4F9B
:10DA3000CE010D960E948796F12C811115C069EFD9
:10DA400077E0CE0101960E940A98BE016F5F7F4F7A
:10DA5000CE010D960E948796FF24F3948111F12C3C
:10DA6000CE0101960E949E97CE0107960E949E9736
:10DA7000FF20A1F050E040E0BE01635F7F4FCE0188
:10DA800001960E94CA58BE016F5F7F4F81EC92E100
:10DA90000E946597CE0101960E949E9764E170E016
:10DAA00080E090E00E94F19FBE01635F7F4FC8015C
:10DAB0000E94EF9790C08D3009F47FCF682FCE0180
:10DAC0000D960E94F5966AE070E080E090E00E947A
:10DAD000F19F61CF8CEC9DE00E942A8818161906F0
:10DAE00014F58CEC9DE00E9408888A30A9F08D30F6
:10DAF00099F09091F80C91110FC0682FCE010D96FE
:10DB00000E94F5968FEFE81AF80A65E070E080E071
:10DB100090E00E94F19FDECF89899A89892BA9F331
:10DB2000D092F80CF2CF64E170E080E090E00E94C7
:10DB3000F19FEF28D1F189899A89892BB1F18091E0
:10DB4000040D882361F164ED75E0CE0101960E9419
:10DB50000A98BE016F5F7F4FCE010D960E94879697
:10DB6000F82ECE0101960E949E97F11018C065EF25
:10DB70007AE083EA9FE00E94539ABE01635F7F4F81
:10DB8000CE0101960E940198BE016F5F7F4F83EA2C
:10DB90009FE00E94639ACE0101960E949E9764E1E5
:10DBA00070E080E090E00E94F19F89899A8920913D
:10DBB000F80C211131CF009709F02ECF64E670E008
:10DBC00080E090E00E94F19F0E948DA664ED7BE0D2
:10DBD000C8010E940A98CE010D960E949E97C80126
:10DBE00062960FB6F894DEBF0FBECDBFDF91CF9126
:10DBF0001F910F91FF90EF90DF900895DF92EF92C9
:10DC0000FF920F931F93CF93DF93CDB7DEB72C977F
:10DC10000FB6F894DEBF0FBECDBF8C011092F80C8A
:10DC200064ED7BE0CE0107960E940A98F12CE12C6E
:10DC3000DD24D3948CEC9DE00E942A8818161906E6
:10DC400094F48091F80C81110EC08CEC9DE00E9440
:10DC500008888A30D1F58B859C85892B09F443C0CF
:10DC6000D092F80C40C062E370E080E090E00E9447
:10DC7000F19FEF2851F08CEC9DE00E94CD8864E686
:10DC800070E080E090E00E94F19F8091F80C81119B
:10DC900031C08B859C85892B69F564ED7BE0C801DB
:10DCA0000E940A98CE0107960E949E97C8012C9662
:10DCB0000FB6F894DEBF0FBECDBFDF91CF911F919D
:10DCC0000F91FF90EF90DF9008958D3021F29091A9
:10DCD000F80C9111C0CF682FCE0107960E94F596DF
:10DCE0008FEFE81AF80A6FE070E080E090E00E94A1
:10DCF000F19FA0CF8091040D882379F0BE01695F68
:10DD00007F4FCE0101960E940198CE0101960E949C
:10DD10008457CE0101960E949E97BE01695F7F4F96
:10DD2000C8010E94EF97BECF4F925F926F927F9291
:10DD30008F929F92AF92BF92EF92FF920F931F9399
:10DD4000CF93DF93CDB7DEB762970FB6F894DEBFFF
:10DD50000FBECDBF7C015B0188EE9CE00E94F38D7D
:10DD6000892BD9F464ED7BE0C7010E940A98C701B2
:10DD700062960FB6F894DEBF0FBECDBFDF91CF9194
:10DD80001F910F91FF90EF90BF90AF909F908F9059
:10DD90007F906F905F904F9008954091EC0C509160
:10DDA000ED0C6091EE0C7091EF0CCE0107960E9485
:10DDB000235A8091040D882359F16CEF7AE0CE014B
:10DDC00001960E940A98BE01695F7F4FCE010196BD
:10DDD0000E94B89661E776E00E94A296BC0183EAB1
:10DDE0009FE00E94559ACE0101960E949E97409115
:10DDF000EC0C5091ED0C6091EE0C7091EF0C20E169
:10DE000083EA9FE00E94619883EA9FE00E94AD98B8
:10DE100070E060E0CE0107960E947696182F8A3255
:10DE200011F01092EC0B0E948DA66093FB0C709386
:10DE3000FC0C8093FD0C9093FE0C64ED7BE0CE0116
:10DE40000D960E940A98812F110F990BC0970A977F
:10DE500008F068C0CE0107960E94A795633071054F
:10DE6000810591050CF084C001E010E082E0982E5D
:10DE70000A151B0509F47CC06CE271E080E090E0BB
:10DE80000E94F19F90924C1010924F10412C512CF7
:10DE9000320188ED9CE00E94F38D892B91F48EE194
:10DEA000481651046104710449F16EE170E080E0AC
:10DEB00090E00E94F19F8FEF481A580A680A780A8A
:10DEC000E8CF8EE14816510461047104B9F0409125
:10DED000DC0C5091DD0C6091DE0C7091DF0CCE01FA
:10DEE00001960E94235ABE016F5F7F4FCE010D96AF
:10DEF0000E946597CE0101960E949E9789899A8912
:10DF0000892B39F0BE01635F7F4FCE0107960E94D7
:10DF100022970F5F1F4F64ED7BE0CE010D960E94AC
:10DF20002A95A6CF6CE271E080E090E00E94F19F1C
:10DF300082E080934C1010924F10812C912C540150
:10DF400088ED9CE00E94F38D892B61F58EE18816A7
:10DF50009104A104B10409F043C089899A89892BED
:10DF600039F0BE01635F7F4FCE0107960E94229772
:10DF700064E670E080E090E00E94F19F82E0809390
:10DF80004C1010924F10BE01695F7F4FC7010E9475
:10DF9000EF97CE010D960E949E97CE0107960E94A4
:10DFA0009E97E5CE8EE188169104A104B104A9F2F2
:10DFB0004091DC0C5091DD0C6091DE0C7091DF0C17
:10DFC000CE0101960E94235ABE016F5F7F4FCE01A2
:10DFD0000D960E946597CE0101960E949E97BDCF37
:10DFE0006EE170E080E090E00E94F19F8FEF881A70
:10DFF000980AA80AB80AA4CFAF92BF92CF92DF9234
:10E00000EF92FF920F931F93CF93DF93CDB7DEB7BD
:10E010002C970FB6F894DEBF0FBECDBF7C015B011D
:10E020000E94E8A7182F811117C064ED7BE0C7019B
:10E030000E940A98C7012C960FB6F894DEBF0FBE57
:10E04000CDBFDF91CF911F910F91FF90EF90DF90A7
:10E05000CF90BF90AF9008958A3211F01092EC0BE0
:10E060000E948DA66093FB0C7093FC0C8093FD0CBA
:10E070009093FE0C612FCE0107960E94D697812FB8
:10E08000012E000C990BC0970A9768F5CE010796F0
:10E090000E94A79563307105810591050CF070C051
:10E0A00001E010E00A151B0509F46AC062E370E0A4
:10E0B00080E090E00E94F19F0E94E8A7D12CC12C43
:10E0C00081113BC08FEFC81AD80A85E1C816D10468
:10E0D00009F456C06EE170E080E090E00E94F19F8C
:10E0E0000E94E8A7EDCF612FCE0101960E94D6973E
:10E0F000BE016F5F7F4FCE0107960E946597CE01EC
:10E1000001960E949E9762E370E080E090E00E949A
:10E11000F19F0E94E8A710E000E0811121C00F5F8D
:10E120001F4F0F31110561F16EE170E080E090E06A
:10E130000E94F19F0E94E8A7F0CF682FCE010196C0
:10E140000E94D697BE016F5F7F4FCE0107960E9457
:10E150002297CE0101960E949E970F5F1F4FA2CF7C
:10E16000682FCE0101960E94D697BE016F5F7F4F48
:10E17000CE0107960E942297CE0101960E949E979B
:10E18000BE01695F7F4FC7010E94EF97CE010796DE
:10E190000E949E974FCF3F924F925F926F927F92D5
:10E1A0008F929F92AF92BF92CF92DF92EF92FF92A7
:10E1B0000F931F93CF93DF93CDB7DEB7E4970FB6DE
:10E1C000F894DEBF0FBECDBF8091EC0B8823D1F059
:10E1D0001092EC0BE4960FB6F894DEBF0FBECDBFE5
:10E1E000DF91CF911F910F91FF90EF90DF90CF9033
:10E1F000BF90AF909F908F907F906F905F904F9067
:10E200003F90089581E08093EC0B64ED7BE0CE01BC
:10E2100085960E940A9864ED7BE0CE018B960E9461
:10E220000A9810E000E082E0382E98EEC92E93E0C4
:10E23000D92EE12CF12CF8013197E031F105B0F441
:10E240008827EA5DFE488F4F0C94CFB90B72A272FB
:10E25000B772C072C972D272E372EC721B732C7304
:10E2600035733E734773E273EB73F47364ED7BE0D5
:10E27000CE0185960E942A958091941190919511D6
:10E28000892B31F46AE676E0CE0185960E942A95C4
:10E290008091941190919511019731F464E676E0A4
:10E2A000CE0185960E942A958091941190919511A6
:10E2B000029731F46EE676E0CE0185960E942A95AB
:10E2C00089A59AA5892B31F06AEA73E1CE0185967A
:10E2D0000E94229763E776E0CE0101960E940A9899
:10E2E00064EA73E1CE0101960E94B896BC01CE01AA
:10E2F0008B960E944E97CE0101960E949E97809128
:10E30000941190919511019709F046C0BE016B5D83
:10E310007F4FCE0101960E94019848EC50E06FEFCC
:10E320007FEFCE0101960E948059CE0101960E9496
:10E330009E97BE01655D7F4FCE0101960E940198B8
:10E3400040ED57E06FEF7FEFCE0101960E94FA5744
:10E35000CE0101960E949E97CE0101960E94DD316A
:10E360008D819E810097A1F0E981FA81208122238D
:10E3700079F0079768F065EF7EE0CE0185960E9400
:10E380002997BE016F5F7F4FCE018B960E944E97FB
:10E39000CE0101960E949E97BE016B5D7F4FCE011C
:10E3A00001960E94019848EC50E06FEF7FEFCE019C
:10E3B00001960E94D658CE0101960E949E97BE01FA
:10E3C000655D7F4FCE0101960E94019848EC50E0B8
:10E3D0006FEF7FEFCE0101960E94FA57CE010196B2
:10E3E0000E949E970E94E8A7982EB12CA12C911014
:10E3F00060C28FEFA81AB80A95E6A916B10409F40D
:10E40000FCC10E94E8A7982E64E170E080E090E0F3
:10E410000E94F19FECCF69EE7EE0CE0185960E94CE
:10E4200029970E948DA64B015C010E948DA6A70131
:10E4300096010E9413B6CA01B90120E831E541E016
:10E4400050E00E9413B620E13EE040E050E00E9420
:10E45000E1B529AB3AAB4BAB5CAB2CE330E040E031
:10E4600050E00E94E1B529013A01AB01BC01CE01A7
:10E4700001960E943495B301A201CE0107960E9435
:10E48000349549A95AA96BA97CA9CE010D960E9481
:10E490003495C501B40120E03CE546E255E00E9418
:10E4A00013B6BA01A901CE0149960E943495BE0166
:10E4B000675E7F4FCE0143960E94019861E07BE04A
:10E4C000CE0143960E94A296BE01635F7F4F0E94D9
:10E4D000B89664E07BE00E94A296BE01695F7F4F20
:10E4E0000E94B89669EC76E00E94A296BE016F5F2A
:10E4F0007F4F0E94B89662ED76E00E94A296BC0122
:10E50000CE014F960E940198CE0143960E949E979D
:10E51000CE0149960E949E97CE010D960E949E972D
:10E52000CE0107960E949E97CE0101960E949E976B
:10E53000BE01615E7F4FCE018B960E946597CE0132
:10E540004F9628CF8091040C9091050C6AED7EE0E7
:10E55000019711F06CEC7EE0CE0185960E94299720
:10E560006CEB7EE0CE018B960E94299715CF6CEA6A
:10E570007EE0CE0185960E9429976FE97EE0F2CF7A
:10E5800062E97EE0CE0185960E94299767E87EE0E9
:10E59000E9CF6BE77EE0CE0185960E9429976AE677
:10E5A0007EE0E0CF8091040C9091050C6FE57EE059
:10E5B000039711F065E57EE0CE0185960E942997CC
:10E5C0006AE47EE0CFCF6DE37EE0CE0185960E94C7
:10E5D00029976EE27EE0C6CF63E27EE0CE018596AB
:10E5E0000E94299760914B1170914C11CE010796B2
:10E5F0000E94619565E67AE0CE0101960E940A9834
:10E60000BE01695F7F4FCE0101960E94B89666E316
:10E610007AE00E94A296BC01CE0185960E942297C4
:10E62000CE0101960E949E97CE0107960E949E976A
:10E6300066E17EE097CF8091040C9091050C65E037
:10E640007EE0029711F065EF7DE0CE0185960E9495
:10E65000299768EE7DE086CF6CED7DE0CE01859652
:10E660000E9429976CEC7DE07DCF61EC7DE0CE01CE
:10E6700085960E94299767EB7DE074CF6BEA7DE079
:10E68000CE0185960E9429976BE97DE06BCFB09013
:10E690004D1160E97DE0CE0185960E94299783E0C7
:10E6A0008B1524F192E0B9160CF073C0BB2031F148
:10E6B00081E0B81609F464C060914D11062E000C7B
:10E6C000770BCE0107960E94619569E279E0CE0151
:10E6D00001960E940A98BE01695F7F4FCE010196A4
:10E6E0000E94B896BC0185EB92E13FC094E0B9125C
:10E6F000E3CF6BE07BE085EB92E146C080904E116A
:10E7000090904F11A0905011B090511120E030E046
:10E7100048E452E4C501B4010E94A4B487FF02C0DA
:10E7200033243394A501940160E070E080EA90E422
:10E730000E9423B7AB01BC01232DCE0107960E9496
:10E74000A69764E87AE0CE0101960E940A98BE017D
:10E75000695F7F4FCE0101960E94B89660E17BE031
:10E760000E94A296BC01CE0185960E942297CE01FE
:10E7700001960E949E97CE0107960E949E9706C022
:10E7800067E07BE0CE0185960E94189760E87DE007
:10E79000E9CE8B2D9AE08902B0011124CE010796B3
:10E7A0000E94619565E67AE0CE0101960E940A9882
:10E7B000BE01695F7F4FCE0101960E94B89669E065
:10E7C0007BE0CECF63E77DE0CE0185960E9429975E
:10E7D00063E67DE0C7CE67E57DE0CE0185960E94C9
:10E7E000299768E47DE0BECE6CE37DE0CE0185969E
:10E7F0000E9429976CE27DE0B5CE64ED7BE083ED6D
:10E8000092E10E942A95CE0101960E94B16CBE0150
:10E810006F5F7F4F83ED92E10E946597CE01019675
:10E820000E949E978091D7129091D812892B89F4DB
:10E8300061E070E0CE0101960E94FC6FBE016F5F47
:10E840007F4F83ED92E10E946597CE0101960E9471
:10E850009E978091D7129091D812892B89F461E00C
:10E8600070E0CE0101960E94946EBE016F5F7F4FF3
:10E8700083ED92E10E946597CE0101960E949E97DA
:10E880008091D7129091D812892B51F48091EC0B82
:10E89000882331F00F5F1F4F0131110509F0CBCCF8
:10E8A000CE018B960E949E97CE0185960E949E97E0
:10E8B00091CC1092EC0BF4CF2F923F924F925F923B
:10E8C0006F927F928F929F92AF92BF92CF92DF9280
:10E8D000EF92FF920F931F93CF93DF93CDB7DEB7E5
:10E8E000C554D1090FB6F894DEBF0FBECDBF8C0161
:10E8F000E090020CF090030C8091040D882349F005
:10E9000062E171E183EA9FE00E94759AC8010E946A
:10E91000409AC8010596059710F40C948187809160
:10E92000020C9091030C80179107E1F00E94B857F8
:10E930000E94D4150C3E2FEF120724F01093030C05
:10E940000093020CB801CE0101960E946195BE01B0
:10E950006F5F7F4F81EC92E10E946597CE01019637
:10E960000E949E9764ED7BE085EB92E10E942A95E0
:10E970006CE57AE0CE0101960E940A984AE050E0E8
:10E980006FEF7FEFCE0101960E94D658CE0101961F
:10E990000E949E97F8017C96E632F10510F00C94E7
:10E9A00062878827E952FB488F4F0C94CFB9728653
:10E9B0006287C786BF8692867C86628777866287F3
:10E9C0006287628762876287197584750A76927793
:10E9D00099776D79207A487B1F7D1C7E717E867EBB
:10E9E000897E6287CA7ECD7E79803682528270832C
:10E9F000DC83A8842A85328531860E94E415CB5BAE
:10EA0000DF4F0FB6F894DEBF0FBECDBFDF91CF91C1
:10EA10001F910F91FF90EF90DF90CF90BF90AF903C
:10EA20009F908F907F906F905F904F903F902F902E
:10EA300008950E94B85789E390E00E94BC5420E0FA
:10EA400030E04AE754E40E940AB5AB01BC0121E082
:10EA5000CE0101960E94A69765EB78E0CE018096E4
:10EA60000E940A98BE016F5F7F4FCE0180960E9480
:10EA7000B89663E17BE00E94A296BC0185EB92E12F
:10EA80000E944E97CE0180960E949E97CE010196DD
:10EA90000E949E9767E17BE08FEA92E10E942A95AF
:10EAA0006FEA72E1CE0101960E9401984AE050E0BF
:10EAB00068E070E0CE0101960E948059CE01019677
:10EAC0000E949E9765EB72E1CE0101960E9401982B
:10EAD0004AE050E06FEF7FEFCE0101960E94FA57B7
:10EAE000CE0101960E949E976FEA72E185EB92E15A
:10EAF0000E9422978091030D882309F4C8C164E61F
:10EB000070E080E090E07DC4C0900402D0900502E7
:10EB10000E94B85789E390E00E94BC5420E030E0A6
:10EB20004AE754E40E940AB50E94CFB7CE0101968D
:10EB30000E94619565EB78E0CE0180960E940A986C
:10EB4000BE016F5F7F4FCE0180960E94B89663E151
:10EB50007BE00E94A296BC0185EB92E10E944E9759
:10EB6000CE0180960E949E97CE0101960E949E97AC
:10EB70008091B9129091BA12A3E0FA2E099710F081
:10EB8000F2E0FF2E80914A1140E050E0BA0183305C
:10EB9000DCF4C6010E9435174B015C0160914B11FA
:10EBA00070914C11072E000C880B990B0E94ABB48E
:10EBB000A50194010E940AB520E030EC4FE754E42F
:10EBC0000E9423B7AB01BC012F2DCE0101960E94FC
:10EBD000A69765E47BE0CE0180960E940A98BE016C
:10EBE0006F5F7F4FCE0180960E94B89669E176E014
:10EBF0000E94A296BC0185EB92E10E942297CE0171
:10EC000080960E949E97CE0101960E949E976FE18A
:10EC10007BE042CF8091030D882309F478C189E617
:10EC20009EE00E94C28D62E370E080E090E00E946E
:10EC3000F19F61E0809190040E94409C60E080918F
:10EC40008E040E94409C64E670E080E090E00E94A8
:10EC5000F19F60918A0470918B0480918C04909153
:10EC60008D040E9463150E948015AB01BC0123E056
:10EC7000CE0180960E94A697BE01605E7F4FCE01B6
:10EC800001960E94019862E47BE0CE0101960E9409
:10EC9000A296BC018FEA92E10E944E97CE010196A6
:10ECA0000E949E97CE0180960E949E976DEC76E022
:10ECB000CE0101960E940A986FEA72E1CE01019698
:10ECC0000E94B896BC0185EB92E10E944E97CE015E
:10ECD00001960E949E970E9480156B017C010E9404
:10ECE0009F9C4B015C018BE19EE40197F1F70E9430
:10ECF00080152B013C010E949F9C9B01AC012819AF
:10ED000039094A095B0949015A0131ED831637E097
:10ED10009306A104B104CCF0A7019601C301B2018E
:10ED20000E9444B66B017C0120E030E0A9010E9402
:10ED30002CB8181674F426EA3BE944EC5BE3C701EF
:10ED4000B6010E94A4B487FF0EC040E050E0BA01B3
:10ED500026C026EA3BE944EC5BEBC701B6010E9402
:10ED60002CB8181694F3C501B40128EE33E040E046
:10ED700050E00E94E1B5CA01B9010E94ABB44B0159
:10ED80005C0120E030E04AE754E4C701B6010E948C
:10ED90000AB5A50194010E9423B7AB01BC0122E092
:10EDA000CE0180960E94A697BE01605E7F4FCE0185
:10EDB00001960E94019860ED76E0CE0101960E94D6
:10EDC000A296BC0189EA92E10E944E97CE0101967B
:10EDD0000E949E97CE0180960E949E9768E27BE0FB
:10EDE000CE0101960E940A9869EA72E1CE0101966D
:10EDF0000E94B896BC0185EB92E10E942297CE0159
:10EE000001960E949E976CE57AE0CE0101960E94E1
:10EE10000A9869EA72E1CE0101960E94B896BC0197
:10EE20008FEA92E10E942297CE0101960E949E975E
:10EE30006EEF7EE0CE0101960E94F8974AE050E026
:10EE400070E060E0CE0101960E948059CE010196EB
:10EE50000E949E976FEA72E1CE0101960E9401988E
:10EE600045E050E06FEF7FEFCE0101960E94FA5728
:10EE7000CE0101960E949E976CE27BE085EB92E1C9
:10EE80000E94189760E0809190040E94409C8091BD
:10EE9000B9129091BA12009799F14197A8F40230F3
:10EEA000110594F065EB72E1CE0101960E94019884
:10EEB0004AE050E06FEF7FEFCE0101960E94FA57D3
:10EEC000CE0101960E949E9765EB72E1CE010196FC
:10EED0000E940198CE0101960E948457CE010196AE
:10EEE0000E949E9765EB72E1CE0101960E94019807
:10EEF000CE0101960E946D18CE0101960E949E9748
:10EF000064E670E080E090E00E94F19F78CD60912F
:10EF100081047091820480918304909184040E9402
:10EF20003B2DB5CF80917B0490917C040E944E2FA5
:10EF3000AECF40917D0426964FAF269760E0842F98
:10EF40000E94409C8091030D811109C08091AA11FB
:10EF5000EFE0CE2ED12CE12CF12C882329F073E0A8
:10EF6000C72ED12CE12CF12C6DE07FE085EB92E1F6
:10EF70000E94299765EB72E1CE0101960E940198EB
:10EF80004AE050E06FEF7FEFCE0101960E9480597A
:10EF9000CE0101960E949E97312C212C21961FAE06
:10EFA000219725961FAE25971CAE1DAE1EAE1FAE37
:10EFB00062E3662E712C812C912C540126968FAD24
:10EFC00026970E947C9C092E000CAA0BBB0B880E76
:10EFD000991EAA1EBB1E65E070E080E090E00E94D2
:10EFE000F19F51E0651A710849F74090D60450909E
:10EFF000D7046090D8047090D904C501B4010E9470
:10F00000ABB420E030E040EA50E40E940AB520E0D2
:10F0100030E040E85AE30E940AB520E030E048E4DE
:10F0200052E40E9423B7A30192010E9444B620E05B
:10F0300030E040E751E40E940AB54B015C01A301B6
:10F0400092016AE979E989E390E40E9444B69B0160
:10F05000AC01C501B4010E9423B720E030E0A90152
:10F060000E9445B620E030E040E251E40E940AB53B
:10F070004B015C01232D322D21964FAD2197259612
:10F080005FAD25970E942CB8181644F4382C292C13
:10F090002196AFAE21972596BFAE259720E030E0B0
:10F0A000A901B401C5010E94A4B487FF04C0812C4A
:10F0B000912CA12CB12C22E0A401B501CE018096A7
:10F0C0000E94A697BE01605E7F4FCE0101960E940E
:10F0D00001986FE37BE0CE0101960E94A296BC01ED
:10F0E0008FEA92E10E944E97CE0101960E949E9770
:10F0F000CE0180960E949E976FEA72E1CE01019642
:10F100000E9401984AE050E070E060E0CE01019674
:10F110000E94FA57CE0101960E949E970E948DA6EA
:10F12000AB01BC018091B70C9091B80CA091B90CC7
:10F13000B091BA0C8C599F4FAF4FBF4F84179507B2
:10F14000A607B70708F0AAC00E9439556CE370E023
:10F1500080E090E00E94F19F8CAD9DADAEADBFAD63
:10F160000196A11DB11D8CAF9DAFAEAFBFAFC8164C
:10F17000D906EA06FB060CF01BCF64E670E080E0DF
:10F1800090E00E94F19F0E94B85764E670E080E032
:10F1900090E00E94F19F65E07FE08FEA92E10E949B
:10F1A00029976FEA72E1CE0101960E94019844E12D
:10F1B00050E070E060E0CE0101960E948059CE01DF
:10F1C00001960E949E9722E0432D522D21966FAD0D
:10F1D000219725967FAD2597CE0180960E94A69710
:10F1E000BE01605E7F4FCE0101960E9401986FE3E1
:10F1F0007BE0CE0101960E94A296BC018FEA92E1CB
:10F200000E944E97CE0101960E949E97CE01809655
:10F210000E949E976FEA72E1CE0101960E940198CA
:10F2200042E350E06FEF7FEFCE0101960E94FA5764
:10F23000CE0101960E949E9764E170E080E090E02C
:10F240000E94F19F0E9439556EE170E080E090E0ED
:10F250000E94F19F6EE170E080E090E00E94F19FDB
:10F2600064E47BE0CE0101960E940A986FEA72E1A5
:10F27000CE0101960E94B89668E47BE00E94A296B7
:10F2800065EB72E10E94B896BC0185EB92E10E94A9
:10F290004E97CE0101960E949E97F9CD0E948DA6B1
:10F2A0000E94A9B44B015C016091B70C7091B80C3D
:10F2B0008091B90C9091BA0C0E94ABB420E030E080
:10F2C00048EC51E40E9445B69B01AC01C501B40174
:10F2D0000E94A4B487FD38CF39CF80917F049091EC
:10F2E000800499270E9435172DE038E643E55BE35B
:10F2F0000E940AB56B017C0120910505309106053D
:10F3000040910705509108050E94A4B418160CF40A
:10F310007BC06091ED047091EE048091EF049091B8
:10F32000F00420E030E048EC52E40E940AB520E00E
:10F3300030E048EA51E40E940AB52091DA043091A5
:10F34000DB044091DC045091DD040E9423B76B0183
:10F350007C016AE17FE08FEA92E10E9429976FEADF
:10F3600072E1CE0101960E94019842E350E070E004
:10F3700060E0CE0101960E948059CE0101960E9464
:10F380009E9722E0B701A601CE0101960E94A697A2
:10F3900062E57BE0CE0180960E940A98BE016F5F15
:10F3A0007F4FCE0180960E94B8966CE47BE00E946D
:10F3B000A296BC0185EB92E10E944E97CE01809609
:10F3C0000E949E97CE0101960E949E9765EB72E186
:10F3D000CE0101960E94019842E350E06FEF7FEF6B
:10F3E000CE0101960E94FA57CE0101960E949E9787
:10F3F0008091030D882309F44ACD60E273E080E038
:10F4000090E00E94F19F43CD2091190530911A059B
:10F4100040911B0550911C05C701B6010E942CB8F4
:10F4200087FF05C0C701B6010E944B8C7ACF60915F
:10F43000010570910205809103059091040571CF3B
:10F440000E94B8576EE47FE085EB92E10E94299715
:10F4500065EB72E1CE0101960E9401984AE050E00E
:10F4600070E060E0CE0101960E948059CE010196C5
:10F470000E949E9765E47FE08FEA92E10E942997BF
:10F480006FEA72E1CE0101960E94019844E150E0DA
:10F490006FEF7FEFCE0101960E94FA57CE010196E1
:10F4A0000E949E978091BB0C9091BC0C823091057C
:10F4B00009F041C00E9460A5811104C01092BC0CEB
:10F4C0001092BB0C8091BB0C9091BC0C029709F47C
:10F4D00048C069E37FE085EB92E10E94299765EBE4
:10F4E00072E1CE0101960E9401984AE050E070E07E
:10F4F00060E0CE0101960E948059CE0101960E94E3
:10F500009E9765EB72E1CE0101960E9401986CE531
:10F510007AE0CE0101960E94A2966FEA72E10E9403
:10F52000B896BC0185EB92E10E944E97CE01019600
:10F530000E949E975DCF892B61F60E9460A588236B
:10F5400039F082E090E09093BC0C8093BB0CBACF72
:10F550000E9460A58111F5CF0E9460A58111F1CFB5
:10F56000B1CF8AE090E00E9410166B017C0120E090
:10F5700030E0A9010E94A4B4181634F08AE090E0AB
:10F580000E9410166B017C015BE0A52EB12C20E0DF
:10F5900030E042ED53E4C701B6010E94A4B418164E
:10F5A0008CF091E0A91AB10869F068EC70E080E095
:10F5B00090E00E94F19F83E090E00E9410166B01A2
:10F5C0007C01E5CF20E030E0A901C701B6010E942F
:10F5D000A4B418166CF16BE27FE085EB92E10E9417
:10F5E000299765EB72E1CE0101960E94019842E3F2
:10F5F00050E06FEF7FEFCE0101960E94FA57CE01E7
:10F6000001960E949E9762E27FE08FEA92E10E945B
:10F6100029976FEA72E1CE0101960E94019842E3B8
:10F6200050E070E060E0CE0101960E948059DCCE8F
:10F6300020E030E048EC52E4C701B6010E94A4B4D7
:10F6400021E087FF20E0B701A601CE0101960E94CC
:10F65000A69761E57BE0CE0180960E940A98BE01E4
:10F660006F5F7F4FCE0180960E94B89666E57BE083
:10F670000E94A296BC0185EB92E10E944E97CE01BA
:10F6800080960E949E97CE0101960E949E97A9CFD8
:10F690000E948DA62B013C0189E69EE00E94C28D4E
:10F6A00064E670E080E090E00E94F19F40E855E25F
:10F6B00060E070E089E69EE00E94865864E670E0B3
:10F6C00080E090E00E94F19F67E87FE08FEA92E19E
:10F6D0000E9429976FEA72E1CE0101960E9401987B
:10F6E00042E350E06FEF7FEFCE0101960E94805918
:10F6F000CE0101960E949E976CE77FE08FEA92E12F
:10F700000E9429976FEA72E1CE0101960E9401984A
:10F7100042E350E06FEF7FEFCE0101960E94FA576F
:10F72000CE0101960E949E978091040C9091050C49
:10F730008D7F1CAEB12CA12CD12CC12CF12CE12C35
:10F74000019709F47AC0DE019096B9AFA8AFFE0127
:10F750007E96FBAFEAAF0E948DA6641975098609F3
:10F760009709683B7B408105910508F066C089E6F2
:10F770009EE00E942A88892B09F44EC02CED35E0CA
:10F7800040E050E020936D0E30936E0E40936F0E6C
:10F790005093700E0E9499A697FD3EC08234910549
:10F7A000C9F7AE014F5F5F4F1A014A010E9499A647
:10F7B00097FF39C089818D3479F590E080E0D101DF
:10F7C0002D911D01820F911DEAADFBADEA17FB07DC
:10F7D000B1F78E5B9F4F2E8D30E0322F22274F8D59
:10F7E000240F311D82179307B9F4EC80F12CFE2C05
:10F7F000EE248D81E80EF11CCE80D12CDC2CCC24A3
:10F800008F81C80ED11CA884B12CBA2CAA2489855A
:10F81000A80EB11CF1E0FCAF62E370E080E090E084
:10F820000E94F19F98CFD4018D934D01E8ADF9ADC1
:10F83000EA17FB0709F0BACFBDCF0E948DA6641965
:10F84000750986099709683B7B408105910518F485
:10F850003CAD3111BCC00E94B8576FEA72E1CE01D5
:10F8600080960E94019842E350E066E070E0CE018D
:10F8700080960E948059CE0180960E949E974CAD42
:10F88000442309F4B3C082E090E09093050C809388
:10F89000040CB501CE0180960E946195B601CE019F
:10F8A00086960E946195B701CE01C2960E9461952D
:10F8B000BE016E5C7F4FCE018C960E94019861E77D
:10F8C00076E0CE018C960E94A296BE016A5D7F4FC3
:10F8D0000E94B89661E776E00E94A296BE01605E43
:10F8E0007F4F0E94B896BC0185EB92E10E944E9733
:10F8F000CE018C960E949E97CE01C2960E949E9742
:10F90000CE0186960E949E97CE0180960E949E9779
:10F9100065EB72E1CE0180960E9401984AE050E0CA
:10F920006FEF7FEFCE0180960E94FA57CE0180964E
:10F930000E949E9766E77FE086EB93E10E94759AAE
:10F94000B501CE0180960E946195B601CE018696E2
:10F950000E946195B701CE018C960E9461956AE57F
:10F960007BE0CE01C2960E940A98BE01645D7F4F83
:10F97000CE01C2960E94B8966CE57AE00E94A296EB
:10F98000BE016A5D7F4F0E94B8966CE57AE00E94E6
:10F99000A296BE01605E7F4F0E94B8966AE67BE049
:10F9A0000E94A296BC0185EB92E10E944E97CE0187
:10F9B000C2960E949E97CE018C960E949E97CE0181
:10F9C00086960E949E97CE0180960E949E9762E343
:10F9D00070E080E090E00E94F19F89E69EE00E9446
:10F9E000C28D62E370E080E090E00BCD6BE67FE0DB
:10F9F00085EB92E10E94299765EB72E1CE0180963A
:10FA00000E9401984AE050E070E060E0CE018096EC
:10FA10000E94FA57CE0180960E949E9768E57FE08B
:10FA200085EB92E10E9429978091040C9091050C3E
:10FA3000029769F61092050C1092040CC8CFE09062
:10FA40007904F0907A0460E77BE08FEA92E10E940B
:10FA50002A950E94B8576FEA72E1CE0101960E9482
:10FA600001984AE050E06FEF7FEFCE0101960E94CF
:10FA70008059CE0101960E949E97C7010E944618A8
:10FA800024966CAF7DAF8EAF9FAF24978090B30468
:10FA90009090B404A090B504B090B604A501940170
:10FAA0006091AF047091B0048091B1049091B20460
:10FAB0000E9444B62B013C0120E030E0A9010E94E5
:10FAC000A4B4882309F48EC0C090BB04D090BC04B9
:10FAD000E090BD04F090BE0420E030E0A901C70131
:10FAE000B6010E94A4B418160CF07CC08091B70433
:10FAF0009091B804A091B904B091BA048CAF9DAFB5
:10FB0000AEAFBFAF9C01AD01C701B6010E94A4B466
:10FB1000882309F467C0A70196016CAD7DAD8EAD59
:10FB20009FAD0E9423B70E947BB86CAF7DAF8EAFB4
:10FB30009FAFA501940124966CAD7DAD8EAD9FADB8
:10FB400024970E9444B6A30192010E9423B72CADD2
:10FB50003DAD4EAD5FAD0E940AB50E949DB79B01C1
:10FB6000AC01C701B6010E940AB56B017C016FEAC6
:10FB700072E1CE0101960E9401984AE050E070E0E7
:10FB800060E0CE0101960E948059CE0101960E944C
:10FB90009E9720E030E64AEE56E4C701B6010E9487
:10FBA0002CB818161CF563E97FE085EB92E10E9402
:10FBB000299765EB72E1CE0101960E9401984AE017
:10FBC00050E06FEF7FEFCE0101960E94FA57CE0111
:10FBD00001960E949E9764E670E080E090E00E94AB
:10FBE000F19F06CCC12CD12C7601C1CF21E0B70109
:10FBF000A601CE0180960E94A6976AE77BE0CE011F
:10FC000001960E940A98BE01605E7F4FCE01019668
:10FC10000E94B8966EE77BE00E94A296BC0185EB3D
:10FC200092E10E944E97CE0101960E949E97CE01CE
:10FC300080960E949E97BDCFE0900402F09005024E
:10FC40000E94B85765E070E080E090E00E94F19F6C
:10FC500080914A1140E050E0BA018330DCF4C701E2
:10FC60000E9435176B017C0160914B1170914C1112
:10FC7000072E000C880B990B0E94ABB4A7019601CC
:10FC80000E940AB520E030EC4FE754E40E9423B70D
:10FC9000AB01BC0123E0CE0101960E94A69765E46A
:10FCA0007BE0CE0180960E940A98BE016F5F7F4F75
:10FCB000CE0180960E94B89669E176E00E94A296F5
:10FCC000BC0185EB92E10E944E97CE0180960E9486
:10FCD0009E97CE0101960E949E9762E87BE00C946D
:10FCE0004C758091D70C91E089278093D70C809137
:10FCF000030D882331F065EB72E18CEC9DE00E94EE
:10FD0000639A68EC70E080E090E07BCB1092030D8A
:10FD1000BEC881E08093030D8093B8118091AF112C
:10FD2000882349F16AE878E081EC92E10E942A9503
:10FD300086EE9FEF9093030C8093020C2091B211FA
:10FD40003091B3118091B4119091B511821793073E
:10FD500024F01092B5111092B4111092A6111092C5
:10FD6000A7111092A8111092A9116CE271E080E025
:10FD700090E00E94F19F61EC72E187EC92E10E94B9
:10FD80004E978091020C9091030C9093FA0C809303
:10FD9000F90C7DC80E94CB707AC886E09FE00E9473
:10FDA000C28D40E052EC61E070E086E09FE00E948E
:10FDB00086588CED95E0A0E0B0E080930A0F909318
:10FDC0000B0FA0930C0FB0930D0F64E670E080E072
:10FDD00090E00E94F19F8091BB0C9091BC0C019728
:10FDE00079F583E090E00E94AA17811104C0109277
:10FDF000BC0C1092BB0C8091BB0C9091BC0C019779
:10FE0000C9F162ED7FE08FEA92E10E9429976FEAE3
:10FE100072E1CE0101960E94019844E150E06FEF3B
:10FE20007FEFCE0101960E94FA57CE0101960E9403
:10FE30009E9766EC7FE085EB92E10E94299726C1B0
:10FE400081E090E00E94AA17882339F081E090E0D9
:10FE50009093BC0C8093BB0CCECF83E090E00E94CB
:10FE6000AA178111F3CF83E090E00E94AA178111B5
:10FE7000EDCFC1CF6AEB7FE085EB92E10E9429973D
:10FE800065EB72E1CE0101960E940198CE010196C8
:10FE90000E94825BCE0101960E949E9762E370E011
:10FEA00080E090E00E94F19F65EB72E1CE01019647
:10FEB0000E94019842E350E06FEF7FEFCE01019680
:10FEC0000E948059CE0101960E949E976EEA7FE0C3
:10FED0008FEA92E10E9429976FEA72E1CE010196C2
:10FEE0000E94019844E150E06FEF7FEFCE01019650
:10FEF0000E94FA57CE0101960E949E978BEB88A331
:10FF00008AEA89A381E08AA368011801412C512C57
:10FF10003201C6016AE070E00E94BBB9892B49F446
:10FF200043E050E0BE01605E7F4F86E09FE00E94AC
:10FF3000B38765E070E080E090E00E94F19FBFEF42
:10FF4000CB1ADB0A7801812C912C540186E09FE0CA
:10FF50000E942A88892B39F4E4E08E169104A104CA
:10FF6000B1040CF049C0F6E0EF16F1040CF044C007
:10FF700086E09FE00E942A88892B71F086E09FE04E
:10FF80000E940888E1E0F0E0EC0FFD1FEE0DFF1D80
:10FF900080832FEFE21AF20A65E070E080E090E0E3
:10FFA0000E94F19F36E0E316F10401F5998188A1E2
:10FFB00098131CC09A8189A1981318C09B818AA1AB
:10FFC000981314C08D8190E0B0E0A0E0BA2FA92F63
:10FFD000982F88272C81820F911DA11DB11D480EDD
:10FFE000591E6A1E7B1E4FEF241A340A5FEF851AD2
:10FFF000950AA50AB50AAACF94E02916310434F46B
:020000021000EC
:10000000A0E9CA16A1E0DA0609F083CFC301B20164
:100010000E94ABB420E030E040E251E40E9423B7FC
:1000200020E030E040E85EE30E940AB56B017C010D
:1000300020E030E040EA51E40E942CB818160CF0A1
:1000400055C021E0B701A601CE0101960E94A697F6
:100050006CEF77E0CE0180960E940A98BE016F5F38
:100060007F4FCE0180960E94B8966AE87BE00E949E
:10007000A296BC0185EB92E10E944E97CE0180963C
:100080000E949E97CE0101960E949E9765EB72E1B9
:10009000CE0101960E9401984AE050E070E060E0D5
:1000A000CE0101960E948059CE0101960E949E9732
:1000B00065EB72E1CE0101960E9401986CE57AE051
:1000C000CE0101960E94A2966FEA72E10E94B89654
:1000D000BC0185EB92E10E944E97CE0101960E94F1
:1000E0009E9786E09FE00E94C28D82C962EA7FE00F
:1000F000A2CE6DE670E1CE0101960E94F8974AE02B
:1001000050E06FEF7FEFCE0101960E94FA57CE01CB
:1001100001960E949E976091880470918904809155
:10012000D4049091D5040E94475574E1872E912CF8
:10013000A12CB12CD12CC12CAFEFCA1ADA0AC501FF
:10014000B4010E94F19F60918804709189048091AC
:10015000D4049091D5040E9447557C01B3E0CB169E
:10016000D10434F08EE1C816D10444F4EF2851F0E4
:1001700094E1890E911CA11CB11CDECFE114F104A5
:1001800009F00CC18091D4049091D5048B30910575
:1001900009F0DFC08091131390911413A0911513EF
:1001A000B09116138093FE0B9093FF0BA093000C5D
:1001B000B093010C80910F1390911013A091111323
:1001C000B09112138093FA0B9093FB0BA093FC0B4E
:1001D000B093FD0B4091FE0B5091FF0B6091000C12
:1001E0007091010C21E0CE0101960E94A69766EF66
:1001F00076E0CE0180960E940A98BE016F5F7F4F25
:10020000CE0180960E94B896BC0185EB92E10E94D7
:100210004E97CE0180960E949E97CE0101960E9435
:100220009E974091FA0B5091FB0B6091FC0B7091E3
:10023000FD0B21E0CE0101960E94A69765EB77E0C9
:10024000CE0180960E940A98BE016F5F7F4FCE015B
:1002500080960E94B896BC0185EB92E10E9422979D
:10026000CE0180960E949E97CE0101960E949E9795
:100270006FE47BE085EB92E10E94189764ED7BE0F0
:10028000CE0101960E940A9844E150E070E060E0DF
:10029000CE0101960E948059CE0101960E949E9740
:1002A000C090FE0BD090FF0BE090000CF090010C82
:1002B00020E030E0A901C701B6010E942CB820E07F
:1002C00030E040E05FE387FD64C0C701B6010E94F3
:1002D00045B60E94CFB7AB01BC01CE0101960E948A
:1002E0003495BE016F5F7F4F8FEA92E10E94659760
:1002F000CE0101960E949E9760E087E00E94F48AFA
:100300006FEA72E186EB93E10E94559A6FED86EBFE
:1003100093E10E94DA986BEB77E086EB93E10E9421
:10032000539A6091FA0B7091FB0B8091FC0B9091AA
:10033000FD0B0E94CFB74AE050E086EB93E10E94AC
:10034000069A6FE47BE086EB93E10E94539A0C944B
:100350007F758631910509F41DCF0C9709F03ACFCE
:100360008091F10B9091F20BA091F30BB091F40BF3
:100370008093FE0B9093FF0BA093000CB093010CA5
:100380008091ED0B9091EE0BA091EF0BB091F00BE3
:1003900019CFC701B6010E9444B69BCFEFEFEE160E
:1003A000FE06D4F06FE570E1CE0101960E94F89749
:1003B0004AE050E070E060E0CE0101960E94805972
:1003C000CE0101960E949E976CE370E185EB92E16D
:1003D0000E9429970C944777FEEFEF16FFEFFF0678
:1003E00081F16EE270E1CE0101960E94F8974AE039
:1003F00050E070E060E0CE0101960E948059CE018D
:1004000001960E949E976FE170E185EB92E10E9458
:100410002997B701CE0101960E946195BE016F5FD9
:100420007F4F85EB92E10E942297CE0101960E94B8
:100430009E9769E070E185EB92E10E94CB960C9467
:1004400047776EEF7FE0CE0101960E94F8974AE071
:1004500050E070E060E0CE0101960E948059CE012C
:1004600001960E949E976EED7FE0B0CF809192043E
:10047000882311F40C94477764ED7BE0CE0101965C
:100480000E940A984AE050E061E070E0CE010196D7
:100490000E948059CE0101960E949E970E94246777
:1004A0000C9447778091030D811109C08091AA11A6
:1004B0006EE1462E512C612C712C882329F053E0DB
:1004C000452E512C612C712C6BE770E185EB92E18C
:1004D0000E94299765EB72E1CE0101960E94019876
:1004E0004AE050E06FEF7FEFCE0101960E94FA578D
:1004F000CE0101960E949E97812C912C54011CAE36
:100500001DAE1EAE1FAE83E20E94D98A87E090E046
:100510000E94D48A0E94B49D66E970E080E090E079
:100520000E94F19F83E20E94D98A80E290E00E94BB
:10053000D48A0E94B49D66E970E080E090E00E9459
:10054000F19F62E070E083E290E00E949B9EC12CEC
:10055000D12C76018091290D90912A0D891B990B40
:10056000181619065CF40E94E08DFE2CED2CDC2C94
:10057000CC24C80ED11CE11CF11CECCFC701B60184
:100580000E94ABB42AE939E949E95FE30E9423B745
:100590000E94CFB7AB01BC0184169506A606B7062C
:1005A00014F44A015C01CE0180960E943495BE018C
:1005B000605E7F4FCE0101960E9401986DE87BE05E
:1005C000CE0101960E94A296BC018FEA92E10E94A0
:1005D0004E97CE0101960E949E97CE0180960E9472
:1005E0009E976FEA72E1CE0101960E9401984EE15A
:1005F00050E070E060E0CE0101960E94D658CE0136
:1006000001960E949E972CAD3DAD4EAD5FAD2F5F24
:100610003F4F4F4F5F4F2CAF3DAF4EAF5FAF4216D6
:100620005306640675060CF06ECFB501A401CE0129
:1006300080960E943495BE01605E7F4FCE01019688
:100640000E9401986DE87BE0CE0101960E94A2967F
:10065000BC018FEA92E10E944E97CE0101960E9462
:100660009E97CE0180960E949E976FEA72E1CE011E
:1006700001960E9401984AE050E070E060E0CE01EF
:1006800001960E948059CE0101960E949E97B50165
:10069000A401CE0101960E9434956AE876E0CE016D
:1006A00080960E940A98BE016F5F7F4FCE018096B0
:1006B0000E94B89661E97BE00E94A29665EB72E128
:1006C0000E94B896BC0185EB92E10E944E97CE0144
:1006D00080960E949E97CE0101960E949E9781C9A6
:1006E000E0900202F090030281E08093E60464E669
:1006F00070E080E090E00E94F19F0E94B857C7012F
:100700000E9435170E94CFB720E034E0A901461BB4
:10071000570BBA01CE0101960E94619566E97BE014
:10072000CE0180960E940A98BE016F5F7F4FCE0176
:1007300080960E94B896BC0185EB92E10E944E978C
:10074000CE0180960E949E97CE0101960E949E97B0
:1007500060E087E00E94F48A6BE870E1CE010196C8
:100760000E94F89742E350E068E070E0CE01019605
:100770000E948059CE0101960E949E9765EB72E11E
:10078000CE0101960E94019842E350E06FEF7FEFA7
:10079000CE0101960E94FA57CE0101960E949E97C3
:1007A0006DE97BE0CE0101960E940A9865EB72E14B
:1007B000CE0101960C948F7A8091000290910102F3
:1007C0000E9435170E94CFB77093BE0C6093BD0C8A
:1007D00062E370E080E090E00E94F19F6091BD0CC8
:1007E0007091BE0CCE0101960E946195BE016F5FB3
:1007F0007F4F85EB92E10E946597CE0101960E94A2
:100800009E9780910D1390910E13892B09F45EC071
:1008100069E073E1CE0180960E940198BE01605E9E
:100820007F4FCE0101960E94019844E150E070E0B4
:1008300060E0CE0101960E948059CE0101960E948F
:100840009E9767EA7BE0CE0101960E940A9865EBCD
:1008500072E1CE0101960E94B896BC018FEA92E146
:100860000E944E97CE0101960E949E976FEA72E118
:10087000CE0101960E94019844E150E06FEF7FEFB6
:10088000CE0101960E94FA57CE0101960E949E97D2
:10089000BE01605E7F4FCE0101960E9401986CE51B
:1008A0007AE0CE0101960E94A2966FEA72E10E9460
:1008B000B896BC0185EB92E10E944E97CE0101965D
:1008C0000E949E97CE0180960C94F67962EB7BE0B5
:1008D0008FEA92E10E942A956FEA72E1CE010196B9
:1008E0000E94019844E150E070E060E0CE01019682
:1008F0000E948059CE0101960E949E9766E97BE096
:10090000CE0101960E940A9865EB72E1CE01019634
:100910000E94B896BC018FEA92E10E944E97CE01E8
:1009200001960E949E976FEA72E1CE0101960E94A5
:10093000019844E150E06FEF7FEFCE0101960E94F5
:10094000FA57CE0101960E949E9767EA7BE02ACF74
:1009500080919204882311F40C9447778091030DC1
:10096000811104C08091AA11882331F082E090E0C7
:100970000E94A5680C944777C0908104D0908204AF
:10098000E0908304F090840420E030E040E450E400
:10099000C701B6010E942CB818160CF054C020E014
:1009A00030E04AEF54E4C701B6010E940AB50E9444
:1009B000CFB76B017C010E94B85760E080E00E94D5
:1009C000F48A6CE970E186EB93E10E94759A61E02C
:1009D00080E00E94F48A64E970E186EB93E10E9472
:1009E000759A64E670E080E090E00E94F19F0E94BA
:1009F0008DA66093BF0C7093C00C8093C10C909334
:100A0000C20C0E948DA68090BF0C9090C00CA0904C
:100A1000C10CB090C20C681979098A099B096C1540
:100A20007D058E059F0514F00C94477783E090E0D8
:100A30000E94A5680E948DA664E170E080E090E0CD
:100A40000E94F19FDECF30E3C32E35E7D32EE12C99
:100A5000F12CB1CF0E9437198CEC9DE00E94CD881B
:100A60000C9447776CEB70E18FEA92E10E94299732
:100A70006FEA72E1CE0101960E9401984AE050E0CF
:100A800070E060E0CE0101960E948059CE0101968F
:100A90000E949E97309006028091CF0C811105C074
:100AA0000E948DA681E08093CF0C8091C70C8111AC
:100AB00005C00E948DA681E08093C70C1092EB0BBD
:100AC0001092EA0BE090EA0BF090EB0B58E2E5167F
:100AD000F1040CF07EC0832D0E947C9CF701EE0F88
:100AE000FF1FE35DF24F918380830E94218B20E002
:100AF00030E040EA50E40E940AB520E030E040E8EF
:100B00005AE30E940AB56B017C014090AB045090FF
:100B1000AC046090AD047090AE04A30192016091AA
:100B2000A7047091A8048091A9049091AA040E943E
:100B300044B69B01AC0160E070E080EC90E40E9460
:100B400044B64B015C0120E030E0A9010E94A4B44E
:100B500020E030E040E650E481111CC0C701B6013E
:100B60000E940AB56093C30C7093C40C8093C50CAB
:100B70009093C60C64E170E080E090E00E94F19FE9
:100B80008091EA0B9091EB0B01969093EB0B809385
:100B9000EA0B98CFC701B6010E940AB5A3019201E2
:100BA0000E9445B620E030E040E850E40E9444B6A0
:100BB000A50194010E9423B720E030E040EC50E40E
:100BC0000E940AB520E030E040E850E40E9445B6BB
:100BD000C9CFC090C30CD090C40CE090C50CF0906D
:100BE000C60C20E030E0A901C701B6010E942CB874
:100BF00087FD22C022E0B701A601CE0180960E94A7
:100C0000A69766EB7BE0CE0101960E940A98BE0192
:100C1000605E7F4FCE0101960E94B896BC0185EBC5
:100C200092E10E944E97CE0101960E949E97CE01BE
:100C300080960E949E9706C06DEA70E185EB92E176
:100C40000E94299765EB72E1CE0101960E940198FE
:100C50004AE050E06FEF7FEFCE0101960E94FA5715
:100C60005BC080919204882311F40C9447778091A3
:100C7000030D81112EC08091AA1181112AC0C0904C
:100C80008104D0908204E0908304F090840420E0FA
:100C900030E04AE754E4C701B6010E940AB50E9459
:100CA000CFB74B015C0120E030E040EA50E4C701DF
:100CB000B6010E940AB520E030E040EA50E40E940C
:100CC00045B60E94CFB7A50194010E9450620C94D2
:100CD000477721E030E040E050E06AE070E080E0FB
:100CE00090E0F3CFC7010E943B510C944777C701B6
:100CF0000E9451280C9447778091040D882311F4A9
:100D00000C9447776AE071E1CE0101960E94F89752
:100D1000CE0101960E948457CE0101960E949E97B3
:100D20000C94477780912B0D90912C0D892B81F499
:100D300081E090E090932C0D80932B0D8EE492E057
:100D40000E94F68C68EC70E080E090E00E94F19FD9
:100D50006DEF70E1CE0101960E94F89744E650E0F5
:100D60006FEF7FEFCE0101960E94FA57CE010196F8
:100D70000E949E97F0E0E0E019950C9447770E945E
:100D800023A60E94B8570E94D4150C9447778091EF
:100D9000AF1191E089278093AF11882309F48BC0AC
:100DA00066EF70E185EB92E10E9429970E948DA683
:100DB0006093A6117093A7118093A8119093A91125
:100DC0008091B2119091B311181619065CF420911C
:100DD000B4113091B5112817390724F01092B511CC
:100DE0001092B4119091B6118091B111981724F01E
:100DF0001092B6111092B7118091AF118093AA1181
:100E000065EB72E1CE0101960E9401984AE050E044
:100E100068E070E0CE0101960E948059CE010196F3
:100E20000E949E9761EE70E1CE0101960E94F897B4
:100E30004AE050E06FEF7FEFCE0101960E94FA5733
:100E4000CE0101960E949E9763ED70E185EB92E1E1
:100E50000E94CB9664ED75E0CE0101960E940A983F
:100E600065EB72E1CE0101960E94B896BC0185EB5C
:100E700092E10E944E97CE0101960E949E9780912A
:100E8000030D8093B8118CE291E00E94218D809136
:100E9000030D882311F40C9447776AE878E081EC1D
:100EA00092E10E942A9586EE9FEF9093030C809327
:100EB000020C0C9447776EEE70E185EB92E10E9494
:100EC00029979ACFF092030CE092020C8CEC9DE0F3
:100ED0000E94CD8865EC70E185EB92E10E94299734
:100EE00064ED7BE0CE0101960E940A984AE050E052
:100EF00070E060E0CE0101960E948059CE0101961B
:100F000098CE0E3FFFEF1F0711F40C94FD7464EDB3
:100F10007BE085EB92E10E942A950C94CA7496E0DE
:100F2000899FD0011124AF5CBC4E90967C936E9348
:100F30005F9791E091969C939197E0919E13F09129
:100F40009F1390919D13992339F0309751F081119F
:100F500008C080914D131994309719F05C968C91CC
:100F6000FACF08950895AF92BF92CF92DF92EF9299
:100F7000FF920F931F93CF93DF936C017B018B0143
:100F8000040F151FEB015E01AE18BF08C017D10793
:100F900059F06991D601ED91FC910190F081E02D1D
:100FA000C6011995892B79F7C501DF91CF911F9162
:100FB0000F91FF90EF90DF90CF90BF90AF9008958A
:100FC000FC01A089B1898C91A689B78982FD0FC0E7
:100FD0009C91818D8F5F8F73228D821749F0A18D37
:100FE000AE0FBF2FB11D5D969C93818F08958C919C
:100FF0000895FC01538D448D252F30E0842F90E01F
:10100000821B930B541710F0CF9608950197089503
:10101000FC01918D828D981761F0A28DAE0FBF2FCC
:10102000B11D5D968C91928D9F5F9F73928F90E022
:1010300008958FEF9FEF0895FC01918D828D981791
:1010400031F0828DE80FF11D858D90E008958FEFCE
:101050009FEF0895FC01918D228D892F90E0805C97
:101060009F4F821B91098F73992708958CEC9DE007
:101070000E942A8821E0892B09F420E0822F08951C
:1010800089E69EE00E942A8821E0892B09F420E06D
:10109000822F089586E09FE00E942A8821E0892B14
:1010A00009F420E0822F089583EA9FE00E942A88B5
:1010B00021E0892B09F420E0822F0895FC01A48D02
:1010C000A80FB92FB11DA35ABF4F2C91848D90E06A
:1010D00001968F739927848FA689B7892C93A0894D
:1010E000B1898C91837080648C93938D848D9813D7
:1010F00006C00288F389E02D80818F7D808308956A
:10110000EF92FF920F931F93CF93DF93EC0181E057
:10111000888F9B8D8C8D98131AC0E889F9898081FE
:1011200085FF15C09FB7F894EE89FF896083E88931
:10113000F98980818370806480839FBF81E090E023
:10114000DF91CF911F910F91FF90EF900895F62EB0
:101150000B8D10E00F5F1F4F0F731127E02E8C8D4A
:101160008E110CC00FB607FCFACFE889F98980818F
:1011700085FFF5CFCE010E945E88F1CFEB8DEC0F9D
:10118000FD2FF11DE35AFF4FF0829FB7F8940B8FAC
:10119000EA89FB8980818062CFCFCF93DF93EC0116
:1011A000888D8823B9F0AA89BB89E889F9898C914F
:1011B00085FD03C0808186FD0DC00FB607FCF7CF0B
:1011C0008C9185FFF2CF808185FFEDCFCE010E940B
:1011D0005E88E9CFDF91CF91089580E090E0892B80
:1011E00029F00E94548881110E94000080E090E064
:1011F000892B29F00E944A8881110E94000080E01A
:1012000090E0892B29F00E94408881110E94000003
:1012100080E090E0892B29F00E94368881110C949F
:10122000000008958150823108F05AC0E82FF0E0A4
:101230008827E25EF6478F4F0C94CFB93E894289EA
:10124000308936893A89708945894B894F89558912
:1012500059895D896389678970896B897189758905
:10126000809180008F778093800008958091800026
:101270008F7DF9CF80918000877FF5CF84B58F7700
:1012800084BD089584B58F7DFBCF8091B0008F77AA
:101290008093B00008958091B0008F7DF9CF809148
:1012A00090008F77809390000895809190008F7DBB
:1012B000F9CF80919000877FF5CF8091A0008F7744
:1012C0008093A00008958091A0008F7DF9CF809138
:1012D000A000877FF5CF809120018F778093200138
:1012E0000895809120018F7DF9CF80912001877F23
:1012F000F5CF08958F929F92AF92BF92CF92DF92D7
:10130000EF92FF920F931F93CF93DF93DB01ED9149
:10131000FC91EC01AC85BD8501E010E0EA17FB070C
:101320000CF045C0EF01CC0FDD1FDC011A968D914A
:101330009C91DC01AC0FBD1FAD90BC908F0100955E
:101340001095017011278CE99FEFE0FF02C084E641
:1013500090E0E9016A017B014C01820E931EB40109
:10136000C5010E94601321E030E0892BB9F48C0E96
:101370009D1EB401C5010E94601322E030E0892B5C
:1013800069F4BE01680D791DC5010E94601323E058
:1013900030E0892B19F40FEF1FEF09C0E6018881B7
:1013A000998101968217930784F499838883C801F1
:1013B000DF91CF911F910F91FF90EF90DF90CF9031
:1013C000BF90AF909F908F90089519821882D70197
:1013D0008D919C91119701968D939C93E8CFFB0181
:1013E00001900020E9F73197AF01461B570BDC0154
:1013F000ED91FC910280F381E02D1994CF93DF935E
:10140000EC0188819981009711F00E94BDBA198280
:1014100018821D821C821B821A82DF91CF9108954F
:101420000C94BDBA0F931F93CF93DF93EC01888187
:101430009981009759F02A813B812617370730F0B0
:1014400081E0DF91CF911F910F9108958B016F5F24
:101450007F4F0E9446BB009759F0998388831B8376
:101460000A832C813D81232B59F7FC011082E8CFA0
:1014700080E0E7CFEF92FF920F931F93CF93DF931C
:101480006115710541F480E0DF91CF911F910F91BB
:10149000FF90EF90089541155105B1F07B01EC01EB
:1014A0000C811D81040F151FB8010E94128A882328
:1014B00051F3288139818C819D81B701820F931F5F
:1014C0000E945FBC1D830C8381E0DECFEF92FF9210
:1014D0000F931F93CF93DF93EC017B018A01BA0135
:1014E0000E94128A81110BC0CE010E94FE89CE019A
:1014F000DF91CF911F910F91FF90EF9008951D8381
:101500000C83B701888199810E945FBCF0CF0F9353
:101510001F93CF93DF938C01EB0188E2FB011192C3
:101520008A95E9F74BE050E06AEB7BE0CE010E9440
:1015300074BC1B8681E090E0A0E0B0E08C879D87C2
:10154000AE87BF87F80185899689A789B08D888B7A
:10155000998BAA8BBB8B82E090E0A0E0B0E08C8BF3
:101560009D8BAE8BBF8B1CA21DA21EA21FA280E072
:1015700090E0A8E4B4E4888F998FAA8FBB8F80E0B5
:1015800090E0A8E4B4EC8C8F9D8FAE8FBF8F8DEC74
:101590009CECACE4BEE388A399A3AAA3BBA3DF9110
:1015A000CF911F910F910895682F80E490E10C94E2
:1015B000FD0B91E09093A90D8093CB131092AA0D8F
:1015C0001092CB0D0895CF93C82F682F607F86EBC4
:1015D00093E10E94841280E1C89FB001112486EB40
:1015E00093E1CF910C948412CF93DF9300D000D07D
:1015F0001F921F92CDB7DEB798E0E1E6F5E0DE017D
:10160000119601900D929A95E1F79091BF1396175C
:1016100008F46FEF70E0660F771F21E030E02C0FC9
:101620003D1F620F731FFB019081890F8068289610
:101630000FB6F894DEBF0FBECDBFDF91CF910C94F3
:10164000E38A2F923F924F925F926F927F928F9296
:101650009F92AF92BF92CF92DF92EF92FF920F9341
:101660001F93CF93DF9300D000D000D01F92CDB74F
:10167000DEB780902D0D90902E0D80912F0D9091C2
:10168000300D881699062CF4382F292FC401832E8B
:10169000922E01E31DE02DE73DE040E050E0BA016D
:1016A000D801CD90DD908D01C816D9060CF06DC023
:1016B000092E000CAA0BBB0B480F591F6A1F7B1F7A
:1016C000C6012017310761F7CB01BA010E94ABB404
:1016D00020E030E048E152E40E9423B76B017C0136
:1016E000EDE2FDE0FA87E987812C912C5401A98570
:1016F000BA856D917D91BA87A987072E000C880B5A
:10170000990B0E94ABB4A70196010E9444B69B01BD
:10171000AC010E940AB59B01AC01C501B4010E9455
:1017200045B64B015C01E985FA850E171F07F9F6EE
:1017300020E030E04CE152E40E9423B70E944DB912
:101740004B015C0120E030E040E85FE30E942CB8F0
:1017500018168CF1C701B6012A960FB6F894DEBFB1
:101760000FBECDBFDF91CF911F910F91FF90EF90F2
:10177000DF90CF90BF90AF909F908F907F906F90B1
:101780005F904F903F902F9008958C149D0454F4D7
:10179000092C000CAA08BB08480D591D6A1D7B1DA9
:1017A00046018FCF0D2C000CEE08FF084C0D5D1D7F
:1017B0006E1D7F1D86CF8DE2282E8DE0382E10E025
:1017C00000E019821A821B821C82D1018D919D91A9
:1017D0001D019C01990F440B550B2D833E834F83B4
:1017E0005887CA01B9010E94ABB4A70196010E94B3
:1017F00044B62B013C0120E030E0A9010E942CB846
:10180000181624F077FA709477F87094A501940173
:10181000C301B2010E94A4B487FF12C089819A81DA
:10182000AB81BC812D813E814F815885820F931FF2
:10183000A41FB51F89839A83AB83BC830F5F1F4F9F
:1018400049855A854215530509F0BFCF20E030E0A5
:1018500040EC5FE3C501B4010E940AB54B015C0195
:10186000053011050CF4A7CF69817A818B819C81A9
:101870000E94ABB46B017C01B801110F880B990B6E
:101880000E94ABB49B01AC01C701B6010E9423B713
:101890006B017C015FCF4F925F926F927F928F922C
:1018A0009F92AF92BF92CF92DF92EF92FF920F93EF
:1018B0001F93CF93DF9300D000D01F921F92CDB71C
:1018C000DEB72B013C01FF24F3940F2D10E0C8017B
:1018D000880F991F880F991F9A838983FC01EB5FFA
:1018E000FA4F80809180A280B380A3019201C5014C
:1018F000B4010E94A4B487FF02C0F394E6CFA9818B
:10190000BA81A351BB4FCD90DD90ED90FC90A30127
:101910009201C501B4010E94A4B4882309F44DC00A
:101920000150104C000F111F000F111FF801EB5F49
:10193000FA4F80819181A281B38189839A83AB839D
:10194000BC8303511B4FD8018D919D910D90BC918B
:10195000A02D8D839E83AF83B88729813A814B81E7
:101960005C81C301B2010E9444B62B013C012D8170
:101970003E814F815885C701B6010E9444B69B0144
:10198000AC01C301B2010E940AB56B017C0129813F
:101990003A814B815C81C501B4010E9444B69B0130
:1019A000AC01C701B6010E9423B72D813E814F8152
:1019B00058850E9445B66B017C01C701B601289687
:1019C0000FB6F894DEBF0FBECDBFDF91CF911F9150
:1019D0000F91FF90EF90DF90CF90BF90AF909F90CE
:1019E0008F907F906F905F904F900895EF92FF924D
:1019F0000F931F93CF93DF931F921F92CDB7DEB744
:101A00008C019A8389838BE2E82E8DE0F82EF70112
:101A10006081CE0101960E946D580F5F1F4F1A839F
:101A20000983F7016181CE0101960E946D58C701BB
:101A30000F900F90DF91CF911F910F91FF90EF903A
:101A40000895EF92FF920F931F93CF93DF931F920E
:101A50001F92CDB7DEB70FEA11E18F5A91417C0199
:101A6000C701800F911F9A838983F80161918F01CB
:101A7000CE0101960E946D58F1E1093B1F0781F7E5
:101A80008FEA91E10F900F90DF91CF911F910F910D
:101A9000FF90EF900895EF92FF920F931F93CF93D3
:101AA000DF931F921F92CDB7DEB70EE111E18E5189
:101AB00091417C01C701800F911F9A838983F801AE
:101AC00061918F01CE0101960E946D58F1E1063AB5
:101AD0001F0781F78EE191E10F900F90DF91CF9179
:101AE0001F910F91FF90EF9008950F931F93CF9345
:101AF000DF93FC01048115810115110539F4FB0107
:101B00001082DF91CF911F910F910895415051099B
:101B10004017510708F48A01EB01FC0160817181D3
:101B2000A801CE010E9474BCC00FD11F1882E9CF5A
:101B3000EF92FF920F931F93CF93DF931F921F9209
:101B4000CDB7DEB70FEA11E18F5A91417C01C70191
:101B5000800F911F9A838983F80161918F01CE01D3
:101B600001960E946D58F2E1093A1F0781F78FEA4A
:101B700091E10F900F90DF91CF911F910F91FF9006
:101B8000EF900895CF93DF93EC010E94CD88EA890E
:101B9000FB8980818F7E8083EA89FB898081877FB2
:101BA0008083EA89FB8980818F778083EA89FB893A
:101BB00080818F7D80838A8D898FDF91CF91089579
:101BC00090912A0D8091290D2FEF3FEF981748F43F
:101BD000E92FF0E0E75FF24F208130E09F5F9093C4
:101BE0002A0DC90108952F923F924F925F926F92F2
:101BF0007F928F929F92AF92BF92CF92DF92EF929D
:101C0000FF920F931F93CF93DF9300D000D01F92CA
